******************************************************************************
                  TI ARM Linker PC v5.1.6                      
******************************************************************************
>> Linked Fri Jan 12 16:33:29 2018

OUTPUT FILE NAME:   <blefi.out>
ENTRY POINT SYMBOL: "_c_int00"  address: 20022029


MEMORY CONFIGURATION

         name            origin    length      used     unused   attr    fill
----------------------  --------  ---------  --------  --------  ----  --------
  SRAM_CODE             20004000   00027eff  00023620  000048df  RW X
  SRAM_DATA             2002bf00   00012eff  0001221e  00000ce1  RW X


SEGMENT ALLOCATION MAP

run origin  load origin   length   init length attrs members
----------  ----------- ---------- ----------- ----- -------
20004000    20004000    00023628   00023628    r-x
  20004000    20004000    0000030c   0000030c    r-- .resetVecs
  2000430c    2000430c    0001fe3e   0001fe3e    r-x .text
  2002414c    2002414c    000027c6   000027c6    r-- .const
  20026918    20026918    00000d10   00000d10    r-- .cinit
2002bf00    2002bf00    00010220   00000000    rw-
  2002bf00    2002bf00    0000f2de   00000000    rw- .bss
  2003b1e0    2003b1e0    00000f40   00000000    rw- .data
2003cdfc    2003cdfc    00002000   00000000    rw-
  2003cdfc    2003cdfc    00002000   00000000    rw- .stack


SECTION ALLOCATION MAP

 output                                  attributes/
section   page    origin      length       input sections
--------  ----  ----------  ----------   ----------------
.bootVecs 
*          0    00000000    00000008     DSECT
                  00000000    00000008     boot.aem4 : boot.oem4 (.bootVecs)

xdc.meta   0    00000000    000000f8     COPY SECTION
                  00000000    000000f8     app_pem4.oem4 (xdc.meta)

.init_array 
*          0    20004000    00000000     UNINITIALIZED

.vecs      0    20004000    00000000     DSECT

.resetVecs 
*          0    20004000    0000030c     
                  20004000    0000030c     app_pem4.oem4 (.resetVecs)

.text      0    2000430c    0001fe3e     
                  2000430c    000025c4     mqtt.a : mqtt_client.obj (.text)
                  200068d0    00001854     mqtt_app.a : device_mqtt.obj (.text)
                  20008124    00001324                : mqtt_app_main.obj (.text)
                  20009448    000011c0     http.obj (.text)
                  2000a608    00000fa0     gateway.a : database.obj (.text)
                  2000b5a8    00000ec0     rtsv7M4_T_le_eabi.lib : _printfi.obj (.text)
                  2000c468    00000cc0     cli.a : cli_handler.obj (.text)
                  2000d128    00000c7c           : cli.obj (.text)
                  2000dda4    00000c3c     cc26xxdnld.obj (.text)
                  2000e9e0    00000bbe     wifi.obj (.text)
                  2000f59e    00000a0a     mqtt.a : mqtt_common.obj (.text)
                  2000ffa8    00000970            : sl_mqtt_client.obj (.text)
                  20010918    00000818     gateway.a : gapbondmgr.obj (.text)
                  20011130    00000732     cc3200.obj (.text)
                  20011862    00000002     app_pem4.oem4 (.text:ti_sysbios_BIOS_nullFunc__I)
                  20011864    00000708     schema.a : schema.obj (.text)
                  20011f6c    000006c4     mqtt.a : cc31xx_sl_net.obj (.text)
                  20012630    0000068c     gateway.a : gateway_events.obj (.text)
                  20012cbc    00000610     ota.a : OtaHttp.obj (.text)
                  200132cc    000005f0     gateway.a : gateway_task.obj (.text)
                  200138bc    000005f0     json.a : jsmn.obj (.text)
                  20013eac    000005ec     simplelink.a : driver.obj (.text:_SlDrvMsgRead)
                  20014498    000005d0     generic_task.obj (.text)
                  20014a68    000005cc     gateway.a : gateway_api.obj (.text)
                  20015034    000005c8     otatask.obj (.text)
                  200155fc    000005ac     npi.a : gap_packets.obj (.text)
                  20015ba8    00000544     ti_rtos.a : osi_tirtos.obj (.text)
                  200160ec    000004f4     mqtt_app.a : CC2650_SensorTag.obj (.text)
                  200165e0    00000478     npi.a : gatt.obj (.text)
                  20016a58    00000428           : gap.obj (.text)
                  20016e80    00000424     ota.a : OtaClient.obj (.text)
                  200172a4    00000424     sysbios.aem4 : BIOS.obj (.text:ti_sysbios_family_arm_m3_Hwi_excDumpRegs__I)
                  200176c8    0000040c     ota.a : OtaApp.obj (.text)
                  20017ad4    00000370     npi.a : uart_def.obj (.text)
                  20017e44    0000035c     ota.a : CdnClient.obj (.text)
                  200181a0    00000356     uart_if.obj (.text)
                  200184f6    00000002     sysbios.aem4 : BIOS.obj (.text:ti_sysbios_gates_GateHwi_Instance_init__E)
                  200184f8    0000033c     ti.targets.arm.rtsarm.aem4 : System.oem4 (.text:xdc_runtime_System_doPrint__I)
                  20018834    00000338     ota.a : LogClient.obj (.text)
                  20018b6c    0000032c     npi.a : npi_cc3200_if.obj (.text)
                  20018e98    00000304     sysbios.aem4 : BIOS.obj (.text:ti_sysbios_knl_Semaphore_pend__E)
                  2001919c    000002d4     rtsv7M4_T_le_eabi.lib : trgdrv.obj (.text)
                  20019470    00000270     simplelink.a : wlan.obj (.text:sl_WlanProfileAdd)
                  200196e0    00000248                  : driver.obj (.text:_SlDrvRxHdrRead)
                  20019928    00000248     sysbios.aem4 : BIOS.obj (.text:ti_sysbios_heaps_HeapMem_free__E)
                  20019b70    00000244     simplelink.a : wlan.obj (.text:sl_WlanConnect)
                  20019db4    00000234     sysbios.aem4 : BIOS.obj (.text:ti_sysbios_heaps_HeapMem_alloc__E)
                  20019fe8    00000228                  : BIOS.obj (.text:ti_sysbios_knl_Task_Instance_finalize__E)
                  2001a210    00000220     gateway.a : gateway_cmds.obj (.text)
                  2001a430    00000208     sysbios.aem4 : BIOS.obj (.text:ti_sysbios_knl_Task_sleep__E)
                  2001a638    000001f8                  : BIOS.obj (.text:ti_sysbios_family_arm_m3_Hwi_excHandlerMax__I)
                  2001a830    000001f4     rtsv7M4_T_le_eabi.lib : ull_div_t2.obj (.text)
                  2001aa24    000001e0     gateway.a : ble_central.obj (.text)
                  2001ac04    000001d0     simplelink.a : driver.obj (.text:_SlDrvReleasePoolObj)
                  2001add4    000001cc                  : driver.obj (.text:_SlDrvMsgWrite)
                  2001afa0    000001bc     sysbios.aem4 : BIOS.obj (.text:ti_sysbios_knl_Task_Instance_init__E)
                  2001b15c    000001b6     rtsv7M4_T_le_eabi.lib : fd_add_t2.obj (.text)
                  2001b312    00000002     app_pem4.oem4 (.text:xdc_runtime_Startup_reset__I)
                  2001b314    00000190     simplelink.a : driver.obj (.text:_SlDrvWaitForPoolObj)
                  2001b4a4    0000018c     sysbios.aem4 : BIOS.obj (.text:ti_sysbios_knl_Task_Module_startup__E)
                  2001b630    00000184     flc.a : flc.obj (.text)
                  2001b7b4    00000184     main.obj (.text)
                  2001b938    00000174     simplelink.a : driver.obj (.text:_SlDrvDriverCBInit)
                  2001baac    00000170                  : driver.obj (.text:_SlFindAndSetActiveObj)
                  2001bc1c    00000168     sysbios.aem4 : BIOS.obj (.text:ti_sysbios_family_arm_m3_Hwi_excBusFault__I)
                  2001bd84    00000160                  : BIOS.obj (.text:ti_sysbios_knl_Mailbox_Instance_init__E)
                  2001bee4    00000154                  : BIOS.obj (.text:ti_sysbios_family_arm_m3_Hwi_excUsageFault__I)
                  2001c038    00000150     simplelink.a : cc_pal.obj (.text:spi_Open)
                  2001c188    00000140     sysbios.aem4 : BIOS.obj (.text:ti_sysbios_family_arm_m3_Hwi_excMemFault__I)
                  2001c2c8    0000013c     simplelink.a : socket.obj (.text:sl_Select)
                  2001c404    0000013c     sysbios.aem4 : BIOS.obj (.text:ti_sysbios_family_arm_m3_Hwi_dispatchC__I)
                  2001c540    00000138     simplelink.a : socket.obj (.text:sl_Accept)
                  2001c678    00000138     sysbios.aem4 : BIOS.obj (.text:ti_sysbios_heaps_HeapMem_Instance_init__E)
                  2001c7b0    00000138                  : BIOS.obj (.text:ti_sysbios_knl_Semaphore_post__E)
                  2001c8e8    00000136     rtsv7M4_T_le_eabi.lib : fd_div_t2.obj (.text)
                  2001ca1e    00000002     --HOLE-- [fill = 0]
                  2001ca20    00000134     driverlib.a : prcm.obj (.text:PRCMCC3200MCUInit)
                  2001cb54    00000130     ti.targets.arm.rtsarm.aem4 : LoggerBuf.oem4 (.text:xdc_runtime_LoggerBuf_write8__E)
                  2001cc84    0000012c     sysbios.aem4 : BIOS.obj (.text:ti_sysbios_knl_Clock_workFunc__E)
                  2001cdb0    00000128     simplelink.a : driver.obj (.text:_SlDrvDataReadOp)
                  2001ced8    00000120     sysbios.aem4 : BIOS.obj (.text:ti_sysbios_knl_Swi_run__I)
                  2001cff8    00000120     ti.targets.arm.rtsarm.aem4 : Error.oem4 (.text:xdc_runtime_Error_policyDefault__E)
                  2001d118    00000118     simplelink.a : socket.obj (.text:sl_SendTo)
                  2001d230    00000110     rtsv7M4_T_le_eabi.lib : strtoul.obj (.text)
                  2001d340    0000010c     pinmux.obj (.text)
                  2001d44c    0000010c     simplelink.a : socket.obj (.text:sl_RecvFrom)
                  2001d558    00000108                  : socket.obj (.text:sl_Connect)
                  2001d660    00000108                  : socket.obj (.text:sl_Send)
                  2001d768    00000104                  : driver.obj (.text:_SlDrvDataWriteOp)
                  2001d86c    00000104                  : netapp.obj (.text:sl_NetAppDnsGetHostByName)
                  2001d970    00000104     ti.targets.arm.rtsarm.aem4 : Core-mem.oem4 (.text:xdc_runtime_Core_createObject__I)
                  2001da74    00000104     app_pem4.oem4 (.text:xdc_runtime_System_printfExtend__I)
                  2001db78    000000fe     simplelink.a : netapp.obj (.text:_SlDrvNetAppEventHandler)
                  2001dc76    000000fc     rtsv7M4_T_le_eabi.lib : fd_mul_t2.obj (.text)
                  2001dd72    00000002     --HOLE-- [fill = 0]
                  2001dd74    000000fc     ti.targets.arm.rtsarm.aem4 : Startup.oem4 (.text:xdc_runtime_Startup_startMods__I)
                  2001de70    000000f4     simplelink.a : fs.obj (.text:sl_FsRead)
                  2001df64    000000f0     driverlib.a : udma.obj (.text:uDMAChannelTransferSet)
                  2001e054    000000ec     simplelink.a : fs.obj (.text:sl_FsWrite)
                  2001e140    000000dc                  : cc_pal.obj (.text:spi_Read)
                  2001e21c    000000d8                  : driver.obj (.text:_SlDrvClassifyRxMsg)
                  2001e2f4    000000d4     ti.targets.arm.rtsarm.aem4 : LoggerBuf.oem4 (.text:xdc_runtime_LoggerBuf_write4__E)
                  2001e3c8    000000d2     smartconfig.obj (.text)
                  2001e49a    00000002     --HOLE-- [fill = 0]
                  2001e49c    000000d0     sysbios.aem4 : m3_Hwi_asm.obj (.text:ti_sysbios_family_arm_m3_Hwi_dispatch__I)
                  2001e56c    000000cc     ti.targets.arm.rtsarm.aem4 : Core-smem.oem4 (.text:xdc_runtime_Core_constructObject__I)
                  2001e638    000000c8     simplelink.a : netapp.obj (.text:_sl_HandleAsync_DnsGetHostByService)
                  2001e700    000000c8     sysbios.aem4 : BIOS.obj (.text:ti_sysbios_knl_Task_schedule__I)
                  2001e7c8    000000c4                  : BIOS.obj (.text:ti_sysbios_family_arm_m3_Hwi_Module_startup__E)
                  2001e88c    000000c0     simplelink.a : driver.obj (.text:_SlRemoveFromList)
                  2001e94c    000000c0     sysbios.aem4 : BIOS.obj (.text:ti_sysbios_knl_Task_exit__E)
                  2001ea0c    000000bc     simplelink.a : driver.obj (.text:_SlDrvMsgReadCmdCtx)
                  2001eac8    000000bc                  : device.obj (.text:sl_Start)
                  2001eb84    000000bc     sysbios.aem4 : BIOS.obj (.text:ti_sysbios_knl_Task_startCore__E)
                  2001ec40    000000b8     simplelink.a : driver.obj (.text:_SlAsyncEventGenericHandler)
                  2001ecf8    000000b4     sysbios.aem4 : BIOS.obj (.text:ti_sysbios_family_arm_m3_Hwi_excHardFault__I)
                  2001edac    000000b4                  : BIOS.obj (.text:ti_sysbios_gates_GateMutex_enter__E)
                  2001ee60    000000b4                  : BIOS.obj (.text:ti_sysbios_knl_Task_checkStacks__E)
                  2001ef14    000000b0     npi.a : ble_events.obj (.text)
                  2001efc4    000000b0     sysbios.aem4 : BIOS.obj (.text:ti_sysbios_family_arm_m3_Hwi_excDebugMon__I)
                  2001f074    000000a8     driverlib.a : interrupt.obj (.text:IntDisable)
                  2001f11c    000000a8                 : interrupt.obj (.text:IntEnable)
                  2001f1c4    000000a8     simplelink.a : netcfg.obj (.text:sl_NetCfgGet)
                  2001f26c    000000a8     sysbios.aem4 : BIOS.obj (.text:ti_sysbios_knl_Swi_post__E)
                  2001f314    000000a8                  : BIOS.obj (.text:ti_sysbios_knl_Task_blockI__E)
                  2001f3bc    000000a8                  : BIOS.obj (.text:ti_sysbios_knl_Task_postInit__I)
                  2001f464    000000a8                  : BIOS.obj (.text:ti_sysbios_knl_Task_yield__E)
                  2001f50c    000000a0     driverlib.a : spi.obj (.text:SPIConfigSetExpClk)
                  2001f5ac    000000a0     auto_init.aem4 : auto_init.oem4 (.text)
                  2001f64c    0000009c     simplelink.a : driver.obj (.text:_SlDrvMsgReadSpawnCtx)
                  2001f6e8    0000009c     rtsv7M4_T_le_eabi.lib : memcpy_t2.obj (.text)
                  2001f784    0000009c     sysbios.aem4 : BIOS.obj (.text:ti_sysbios_family_arm_m3_Hwi_Instance_init__E)
                  2001f820    0000009c                  : BIOS.obj (.text:ti_sysbios_knl_Semaphore_Instance_init__E)
                  2001f8bc    0000009a     ti.targets.arm.rtsarm.aem4 : Text.oem4 (.text:xdc_runtime_Text_putSite__E)
                  2001f956    00000002     --HOLE-- [fill = 0]
                  2001f958    00000098     simplelink.a : fs.obj (.text:_sl_GetCreateFsMode)
                  2001f9f0    00000094     driverlib.a : prcm.obj (.text:PRCMPeripheralClockGet)
                  2001fa84    00000094     sysbios.aem4 : BIOS.obj (.text:ti_sysbios_knl_Mailbox_post__E)
                  2001fb18    00000094                  : BIOS.obj (.text:ti_sysbios_knl_Task_unblockI__E)
                  2001fbac    00000094     ti.targets.arm.rtsarm.aem4 : Text.oem4 (.text:xdc_runtime_Text_putMod__E)
                  2001fc40    00000090     simplelink.a : wlan.obj (.text:sl_WlanSmartConfigStart)
                  2001fcd0    0000008c                  : cc_pal.obj (.text:SetupDMAReceive)
                  2001fd5c    0000008c                  : cc_pal.obj (.text:SetupDMASend)
                  2001fde8    0000008c                  : netapp.obj (.text:_sl_HandleAsync_DnsGetHostByName)
                  2001fe74    0000008c                  : netapp.obj (.text:_sl_HandleAsync_PingResponse)
                  2001ff00    0000008c                  : cc_pal.obj (.text:spi_Write)
                  2001ff8c    00000088     driverlib.a : prcm.obj (.text:PRCMHibernateIntervalSet)
                  20020014    00000088                 : pin.obj (.text:PinConfigSet)
                  2002009c    00000088     rtsv7M4_T_le_eabi.lib : vsnprintf.obj (.text)
                  20020124    00000088     simplelink.a : socket.obj (.text:sl_Bind)
                  200201ac    00000088                  : fs.obj (.text:sl_FsClose)
                  20020234    00000088     sysbios.aem4 : BIOS.obj (.text:ti_sysbios_knl_Mailbox_Module_startup__E)
                  200202bc    00000086     rtsv7M4_T_le_eabi.lib : fd_cmp_t2.obj (.text:__aeabi_cdcmple)
                  20020342    00000086                           : fd_cmp_t2.obj (.text:__aeabi_cdrcmple)
                  200203c8    00000084     simplelink.a : cc_pal.obj (.text:NwpPowerOnPreamble)
                  2002044c    00000084     sysbios.aem4 : BIOS.obj (.text:ti_sysbios_family_arm_m3_Hwi_initNVIC__E)
                  200204d0    00000084                  : BIOS.obj (.text:ti_sysbios_knl_Mailbox_pend__E)
                  20020554    00000082     driverlib.a : gpio.obj (.text:GPIOIntTypeSet)
                  200205d6    00000002     --HOLE-- [fill = 0]
                  200205d8    00000080     simplelink.a : driver.obj (.text:_SlDrvCmdOp)
                  20020658    00000080                  : cc_pal.obj (.text:spi_Read_CPU)
                  200206d8    00000080                  : cc_pal.obj (.text:spi_Write_CPU)
                  20020758    00000080     ti.targets.arm.rtsarm.aem4 : LoggerBuf.oem4 (.text:xdc_runtime_LoggerBuf_setFilterLevel__E)
                  200207d8    0000007c     driverlib.a : prcm.obj (.text:PRCMRTCGet)
                  20020854    0000007c     simplelink.a : device.obj (.text:_sl_HandleAsync_InitComplete)
                  200208d0    0000007c                  : fs.obj (.text:sl_FsGetInfo)
                  2002094c    00000078                  : socket.obj (.text:_sl_HandleAsync_Connect)
                  200209c4    00000078     rtsv7M4_T_le_eabi.lib : memset_t2.obj (.text)
                  20020a3c    00000078     simplelink.a : fs.obj (.text:sl_FsOpen)
                  20020ab4    00000076     driverlib.a : uart.obj (.text:UARTConfigSetExpClk)
                  20020b2a    00000002     --HOLE-- [fill = 0]
                  20020b2c    00000074     simplelink.a : socket.obj (.text:sl_Recv)
                  20020ba0    00000070     sysbios.aem4 : BIOS.obj (.text:ti_sysbios_family_arm_m3_Hwi_postInit__I)
                  20020c10    00000070                  : BIOS.obj (.text:ti_sysbios_knl_Mailbox_Instance_finalize__E)
                  20020c80    00000070     ti.targets.arm.rtsarm.aem4 : Memory.oem4 (.text:xdc_runtime_Memory_alloc__E)
                  20020cf0    0000006c     simplelink.a : driver.obj (.text:_SlDrvCmdSend)
                  20020d5c    0000006c     ti.targets.arm.rtsarm.aem4 : Error.oem4 (.text:xdc_runtime_Error_print__E)
                  20020dc8    0000006c                                : LoggerBuf.oem4 (.text:xdc_runtime_LoggerBuf_getFilterLevel__E)
                  20020e34    00000068     simplelink.a : netapp.obj (.text:_sl_NetAppSendTokenValue)
                  20020e9c    00000068                  : socket.obj (.text:sl_SetSockOpt)
                  20020f04    00000066     ti.targets.arm.rtsarm.aem4 : Core-mem.oem4 (.text:xdc_runtime_Core_deleteObject__I)
                  20020f6a    00000002     --HOLE-- [fill = 0]
                  20020f6c    00000064     app_pem4.oem4 (.text:ti_sysbios_family_arm_m3_Hwi_create)
                  20020fd0    00000064     app_pem4.oem4 (.text:ti_sysbios_knl_Mailbox_create)
                  20021034    00000064     driverlib.a : udma.obj (.text:uDMAChannelAttributeDisable)
                  20021098    00000064                 : udma.obj (.text:uDMAChannelAttributeEnable)
                  200210fc    00000060     simplelink.a : socket.obj (.text:_sl_HandleAsync_Accept)
                  2002115c    00000060     npi.a : hci.obj (.text)
                  200211bc    00000060     rtsv7M4_T_le_eabi.lib : sprintf.obj (.text)
                  2002121c    00000060                           : trgmsg.obj (.text)
                  2002127c    00000060     simplelink.a : wlan.obj (.text:sl_WlanPolicySet)
                  200212dc    00000060     sysbios.aem4 : BIOS.obj (.text:ti_sysbios_family_arm_m3_TimestampProvider_get64__E)
                  2002133c    00000060                  : BIOS.obj (.text:ti_sysbios_knl_Clock_logTick__E)
                  2002139c    00000060     ti.targets.arm.rtsarm.aem4 : System.oem4 (.text:xdc_runtime_System_formatNum__I)
                  200213fc    0000005e     rtsv7M4_T_le_eabi.lib : copy_decompress_rle.obj (.text)
                  2002145a    00000002     --HOLE-- [fill = 0]
                  2002145c    0000005c     simplelink.a : socket.obj (.text:sl_Socket)
                  200214b8    0000005c     sysbios.aem4 : BIOS.obj (.text:ti_sysbios_family_arm_m3_Timer_setPeriod__E)
                  20021514    0000005c     app_pem4.oem4 (.text:ti_sysbios_knl_Task_create)
                  20021570    0000005c     app_pem4.oem4 (.text:xdc_runtime_LoggerBuf_Object__create__S)
                  200215cc    0000005b     ti.targets.arm.rtsarm.aem4 : Text.oem4 (.text:xdc_runtime_Text_putLab__E)
                  20021627    00000001     --HOLE-- [fill = 0]
                  20021628    0000005a     rtsv7M4_T_le_eabi.lib : ltoa.obj (.text)
                  20021682    00000002     --HOLE-- [fill = 0]
                  20021684    00000058     driverlib.a : interrupt.obj (.text:IntPendClear)
                  200216dc    00000058                 : prcm.obj (.text:PRCMPeripheralReset)
                  20021734    00000058     sysbios.aem4 : BIOS.obj (.text:ti_sysbios_knl_Swi_restoreHwi__E)
                  2002178c    00000058                  : BIOS.obj (.text:ti_sysbios_knl_Swi_schedule__I)
                  200217e4    00000054     simplelink.a : socket.obj (.text:_sl_HandleAsync_Select)
                  20021838    00000054     sysbios.aem4 : BIOS.obj (.text:ti_sysbios_family_arm_m3_Timer_start__E)
                  2002188c    00000050     driverlib.a : prcm.obj (.text:PRCMSlowClkCtrGet)
                  200218dc    00000050     simplelink.a : device.obj (.text:_sl_HandleAsync_Stop)
                  2002192c    00000050                  : fs.obj (.text:sl_FsDel)
                  2002197c    00000050     ti.targets.arm.rtsarm.aem4 : Startup.oem4 (.text:xdc_runtime_Startup_exec__E)
                  200219cc    00000050                                : Text.oem4 (.text:xdc_runtime_Text_visitRope2__I)
                  20021a1c    0000004c     driverlib.a : spi.obj (.text:SPIIntEnable)
                  20021a68    0000004c     simplelink.a : driver.obj (.text:_SlDrvProtectAsyncRespSetting)
                  20021ab4    0000004c                  : driver.obj (.text:_SlDrvRxIrqHandler)
                  20021b00    0000004c                  : socket.obj (.text:_sl_BuildAddress)
                  20021b4c    0000004c     rtsv7M4_T_le_eabi.lib : atoi.obj (.text)
                  20021b98    0000004c                           : atol.obj (.text)
                  20021be4    0000004c     sysbios.aem4 : m3_TaskSupport_asm.obj (.text:ti_sysbios_family_arm_m3_TaskSupport_buildTaskStack)
                  20021c30    0000004c                  : BIOS.obj (.text:ti_sysbios_knl_Swi_runLoop__I)
                  20021c7c    0000004c     driverlib.a : udma.obj (.text:uDMAChannelAssign)
                  20021cc8    0000004a     cli.a : conversions.obj (.text)
                  20021d12    00000002     --HOLE-- [fill = 0]
                  20021d14    00000048     driverlib.a : prcm.obj (.text:PRCMHibernateWakeupSourceEnable)
                  20021d5c    00000048                 : spi.obj (.text:SPIIntClear)
                  20021da4    00000048     simplelink.a : driver.obj (.text:_SlDrvBasicCmd)
                  20021dec    00000048     rtsv7M4_T_le_eabi.lib : fd_toi_t2.obj (.text)
                  20021e34    00000048     sysbios.aem4 : BIOS.obj (.text:ti_sysbios_family_arm_m3_Hwi_excReserved__I)
                  20021e7c    00000048                  : m3_Hwi_asm_switch.obj (.text:ti_sysbios_family_arm_m3_Hwi_initStacks__E)
                  20021ec4    00000048                  : BIOS.obj (.text:ti_sysbios_family_arm_m3_Timer_initDevice__I)
                  20021f0c    00000048                  : BIOS.obj (.text:ti_sysbios_heaps_HeapMem_getStats__E)
                  20021f54    00000048     ti.targets.arm.rtsarm.aem4 : Assert.oem4 (.text:xdc_runtime_Assert_raise__I)
                  20021f9c    00000046                                : Core-params.oem4 (.text:xdc_runtime_Core_assignParams__I)
                  20021fe2    00000002     --HOLE-- [fill = 0]
                  20021fe4    00000044     driverlib.a : spi.obj (.text:SPIDmaMaskGet)
                  20022028    00000044     boot.aem4 : boot.oem4 (.text)
                  2002206c    00000044     simplelink.a : cc_pal.obj (.text:cc_SetupTransfer)
                  200220b0    00000044     rtsv7M4_T_le_eabi.lib : cpy_tbl.obj (.text)
                  200220f4    00000044                           : exit.obj (.text)
                  20022138    00000044                           : xdtest.obj (.text)
                  2002217c    00000044     sysbios.aem4 : BIOS.obj (.text:ti_sysbios_family_arm_m3_Hwi_disableInterrupt__E)
                  200221c0    00000044                  : BIOS.obj (.text:ti_sysbios_family_arm_m3_Hwi_enableInterrupt__E)
                  20022204    00000044                  : BIOS.obj (.text:ti_sysbios_knl_Task_allBlockedFunction__I)
                  20022248    00000044     ti.targets.arm.rtsarm.aem4 : Error.oem4 (.text:xdc_runtime_Error_setX__E)
                  2002228c    00000044                                : LoggerBuf.oem4 (.text:xdc_runtime_LoggerBuf_filterOutEvent__I)
                  200222d0    00000044                                : SysMin.oem4 (.text:xdc_runtime_SysMin_flush__E)
                  20022314    00000042     rtsv7M4_T_le_eabi.lib : u_divt2.obj (.text)
                  20022356    00000042     simplelink.a : socket.obj (.text:sl_Htonl)
                  20022398    00000040     driverlib.a : pin.obj (.text:PinModeSet)
                  200223d8    00000040     rtsv7M4_T_le_eabi.lib : strtok.obj (.text)
                  20022418    00000040     sysbios.aem4 : BIOS.obj (.text:ti_sysbios_family_arm_m3_Timer_Module_startup__E)
                  20022458    00000040                  : BIOS.obj (.text:ti_sysbios_knl_Mailbox_postInit__I)
                  20022498    0000003e     app_pem4.oem4 (.text:realloc)
                  200224d6    0000003c     simplelink.a : netapp.obj (.text:CopyPingResultsToReport)
                  20022512    00000002     --HOLE-- [fill = 0]
                  20022514    0000003c     driverlib.a : prcm.obj (.text:PRCMPeripheralClkEnable)
                  20022550    0000003c     simplelink.a : socket.obj (.text:_sl_TruncatePayloadByProtocol)
                  2002258c    0000003c                  : socket.obj (.text:sl_Htons)
                  200225c8    0000003c                  : socket.obj (.text:sl_Listen)
                  20022604    0000003c     sysbios.aem4 : BIOS.obj (.text:ti_sysbios_family_arm_m3_Hwi_excSvCall__I)
                  20022640    0000003c                  : BIOS.obj (.text:ti_sysbios_heaps_HeapMem_init__I)
                  2002267c    0000003c                  : BIOS.obj (.text:ti_sysbios_knl_Swi_startup__E)
                  200226b8    0000003c     driverlib.a : udma.obj (.text:uDMAChannelControlSet)
                  200226f4    0000003c     ti.targets.arm.rtsarm.aem4 : Text.oem4 (.text:xdc_runtime_Text_xprintf__I)
                  20022730    0000003a                                : LoggerBuf.oem4 (.text:xdc_runtime_LoggerBuf_Instance_init__E)
                  2002276a    00000002     --HOLE-- [fill = 0]
                  2002276c    00000038     simplelink.a : cc_pal.obj (.text:NwpPowerOff)
                  200227a4    00000038     sysbios.aem4 : BIOS.obj (.text:ti_sysbios_family_arm_m3_Hwi_excNoIsr__I)
                  200227dc    00000038                  : BIOS.obj (.text:ti_sysbios_family_arm_m3_Hwi_getStackInfo__E)
                  20022814    00000038                  : BIOS.obj (.text:ti_sysbios_family_arm_m3_TaskSupport_start__E)
                  2002284c    00000038                  : BIOS.obj (.text:ti_sysbios_knl_Task_processVitalTaskFlag__I)
                  20022884    00000038     ti.targets.arm.rtsarm.aem4 : SysMin.oem4 (.text:xdc_runtime_SysMin_putch__E)
                  200228bc    00000038                                : System.oem4 (.text:xdc_runtime_System_atexit__E)
                  200228f4    00000036     driverlib.a : gpio.obj (.text:GPIODirModeSet)
                  2002292a    00000002     --HOLE-- [fill = 0]
                  2002292c    00000034                 : prcm.obj (.text:PRCMPeripheralStatusGet)
                  20022960    00000034                 : spi.obj (.text:SPIFIFOLevelSet)
                  20022994    00000034     rtsv7M4_T_le_eabi.lib : strstr.obj (.text)
                  200229c8    00000034     sysbios.aem4 : BIOS.obj (.text:ti_sysbios_family_arm_m3_Hwi_excNmi__I)
                  200229fc    00000034                  : BIOS.obj (.text:ti_sysbios_family_arm_m3_Timer_periodicStub__I)
                  20022a30    00000034                  : BIOS.obj (.text:ti_sysbios_hal_Hwi_checkStack)
                  20022a64    00000034     app_pem4.oem4 (.text:ti_sysbios_knl_Semaphore_create)
                  20022a98    00000034     ti.targets.arm.rtsarm.aem4 : Core-label.oem4 (.text:xdc_runtime_Core_assignLabel__I)
                  20022acc    00000033                                : Text.oem4 (.text:xdc_runtime_Text_printVisFxn__I)
                  20022aff    00000001     --HOLE-- [fill = 0]
                  20022b00    00000032     sysbios.aem4 : BIOS.obj (.text:ti_sysbios_knl_Semaphore_pendTimeout__I)
                  20022b32    00000030     driverlib.a : pin.obj (.text:PinTypeGPIO)
                  20022b62    00000002     --HOLE-- [fill = 0]
                  20022b64    00000030                 : uart.obj (.text:UARTDisable)
                  20022b94    00000030     simplelink.a : device.obj (.text:_SlDrvDeviceEventHandler)
                  20022bc4    00000030                  : fs.obj (.text:_sl_Strlen)
                  20022bf4    00000030     rtsv7M4_T_le_eabi.lib : strncpy.obj (.text)
                  20022c24    00000030     simplelink.a : socket.obj (.text:sl_Close)
                  20022c54    00000030     app_pem4.oem4 (.text:ti_sysbios_BIOS_atExitFunc__I)
                  20022c84    00000030     app_pem4.oem4 (.text:ti_sysbios_gates_GateHwi_Object__create__S)
                  20022cb4    00000030     app_pem4.oem4 (.text:ti_sysbios_gates_GateMutex_Object__create__S)
                  20022ce4    00000030     app_pem4.oem4 (.text:ti_sysbios_heaps_HeapMem_Object__create__S)
                  20022d14    00000030     app_pem4.oem4 (.text:ti_sysbios_knl_Semaphore_construct)
                  20022d44    00000030     ti.targets.arm.rtsarm.aem4 : SysMin.oem4 (.text:xdc_runtime_SysMin_abort__E)
                  20022d74    00000030                                : System.oem4 (.text:xdc_runtime_System_processAtExit__E)
                  20022da4    0000002e     app_pem4.oem4 (.text:malloc)
                  20022dd2    0000002e     rtsv7M4_T_le_eabi.lib : i_tofd_t2.obj (.text)
                  20022e00    0000002c     simplelink.a : cc_pal.obj (.text:DmaSpiSwIntHandler)
                  20022e2c    0000002c                  : cc_pal.obj (.text:NwpPowerOn)
                  20022e58    0000002c     driverlib.a : prcm.obj (.text:PRCMSysResetCauseGet)
                  20022e84    0000002c     sysbios.aem4 : BIOS.obj (.text:ti_sysbios_family_arm_m3_Hwi_Instance_finalize__E)
                  20022eb0    0000002c                  : BIOS.obj (.text:ti_sysbios_hal_Hwi_initStack)
                  20022edc    0000002c     app_pem4.oem4 (.text:ti_sysbios_knl_Clock_doTick__I)
                  20022f08    0000002c     app_pem4.oem4 (.text:ti_sysbios_knl_Queue_construct)
                  20022f34    0000002c     sysbios.aem4 : BIOS.obj (.text:ti_sysbios_knl_Task_restore__E)
                  20022f60    0000002c     ti.targets.arm.rtsarm.aem4 : Text.oem4 (.text:xdc_runtime_Text_cordText__E)
                  20022f8c    0000002a     rtsv7M4_T_le_eabi.lib : strspn.obj (.text)
                  20022fb6    0000002a     ti.targets.arm.rtsarm.aem4 : System.oem4 (.text:xdc_runtime_System_putchar__I)
                  20022fe0    00000028     driverlib.a : prcm.obj (.text:IsRTCUsed)
                  20023008    00000028                 : prcm.obj (.text:PRCMPeripheralClkDisable)
                  20023030    00000028     simplelink.a : socket.obj (.text:SL_FD_ISSET)
                  20023058    00000028     ti.targets.arm.rtsarm.aem4 : LoggerBuf.oem4 (.text:xdc_runtime_LoggerBuf_Module_startup__E)
                  20023080    00000026     simplelink.a : cc_pal.obj (.text:NwpRegisterInterruptHandler)
                  200230a6    00000026     rtsv7M4_T_le_eabi.lib : strncmp.obj (.text)
                  200230cc    00000026     ti.targets.arm.rtsarm.aem4 : System.oem4 (.text:xdc_runtime_System_avprintf__E)
                  200230f2    00000002     --HOLE-- [fill = 0]
                  200230f4    00000024     driverlib.a : prcm.obj (.text:RTCU16MSecRegRead)
                  20023118    00000024                 : prcm.obj (.text:RTCUseSet)
                  2002313c    00000024                 : uart.obj (.text:UARTEnable)
                  20023160    00000024     simplelink.a : driver.obj (.text:_SlDrvProtectionObjLockWaitForever)
                  20023184    00000024     rtsv7M4_T_le_eabi.lib : memmov.obj (.text)
                  200231a8    00000024     app_pem4.oem4 (.text:ti_sysbios_BIOS_errorRaiseHook__I)
                  200231cc    00000024     app_pem4.oem4 (.text:ti_sysbios_BIOS_registerRTSLock__I)
                  200231f0    00000024     app_pem4.oem4 (.text:ti_sysbios_BIOS_removeRTSLock__I)
                  20023214    00000024     app_pem4.oem4 (.text:ti_sysbios_BIOS_startFunc__I)
                  20023238    00000024     sysbios.aem4 : BIOS.obj (.text:ti_sysbios_family_arm_m3_Hwi_doTaskRestore__I)
                  2002325c    00000024                  : BIOS.obj (.text:ti_sysbios_family_arm_m3_Timer_startup__E)
                  20023280    00000024     app_pem4.oem4 (.text:ti_sysbios_gates_GateMutex_Object__delete__S)
                  200232a4    00000024     sysbios.aem4 : BIOS.obj (.text:ti_sysbios_knl_Clock_Module_startup__E)
                  200232c8    00000024     app_pem4.oem4 (.text:ti_sysbios_knl_Semaphore_Object__delete__S)
                  200232ec    00000024     sysbios.aem4 : BIOS.obj (.text:ti_sysbios_knl_Swi_Module_startup__E)
                  20023310    00000024     ti.targets.arm.rtsarm.aem4 : System.oem4 (.text:xdc_runtime_System_vprintf__E)
                  20023334    00000022     driverlib.a : gpio.obj (.text:GPIOIntStatus)
                  20023356    00000022     simplelink.a : socket.obj (.text:SL_FD_SET)
                  20023378    00000022     driverlib.a : spi.obj (.text:SPIReset)
                  2002339a    00000022                 : spi.obj (.text:SPIWordCountSet)
                  200233bc    00000022     rtsv7M4_T_le_eabi.lib : memcmp.obj (.text)
                  200233de    00000022                           : strcspn.obj (.text)
                  20023400    00000022     app_pem4.oem4 (.text:xdc_runtime_SysMin_output__I)
                  20023422    00000020     driverlib.a : gpio.obj (.text:GPIOPinWrite)
                  20023442    00000020                 : spi.obj (.text:SPIDataGet)
                  20023462    00000002     --HOLE-- [fill = 0]
                  20023464    00000020     simplelink.a : driver.obj (.text:_SlDrvProtectionObjUnLock)
                  20023484    00000020     mqtt.a : cc3200_platform.obj (.text)
                  200234a4    00000020     app_pem4.oem4 (.text:ti_sysbios_family_arm_m3_Hwi_Object__delete__S)
                  200234c4    00000020     sysbios.aem4 : m3_Hwi_asm.obj (.text:ti_sysbios_family_arm_m3_Hwi_excHandlerAsm__I)
                  200234e4    00000020                  : BIOS.obj (.text:ti_sysbios_family_arm_m3_Hwi_excHandler__I)
                  20023504    00000020                  : BIOS.obj (.text:ti_sysbios_family_arm_m3_TimestampProvider_Module_startup__E)
                  20023524    00000020     app_pem4.oem4 (.text:ti_sysbios_gates_GateHwi_Object__delete__S)
                  20023544    00000020     app_pem4.oem4 (.text:ti_sysbios_heaps_HeapMem_Object__delete__S)
                  20023564    00000020     sysbios.aem4 : BIOS.obj (.text:ti_sysbios_knl_Idle_run__E)
                  20023584    00000020     app_pem4.oem4 (.text:ti_sysbios_knl_Mailbox_Object__delete__S)
                  200235a4    00000020     app_pem4.oem4 (.text:ti_sysbios_knl_Semaphore_Object__destruct__S)
                  200235c4    00000020     app_pem4.oem4 (.text:ti_sysbios_knl_Task_Object__delete__S)
                  200235e4    00000020     sysbios.aem4 : BIOS.obj (.text:ti_sysbios_knl_Task_enter__I)
                  20023604    00000020     app_pem4.oem4 (.text:xdc_runtime_LoggerBuf_Object__delete__S)
                  20023624    00000020     ti.targets.arm.rtsarm.aem4 : LoggerBuf.oem4 (.text:xdc_runtime_LoggerBuf_reset__E)
                  20023644    00000020                                : Registry.oem4 (.text:xdc_runtime_Registry_findById__E)
                  20023664    00000020                                : SysMin.oem4 (.text:xdc_runtime_SysMin_Module_startup__E)
                  20023684    0000001e     driverlib.a : spi.obj (.text:SPIDataPut)
                  200236a2    0000001e                 : uart.obj (.text:UARTCharPut)
                  200236c0    0000001e     simplelink.a : cc_pal.obj (.text:cc_UDMAChannelSelect)
                  200236de    0000001e     sysbios.aem4 : m3_Hwi_asm_switch.obj (.text:ti_sysbios_family_xxx_Hwi_switchAndRunFunc)
                  200236fc    0000001c     driverlib.a : uart.obj (.text:UARTCharGetNonBlocking)
                  20023718    0000001c     simplelink.a : driver.obj (.text:_SlDrvObjLockWaitForever)
                  20023734    0000001c                  : driver.obj (.text:_SlDrvSyncObjWaitForever)
                  20023750    0000001c     rtsv7M4_T_le_eabi.lib : memccpy.obj (.text)
                  2002376c    0000001c     app_pem4.oem4 (.text:ti_sysbios_BIOS_rtsLock__I)
                  20023788    0000001c     sysbios.aem4 : BIOS.obj (.text:ti_sysbios_family_arm_m3_Hwi_setPriority__E)
                  200237a4    0000001c                  : BIOS.obj (.text:ti_sysbios_gates_GateMutex_Instance_init__E)
                  200237c0    0000001c     app_pem4.oem4 (.text:ti_sysbios_knl_Queue_Object__destruct__S)
                  200237dc    0000001c     driverlib.a : udma.obj (.text:uDMAChannelEnable)
                  200237f8    0000001c     ti.targets.arm.rtsarm.aem4 : Error.oem4 (.text:xdc_runtime_Error_raiseX__E)
                  20023814    0000001c                                : Memory.oem4 (.text:xdc_runtime_Memory_valloc__E)
                  20023830    0000001c                                : SysMin.oem4 (.text:xdc_runtime_SysMin_exit__E)
                  2002384c    0000001c                                : System.oem4 (.text:xdc_runtime_System_abort__E)
                  20023868    0000001a     driverlib.a : gpio.obj (.text:GPIOIntDisable)
                  20023882    0000001a                 : gpio.obj (.text:GPIOIntEnable)
                  2002389c    0000001a                 : pin.obj (.text:PinTypeUART)
                  200238b6    0000001a                 : spi.obj (.text:SPIDmaEnable)
                  200238d0    0000001a                 : spi.obj (.text:SPIFIFOEnable)
                  200238ea    0000001a     rtsv7M4_T_le_eabi.lib : strcat.obj (.text)
                  20023904    0000001a     app_pem4.oem4 (.text:ti_sysbios_family_arm_m3_Hwi_Handle__label__S)
                  2002391e    0000001a     sysbios.aem4 : m3_Hwi_asm.obj (.text:ti_sysbios_family_arm_m3_Hwi_pendSV__I)
                  20023938    0000001a     app_pem4.oem4 (.text:ti_sysbios_gates_GateHwi_Handle__label__S)
                  20023952    0000001a     app_pem4.oem4 (.text:ti_sysbios_gates_GateMutex_Handle__label__S)
                  2002396c    0000001a     app_pem4.oem4 (.text:ti_sysbios_heaps_HeapMem_Handle__label__S)
                  20023986    0000001a     app_pem4.oem4 (.text:ti_sysbios_knl_Swi_Handle__label__S)
                  200239a0    0000001a     app_pem4.oem4 (.text:ti_sysbios_knl_Task_Handle__label__S)
                  200239ba    0000001a     sysbios.aem4 : BIOS.obj (.text:ti_sysbios_knl_Task_sleepTimeout__I)
                  200239d4    0000001a     app_pem4.oem4 (.text:xdc_runtime_LoggerBuf_Handle__label__S)
                  200239ee    0000001a     app_pem4.oem4 (.text:xdc_runtime_System_aprintf__E)
                  20023a08    0000001a     app_pem4.oem4 (.text:xdc_runtime_System_printf__E)
                  20023a22    00000018     driverlib.a : gpio.obj (.text:GPIOPinRead)
                  20023a3a    00000002     --HOLE-- [fill = 0]
                  20023a3c    00000018                 : prcm.obj (.text:PRCMHibernateEnter)
                  20023a54    00000018                 : spi.obj (.text:SPICSDisable)
                  20023a6c    00000018                 : spi.obj (.text:SPICSEnable)
                  20023a84    00000018                 : spi.obj (.text:SPIDisable)
                  20023a9c    00000018                 : spi.obj (.text:SPIEnable)
                  20023ab4    00000018                 : uart.obj (.text:UARTCharsAvail)
                  20023acc    00000018                 : uart.obj (.text:UARTFIFOLevelSet)
                  20023ae4    00000018                 : uart.obj (.text:UARTIntDisable)
                  20023afc    00000018                 : uart.obj (.text:UARTIntEnable)
                  20023b14    00000018     simplelink.a : driver.obj (.text:_SlDrvObjUnLock)
                  20023b2c    00000018                  : driver.obj (.text:_SlDrvSyncObjSignal)
                  20023b44    00000018                  : device.obj (.text:_sl_GetStartResponseConvert)
                  20023b5c    00000018     app_pem4.oem4 (.text:free)
                  20023b74    00000018     rtsv7M4_T_le_eabi.lib : args_main.obj (.text)
                  20023b8c    00000018                           : ll_mul_t2.obj (.text)
                  20023ba4    00000018                           : strcmp.obj (.text)
                  20023bbc    00000018     app_pem4.oem4 (.text:ti_sysbios_BIOS_rtsUnlock__I)
                  20023bd4    00000018     app_pem4.oem4 (.text:ti_sysbios_family_arm_m3_Hwi_Module__startupDone__F)
                  20023bec    00000018     app_pem4.oem4 (.text:ti_sysbios_family_arm_m3_Timer_Module__startupDone__F)
                  20023c04    00000018     sysbios.aem4 : BIOS.obj (.text:ti_sysbios_gates_GateMutex_leave__E)
                  20023c1c    00000018     ti.targets.arm.rtsarm.aem4 : Error.oem4 (.text:xdc_runtime_Error_check__E)
                  20023c34    00000018                                : System.oem4 (.text:xdc_runtime_System_exit__E)
                  20023c4c    00000018                                : Text.oem4 (.text:xdc_runtime_Text_ropeText__E)
                  20023c64    00000016     driverlib.a : prcm.obj (.text:PRCMHIBRegRead)
                  20023c7a    00000016                 : prcm.obj (.text:PRCMHIBRegWrite)
                  20023c90    00000016                 : uart.obj (.text:UARTCharGet)
                  20023ca6    00000016     simplelink.a : driver.obj (.text:_SlDrvMemZero)
                  20023cbc    00000016     app_pem4.oem4 (.text:ti_sysbios_BIOS_exitFunc__I)
                  20023cd2    00000014     driverlib.a : cpu.obj (.text:CPUcpsie)
                  20023ce6    00000014                 : gpio.obj (.text:GPIOIntClear)
                  20023cfa    00000002     --HOLE-- [fill = 0]
                  20023cfc    00000014     rtsv7M4_T_le_eabi.lib : _lock.obj (.text)
                  20023d10    00000014                           : strlen.obj (.text)
                  20023d24    00000014     app_pem4.oem4 (.text:ti_sysbios_family_arm_m3_Hwi_Object__get__S)
                  20023d38    00000014     sysbios.aem4 : BIOS.obj (.text:ti_sysbios_family_arm_m3_Hwi_switchFromBootStack__E)
                  20023d4c    00000014     app_pem4.oem4 (.text:ti_sysbios_heaps_HeapMem_Object__get__S)
                  20023d60    00000014     app_pem4.oem4 (.text:ti_sysbios_knl_Swi_Object__get__S)
                  20023d74    00000014     app_pem4.oem4 (.text:xdc_runtime_LoggerBuf_Object__get__S)
                  20023d88    00000012     driverlib.a : uart.obj (.text:UARTIntClear)
                  20023d9a    00000012     rtsv7M4_T_le_eabi.lib : copy_zero_init.obj (.text:decompress:ZI)
                  20023dac    00000012     sysbios.aem4 : BIOS.obj (.text:ti_sysbios_hal_Hwi_Module_startup__E)
                  20023dbe    00000012                  : BIOS.obj (.text:ti_sysbios_hal_Timer_Module_startup__E)
                  20023dd0    00000012     ti.targets.arm.rtsarm.aem4 : LoggerBuf.oem4 (.text:xdc_runtime_LoggerBuf_Instance_finalize__E)
                  20023de2    00000012                                : LoggerBuf.oem4 (.text:xdc_runtime_LoggerBuf_write1__E)
                  20023df4    00000012                                : LoggerBuf.oem4 (.text:xdc_runtime_LoggerBuf_write2__E)
                  20023e06    00000012     app_pem4.oem4 (.text:xdc_runtime_Startup_exec__I)
                  20023e18    00000010     driverlib.a : prcm.obj (.text:RTCU32SecRegRead)
                  20023e28    00000010     simplelink.a : socket.obj (.text:SL_FD_ZERO)
                  20023e38    00000010     rtsv7M4_T_le_eabi.lib : strcpy.obj (.text)
                  20023e48    00000010     sysbios.aem4 : BIOS.obj (.text:ti_sysbios_BIOS_setThreadType__E)
                  20023e58    00000010                  : BIOS.obj (.text:ti_sysbios_BIOS_start__E)
                  20023e68    00000010                  : BIOS.obj (.text:ti_sysbios_family_arm_m3_Hwi_getHandle__E)
                  20023e78    00000010                  : m3_TaskSupport_asm.obj (.text:ti_sysbios_family_arm_m3_TaskSupport_glue)
                  20023e88    00000010                  : m3_TaskSupport_asm.obj (.text:ti_sysbios_family_arm_m3_TaskSupport_swap__E)
                  20023e98    00000010                  : BIOS.obj (.text:ti_sysbios_gates_GateMutex_Instance_finalize__E)
                  20023ea8    00000010     app_pem4.oem4 (.text:ti_sysbios_knl_Mailbox_Object__get__S)
                  20023eb8    00000010     sysbios.aem4 : BIOS.obj (.text:ti_sysbios_knl_Semaphore_Instance_finalize__E)
                  20023ec8    00000010                  : BIOS.obj (.text:ti_sysbios_knl_Swi_disable__E)
                  20023ed8    00000010     app_pem4.oem4 (.text:ti_sysbios_knl_Task_Object__get__S)
                  20023ee8    00000010     sysbios.aem4 : BIOS.obj (.text:ti_sysbios_knl_Task_disable__E)
                  20023ef8    00000010     ti.targets.arm.rtsarm.aem4 : Gate.oem4 (.text:xdc_runtime_Gate_leaveSystem__E)
                  20023f08    00000010                                : LoggerBuf.oem4 (.text:xdc_runtime_LoggerBuf_write0__E)
                  20023f18    00000010                                : Memory.oem4 (.text:xdc_runtime_Memory_free__E)
                  20023f28    00000010                                : SysMin.oem4 (.text:xdc_runtime_SysMin_ready__E)
                  20023f38    00000010                                : System.oem4 (.text:xdc_runtime_System_vsnprintf__E)
                  20023f48    00000010     app_pem4.oem4 (.text:xdc_runtime_Text_visitRope__I)
                  20023f58    0000000e     simplelink.a : driver.obj (.text:_SlDrvResetCmdExt)
                  20023f66    0000000e     rtsv7M4_T_le_eabi.lib : copy_decompress_none.obj (.text:decompress:none)
                  20023f74    0000000e                           : xdclass.obj (.text)
                  20023f82    0000000e     sysbios.aem4 : BIOS.obj (.text:ti_sysbios_knl_Queue_empty__E)
                  20023f90    0000000c     simplelink.a : cc_pal.obj (.text:NwpMaskInterrupt)
                  20023f9c    0000000c                  : cc_pal.obj (.text:NwpUnMaskInterrupt)
                  20023fa8    0000000c                  : wlan.obj (.text:sl_WlanDisconnect)
                  20023fb4    0000000c                  : wlan.obj (.text:sl_WlanSmartConfigStop)
                  20023fc0    0000000c     app_pem4.oem4 (.text:ti_sysbios_family_arm_m3_Hwi_Params__init__S)
                  20023fcc    0000000c     sysbios.aem4 : BIOS.obj (.text:ti_sysbios_family_arm_m3_Hwi_disableFxn__E)
                  20023fd8    0000000c                  : BIOS.obj (.text:ti_sysbios_family_arm_m3_TaskSupport_checkStack__E)
                  20023fe4    0000000c                  : BIOS.obj (.text:ti_sysbios_family_arm_m3_TaskSupport_getStackAlignment__E)
                  20023ff0    0000000c                  : BIOS.obj (.text:ti_sysbios_gates_GateHwi_enter__E)
                  20023ffc    0000000c     app_pem4.oem4 (.text:ti_sysbios_knl_Queue_Object__get__S)
                  20024008    0000000c     app_pem4.oem4 (.text:ti_sysbios_knl_Semaphore_Params__init__S)
                  20024014    0000000c     app_pem4.oem4 (.text:ti_sysbios_knl_Task_Params__init__S)
                  20024020    0000000c     ti.targets.arm.rtsarm.aem4 : Error.oem4 (.text:xdc_runtime_Error_init__E)
                  2002402c    0000000c                                : Gate.oem4 (.text:xdc_runtime_Gate_enterSystem__E)
                  20024038    0000000c                                : Memory.oem4 (.text:xdc_runtime_Memory_calloc__E)
                  20024044    0000000c                                : Memory.oem4 (.text:xdc_runtime_Memory_getMaxDefaultTypeAlign__E)
                  20024050    0000000a     driverlib.a : interrupt.obj (.text:IntMasterEnable)
                  2002405a    0000000a     app_pem4.oem4 (.text:xdc_runtime_IHeap_alloc)
                  20024064    0000000a     app_pem4.oem4 (.text:xdc_runtime_IHeap_free)
                  2002406e    0000000a     ti.targets.arm.rtsarm.aem4 : LoggerBuf.oem4 (.text:xdc_runtime_LoggerBuf_disable__E)
                  20024078    0000000a                                : LoggerBuf.oem4 (.text:xdc_runtime_LoggerBuf_enable__E)
                  20024082    00000008     driverlib.a : prcm.obj (.text:PRCMRTCInUseSet)
                  2002408a    00000008     sysbios.aem4 : BIOS.obj (.text:ti_sysbios_family_arm_m3_Hwi_doSwiRestore__I)
                  20024092    00000008                  : BIOS.obj (.text:ti_sysbios_family_arm_m3_Hwi_startup__E)
                  2002409a    00000008                  : BIOS.obj (.text:ti_sysbios_knl_Idle_loop__E)
                  200240a2    00000006     driverlib.a : utils.obj (.text:UtilsDelay)
                  200240a8    00000006     ti.targets.arm.rtsarm.aem4 : xdc_noinit.oem4 (.text:__xdc__init)
                  200240ae    00000006     rtsv7M4_T_le_eabi.lib : copy_decompress_rle.obj (.text:decompress:rle24)
                  200240b4    00000006     sysbios.aem4 : BIOS.obj (.text:ti_sysbios_family_arm_m3_Hwi_restoreFxn__E)
                  200240ba    00000006                  : BIOS.obj (.text:ti_sysbios_gates_GateHwi_leave__E)
                  200240c0    00000006                  : BIOS.obj (.text:ti_sysbios_heaps_HeapMem_isBlocking__E)
                  200240c6    00000006                  : BIOS.obj (.text:ti_sysbios_knl_Queue_Instance_init__E)
                  200240cc    00000006     ti.targets.arm.rtsarm.aem4 : System.oem4 (.text:xdc_runtime_System_Module_startup__E)
                  200240d2    00000004                                : LoggerBuf.oem4 (.text:LoggerBuf_instanceStartup)
                  200240d6    00000004     app_pem4.oem4 (.text:ti_sysbios_BIOS_RtsGateProxy_enter__E)
                  200240da    00000004     app_pem4.oem4 (.text:ti_sysbios_BIOS_RtsGateProxy_leave__E)
                  200240de    00000004     app_pem4.oem4 (.text:ti_sysbios_family_arm_m3_Hwi_delete)
                  200240e2    00000004     app_pem4.oem4 (.text:ti_sysbios_family_arm_m3_TaskSupport_Module__startupDone__S)
                  200240e6    00000004     sysbios.aem4 : BIOS.obj (.text:ti_sysbios_family_arm_m3_Timer_getMaxTicks__E)
                  200240ea    00000004                  : BIOS.obj (.text:ti_sysbios_gates_GateHwi_query__E)
                  200240ee    00000004                  : BIOS.obj (.text:ti_sysbios_gates_GateMutex_query__E)
                  200240f2    00000004     app_pem4.oem4 (.text:ti_sysbios_hal_Hwi_HwiProxy_Module__startupDone__S)
                  200240f6    00000004     app_pem4.oem4 (.text:ti_sysbios_hal_Timer_TimerProxy_Module__startupDone__S)
                  200240fa    00000004     app_pem4.oem4 (.text:ti_sysbios_heaps_HeapMem_Module_GateProxy_enter__E)
                  200240fe    00000004     app_pem4.oem4 (.text:ti_sysbios_heaps_HeapMem_Module_GateProxy_leave__E)
                  20024102    00000004     app_pem4.oem4 (.text:ti_sysbios_knl_Clock_TimerProxy_Module__startupDone__S)
                  20024106    00000004     app_pem4.oem4 (.text:ti_sysbios_knl_Clock_TimerProxy_getMaxTicks__E)
                  2002410a    00000004     app_pem4.oem4 (.text:ti_sysbios_knl_Mailbox_delete)
                  2002410e    00000004     app_pem4.oem4 (.text:ti_sysbios_knl_Queue_destruct)
                  20024112    00000004     app_pem4.oem4 (.text:ti_sysbios_knl_Semaphore_delete)
                  20024116    00000004     app_pem4.oem4 (.text:ti_sysbios_knl_Semaphore_destruct)
                  2002411a    00000004     app_pem4.oem4 (.text:ti_sysbios_knl_Task_SupportProxy_Module__startupDone__S)
                  2002411e    00000004     app_pem4.oem4 (.text:ti_sysbios_knl_Task_delete)
                  20024122    00000004     sysbios.aem4 : BIOS.obj (.text:ti_sysbios_knl_Task_startup__E)
                  20024126    00000004     ti.targets.arm.rtsarm.aem4 : Error.oem4 (.text:xdc_runtime_Error_getSite__E)
                  2002412a    00000004     app_pem4.oem4 (.text:xdc_runtime_LoggerBuf_Module_GateProxy_enter__E)
                  2002412e    00000004     app_pem4.oem4 (.text:xdc_runtime_LoggerBuf_Module_GateProxy_leave__E)
                  20024132    00000004     app_pem4.oem4 (.text:xdc_runtime_Memory_HeapProxy_alloc__E)
                  20024136    00000004     app_pem4.oem4 (.text:xdc_runtime_Memory_HeapProxy_free__E)
                  2002413a    00000004     app_pem4.oem4 (.text:xdc_runtime_System_Module_GateProxy_enter__E)
                  2002413e    00000004     app_pem4.oem4 (.text:xdc_runtime_System_Module_GateProxy_leave__E)
                  20024142    00000004     ti.targets.arm.rtsarm.aem4 : System.oem4 (.text:xdc_runtime_System_aprintf_va__F)
                  20024146    00000004                                : System.oem4 (.text:xdc_runtime_System_printf_va__F)

.const     0    2002414c    000027c6     
                  2002414c    0000178e     app_pem4.oem4 (.const:xdc_runtime_Text_charTab__A)
                  200258da    00000102     rtsv7M4_T_le_eabi.lib : ctype.obj (.const:.string:_ctypes_)
                  200259dc    00000100     driverlib.a : pin.obj (.const:g_ulPinToPadMap)
                  20025adc    000000f8     mqtt_app.a : mqtt_app_main.obj (.const:.string)
                  20025bd4    000000be                : device_mqtt.obj (.const:.string)
                  20025c92    000000b8     app_pem4.oem4 (.const:xdc_runtime_Text_nodeTab__A)
                  20025d4a    00000002     app_pem4.oem4 (.const:ti_sysbios_family_arm_m3_Hwi_Module__id__C)
                  20025d4c    000000b0     simplelink.a : wlan.obj (.const:$P$T0$1)
                  20025dfc    000000a8     driverlib.a : prcm.obj (.const:PRCM_PeriphRegsList)
                  20025ea4    00000080                 : interrupt.obj (.const)
                  20025f24    00000048     app_pem4.oem4 (.const:.string)
                  20025f6c    00000040     cc26xxdnld.obj (.const:$P$T0$1)
                  20025fac    0000003c     simplelink.a : driver.obj (.const:OpcodeTranslateTable)
                  20025fe8    0000003c                  : wlan.obj (.const)
                  20026024    0000003c     app_pem4.oem4 (.const:ti_sysbios_knl_Task_Object__PARAMS__C)
                  20026060    0000003c     app_pem4.oem4 (.const:xdc_runtime_LoggerBuf_Module__FXNS__C)
                  2002609c    00000038     wifi.obj (.const:.string)
                  200260d4    00000038     simplelink.a : driver.obj (.const:_SlActionLookupTable)
                  2002610c    00000038                  : fs.obj (.const)
                  20026144    00000034                  : driver.obj (.const)
                  20026178    00000034                  : socket.obj (.const)
                  200261ac    00000034     app_pem4.oem4 (.const:ti_sysbios_knl_Mailbox_Object__PARAMS__C)
                  200261e0    00000030     app_pem4.oem4 (.const:ti_sysbios_family_arm_m3_Hwi_Object__PARAMS__C)
                  20026210    00000030     app_pem4.oem4 (.const:xdc_runtime_Startup_sfxnTab__A)
                  20026240    0000002f     gateway.a : gateway_events.obj (.const:.string)
                  2002626f    0000002d     npi.a : uart_def.obj (.const:.string)
                  2002629c    00000028     simplelink.a : netapp.obj (.const)
                  200262c4    00000028     app_pem4.oem4 (.const:ti_sysbios_heaps_HeapMem_Module__FXNS__C)
                  200262ec    00000026     mqtt_app.a : CC2650_SensorTag.obj (.const:.string)
                  20026312    00000002     app_pem4.oem4 (.const:ti_sysbios_family_arm_m3_Hwi_Module__loggerDefined__C)
                  20026314    00000024     app_pem4.oem4 (.const:ti_sysbios_gates_GateHwi_Module__FXNS__C)
                  20026338    00000024     app_pem4.oem4 (.const:ti_sysbios_gates_GateMutex_Module__FXNS__C)
                  2002635c    00000024     app_pem4.oem4 (.const:ti_sysbios_heaps_HeapMem_Object__PARAMS__C)
                  20026380    00000024     app_pem4.oem4 (.const:ti_sysbios_knl_Semaphore_Object__PARAMS__C)
                  200263a4    00000024     app_pem4.oem4 (.const:xdc_runtime_LoggerBuf_Object__PARAMS__C)
                  200263c8    00000023     smartconfig.obj (.const:.string)
                  200263eb    00000001     app_pem4.oem4 (.const:xdc_runtime_Error_policy__C)
                  200263ec    00000020     mqtt.a : cc31xx_sl_net.obj (.const)
                  2002640c    00000020     app_pem4.oem4 (.const:ti_sysbios_family_arm_m3_Hwi_Object__DESC__C)
                  2002642c    00000020     app_pem4.oem4 (.const:ti_sysbios_gates_GateHwi_Object__DESC__C)
                  2002644c    00000020     app_pem4.oem4 (.const:ti_sysbios_gates_GateMutex_Object__DESC__C)
                  2002646c    00000020     app_pem4.oem4 (.const:ti_sysbios_heaps_HeapMem_Object__DESC__C)
                  2002648c    00000020     app_pem4.oem4 (.const:ti_sysbios_knl_Mailbox_Object__DESC__C)
                  200264ac    00000020     app_pem4.oem4 (.const:ti_sysbios_knl_Queue_Object__DESC__C)
                  200264cc    00000020     app_pem4.oem4 (.const:ti_sysbios_knl_Semaphore_Object__DESC__C)
                  200264ec    00000020     app_pem4.oem4 (.const:ti_sysbios_knl_Task_Object__DESC__C)
                  2002650c    00000020     app_pem4.oem4 (.const:xdc_runtime_LoggerBuf_Object__DESC__C)
                  2002652c    0000001e     gateway.a : gateway_task.obj (.const:.string)
                  2002654a    00000018               : database.obj (.const:.string)
                  20026562    00000002     app_pem4.oem4 (.const:ti_sysbios_family_arm_m3_Timer_Module__id__C)
                  20026564    00000018     driverlib.a : spi.obj (.const)
                  2002657c    00000018     app_pem4.oem4 (.const:ti_sysbios_gates_GateHwi_Object__PARAMS__C)
                  20026594    00000018     app_pem4.oem4 (.const:ti_sysbios_gates_GateMutex_Object__PARAMS__C)
                  200265ac    00000018     app_pem4.oem4 (.const:ti_sysbios_knl_Queue_Object__PARAMS__C)
                  200265c4    00000018     app_pem4.oem4 (.const:xdc_runtime_Startup_sfxnRts__A)
                  200265dc    00000011     ti.targets.arm.rtsarm.aem4 : System.oem4 (.const:.string)
                  200265ed    00000010     simplelink.a : socket.obj (.const:.string)
                  200265fd    0000000e     cc3200.obj (.const:.string)
                  2002660b    0000000d     gateway.a : ble_central.obj (.const:.string)
                  20026618    0000000c     app_pem4.oem4 (.const:xdc_runtime_Startup_firstFxns__A)
                  20026624    0000000b     mqtt.a : mqtt_client.obj (.const:.string)
                  2002662f    00000009     cli.a : cli.obj (.const:.string)
                  20026638    00000008     simplelink.a : device.obj (.const:.string)
                  20026640    00000008                  : netcfg.obj (.const)
                  20026648    00000008     app_pem4.oem4 (.const:ti_sysbios_family_arm_m3_Hwi_excHookFuncs__A)
                  20026650    00000008     app_pem4.oem4 (.const:ti_sysbios_knl_Idle_funcList__C)
                  20026658    00000008     app_pem4.oem4 (.const:xdc_runtime_Startup_firstFxns__C)
                  20026660    00000008     app_pem4.oem4 (.const:xdc_runtime_Startup_lastFxns__C)
                  20026668    00000004     app_pem4.oem4 (.const:ti_sysbios_family_arm_m3_Hwi_E_NMI__C)
                  2002666c    00000004     app_pem4.oem4 (.const:ti_sysbios_family_arm_m3_Hwi_E_alreadyDefined__C)
                  20026670    00000004     app_pem4.oem4 (.const:ti_sysbios_family_arm_m3_Hwi_E_busFault__C)
                  20026674    00000004     app_pem4.oem4 (.const:ti_sysbios_family_arm_m3_Hwi_E_debugMon__C)
                  20026678    00000004     app_pem4.oem4 (.const:ti_sysbios_family_arm_m3_Hwi_E_hardFault__C)
                  2002667c    00000004     app_pem4.oem4 (.const:ti_sysbios_family_arm_m3_Hwi_E_memFault__C)
                  20026680    00000004     app_pem4.oem4 (.const:ti_sysbios_family_arm_m3_Hwi_E_noIsr__C)
                  20026684    00000004     app_pem4.oem4 (.const:ti_sysbios_family_arm_m3_Hwi_E_reserved__C)
                  20026688    00000004     app_pem4.oem4 (.const:ti_sysbios_family_arm_m3_Hwi_E_svCall__C)
                  2002668c    00000004     app_pem4.oem4 (.const:ti_sysbios_family_arm_m3_Hwi_E_usageFault__C)
                  20026690    00000004     app_pem4.oem4 (.const:ti_sysbios_family_arm_m3_Hwi_LD_end__C)
                  20026694    00000004     app_pem4.oem4 (.const:ti_sysbios_family_arm_m3_Hwi_LM_begin__C)
                  20026698    00000004     app_pem4.oem4 (.const:ti_sysbios_family_arm_m3_Hwi_Module__diagsEnabled__C)
                  2002669c    00000004     app_pem4.oem4 (.const:ti_sysbios_family_arm_m3_Hwi_Module__diagsIncluded__C)
                  200266a0    00000004     app_pem4.oem4 (.const:ti_sysbios_family_arm_m3_Hwi_Module__diagsMask__C)
                  200266a4    00000004     app_pem4.oem4 (.const:ti_sysbios_family_arm_m3_Hwi_Module__loggerFxn1__C)
                  200266a8    00000004     app_pem4.oem4 (.const:ti_sysbios_family_arm_m3_Hwi_Module__loggerFxn8__C)
                  200266ac    00000004     app_pem4.oem4 (.const:ti_sysbios_family_arm_m3_Hwi_Module__loggerObj__C)
                  200266b0    00000004     app_pem4.oem4 (.const:ti_sysbios_family_arm_m3_Hwi_NUM_INTERRUPTS__C)
                  200266b4    00000004     app_pem4.oem4 (.const:ti_sysbios_family_arm_m3_Hwi_Object__count__C)
                  200266b8    00000004     app_pem4.oem4 (.const:ti_sysbios_family_arm_m3_Hwi_ccr__C)
                  200266bc    00000004     app_pem4.oem4 (.const:ti_sysbios_family_arm_m3_Hwi_excHandlerFunc__C)
                  200266c0    00000004     app_pem4.oem4 (.const:ti_sysbios_family_arm_m3_Hwi_excHookFuncs__C)
                  200266c4    00000004     app_pem4.oem4 (.const:ti_sysbios_family_arm_m3_Hwi_nullIsrFunc__C)
                  200266c8    00000004     app_pem4.oem4 (.const:ti_sysbios_family_arm_m3_Hwi_priGroup__C)
                  200266cc    00000004     app_pem4.oem4 (.const:ti_sysbios_family_arm_m3_TaskSupport_stackAlignment__C)
                  200266d0    00000004     app_pem4.oem4 (.const:ti_sysbios_family_arm_m3_Timer_E_cannotSupport__C)
                  200266d4    00000004     app_pem4.oem4 (.const:ti_sysbios_family_arm_m3_Timer_startupNeeded__C)
                  200266d8    00000004     app_pem4.oem4 (.const:ti_sysbios_gates_GateMutex_A_badContext__C)
                  200266dc    00000004     app_pem4.oem4 (.const:ti_sysbios_gates_GateMutex_Instance_State_sem__O)
                  200266e0    00000004     app_pem4.oem4 (.const:ti_sysbios_gates_GateMutex_Module__diagsEnabled__C)
                  200266e4    00000004     app_pem4.oem4 (.const:ti_sysbios_gates_GateMutex_Module__diagsIncluded__C)
                  200266e8    00000004     app_pem4.oem4 (.const:ti_sysbios_gates_GateMutex_Module__diagsMask__C)
                  200266ec    00000004     app_pem4.oem4 (.const:ti_sysbios_hal_Hwi_E_stackOverflow__C)
                  200266f0    00000004     app_pem4.oem4 (.const:ti_sysbios_heaps_HeapMem_A_align__C)
                  200266f4    00000004     app_pem4.oem4 (.const:ti_sysbios_heaps_HeapMem_A_heapSize__C)
                  200266f8    00000004     app_pem4.oem4 (.const:ti_sysbios_heaps_HeapMem_A_invalidFree__C)
                  200266fc    00000004     app_pem4.oem4 (.const:ti_sysbios_heaps_HeapMem_A_zeroBlock__C)
                  20026700    00000004     app_pem4.oem4 (.const:ti_sysbios_heaps_HeapMem_E_memory__C)
                  20026704    00000004     app_pem4.oem4 (.const:ti_sysbios_heaps_HeapMem_Module__diagsEnabled__C)
                  20026708    00000004     app_pem4.oem4 (.const:ti_sysbios_heaps_HeapMem_Module__diagsIncluded__C)
                  2002670c    00000004     app_pem4.oem4 (.const:ti_sysbios_heaps_HeapMem_Module__diagsMask__C)
                  20026710    00000004     app_pem4.oem4 (.const:ti_sysbios_heaps_HeapMem_Module__gateObj__C)
                  20026714    00000004     app_pem4.oem4 (.const:ti_sysbios_heaps_HeapMem_Object__count__C)
                  20026718    00000004     app_pem4.oem4 (.const:ti_sysbios_heaps_HeapMem_reqAlign__C)
                  2002671c    00000004     app_pem4.oem4 (.const:ti_sysbios_knl_Clock_LM_begin__C)
                  20026720    00000004     app_pem4.oem4 (.const:ti_sysbios_knl_Clock_LM_tick__C)
                  20026724    00000004     app_pem4.oem4 (.const:ti_sysbios_knl_Clock_LW_delayed__C)
                  20026728    00000004     app_pem4.oem4 (.const:ti_sysbios_knl_Clock_Module_State_clockQ__O)
                  2002672c    00000004     app_pem4.oem4 (.const:ti_sysbios_knl_Clock_Module__diagsEnabled__C)
                  20026730    00000004     app_pem4.oem4 (.const:ti_sysbios_knl_Clock_Module__diagsIncluded__C)
                  20026734    00000004     app_pem4.oem4 (.const:ti_sysbios_knl_Clock_Module__diagsMask__C)
                  20026738    00000004     app_pem4.oem4 (.const:ti_sysbios_knl_Clock_Module__loggerFxn1__C)
                  2002673c    00000004     app_pem4.oem4 (.const:ti_sysbios_knl_Clock_Module__loggerFxn2__C)
                  20026740    00000004     app_pem4.oem4 (.const:ti_sysbios_knl_Clock_Module__loggerObj__C)
                  20026744    00000004     app_pem4.oem4 (.const:ti_sysbios_knl_Clock_tickPeriod__C)
                  20026748    00000004     app_pem4.oem4 (.const:ti_sysbios_knl_Idle_funcList__A)
                  2002674c    00000004     app_pem4.oem4 (.const:ti_sysbios_knl_Mailbox_A_invalidBufSize__C)
                  20026750    00000004     app_pem4.oem4 (.const:ti_sysbios_knl_Mailbox_Instance_State_dataQue__O)
                  20026754    00000004     app_pem4.oem4 (.const:ti_sysbios_knl_Mailbox_Instance_State_dataSem__O)
                  20026758    00000004     app_pem4.oem4 (.const:ti_sysbios_knl_Mailbox_Instance_State_freeQue__O)
                  2002675c    00000004     app_pem4.oem4 (.const:ti_sysbios_knl_Mailbox_Instance_State_freeSem__O)
                  20026760    00000004     app_pem4.oem4 (.const:ti_sysbios_knl_Mailbox_Module__diagsEnabled__C)
                  20026764    00000004     app_pem4.oem4 (.const:ti_sysbios_knl_Mailbox_Module__diagsIncluded__C)
                  20026768    00000004     app_pem4.oem4 (.const:ti_sysbios_knl_Mailbox_Module__diagsMask__C)
                  2002676c    00000004     app_pem4.oem4 (.const:ti_sysbios_knl_Mailbox_Object__count__C)
                  20026770    00000004     app_pem4.oem4 (.const:ti_sysbios_knl_Mailbox_maxTypeAlign__C)
                  20026774    00000004     app_pem4.oem4 (.const:ti_sysbios_knl_Semaphore_A_badContext__C)
                  20026778    00000004     app_pem4.oem4 (.const:ti_sysbios_knl_Semaphore_A_noEvents__C)
                  2002677c    00000004     app_pem4.oem4 (.const:ti_sysbios_knl_Semaphore_A_overflow__C)
                  20026780    00000004     app_pem4.oem4 (.const:ti_sysbios_knl_Semaphore_A_pendTaskDisabled__C)
                  20026784    00000004     app_pem4.oem4 (.const:ti_sysbios_knl_Semaphore_Instance_State_pendQ__O)
                  20026788    00000004     app_pem4.oem4 (.const:ti_sysbios_knl_Semaphore_LM_pend__C)
                  2002678c    00000004     app_pem4.oem4 (.const:ti_sysbios_knl_Semaphore_LM_post__C)
                  20026790    00000004     app_pem4.oem4 (.const:ti_sysbios_knl_Semaphore_Module__diagsEnabled__C)
                  20026794    00000004     app_pem4.oem4 (.const:ti_sysbios_knl_Semaphore_Module__diagsIncluded__C)
                  20026798    00000004     app_pem4.oem4 (.const:ti_sysbios_knl_Semaphore_Module__diagsMask__C)
                  2002679c    00000004     app_pem4.oem4 (.const:ti_sysbios_knl_Semaphore_Module__loggerFxn2__C)
                  200267a0    00000004     app_pem4.oem4 (.const:ti_sysbios_knl_Semaphore_Module__loggerFxn4__C)
                  200267a4    00000004     app_pem4.oem4 (.const:ti_sysbios_knl_Semaphore_Module__loggerObj__C)
                  200267a8    00000004     app_pem4.oem4 (.const:ti_sysbios_knl_Swi_LD_end__C)
                  200267ac    00000004     app_pem4.oem4 (.const:ti_sysbios_knl_Swi_LM_begin__C)
                  200267b0    00000004     app_pem4.oem4 (.const:ti_sysbios_knl_Swi_LM_post__C)
                  200267b4    00000004     app_pem4.oem4 (.const:ti_sysbios_knl_Swi_Module__diagsEnabled__C)
                  200267b8    00000004     app_pem4.oem4 (.const:ti_sysbios_knl_Swi_Module__diagsIncluded__C)
                  200267bc    00000004     app_pem4.oem4 (.const:ti_sysbios_knl_Swi_Module__diagsMask__C)
                  200267c0    00000004     app_pem4.oem4 (.const:ti_sysbios_knl_Swi_Module__loggerFxn1__C)
                  200267c4    00000004     app_pem4.oem4 (.const:ti_sysbios_knl_Swi_Module__loggerFxn4__C)
                  200267c8    00000004     app_pem4.oem4 (.const:ti_sysbios_knl_Swi_Module__loggerObj__C)
                  200267cc    00000004     app_pem4.oem4 (.const:ti_sysbios_knl_Swi_Object__count__C)
                  200267d0    00000004     app_pem4.oem4 (.const:ti_sysbios_knl_Task_A_badPriority__C)
                  200267d4    00000004     app_pem4.oem4 (.const:ti_sysbios_knl_Task_A_badTaskState__C)
                  200267d8    00000004     app_pem4.oem4 (.const:ti_sysbios_knl_Task_A_badThreadType__C)
                  200267dc    00000004     app_pem4.oem4 (.const:ti_sysbios_knl_Task_A_badTimeout__C)
                  200267e0    00000004     app_pem4.oem4 (.const:ti_sysbios_knl_Task_A_noPendElem__C)
                  200267e4    00000004     app_pem4.oem4 (.const:ti_sysbios_knl_Task_A_sleepTaskDisabled__C)
                  200267e8    00000004     app_pem4.oem4 (.const:ti_sysbios_knl_Task_E_spOutOfBounds__C)
                  200267ec    00000004     app_pem4.oem4 (.const:ti_sysbios_knl_Task_E_stackOverflow__C)
                  200267f0    00000004     app_pem4.oem4 (.const:ti_sysbios_knl_Task_LD_block__C)
                  200267f4    00000004     app_pem4.oem4 (.const:ti_sysbios_knl_Task_LD_exit__C)
                  200267f8    00000004     app_pem4.oem4 (.const:ti_sysbios_knl_Task_LD_ready__C)
                  200267fc    00000004     app_pem4.oem4 (.const:ti_sysbios_knl_Task_LM_sleep__C)
                  20026800    00000004     app_pem4.oem4 (.const:ti_sysbios_knl_Task_LM_switch__C)
                  20026804    00000004     app_pem4.oem4 (.const:ti_sysbios_knl_Task_LM_yield__C)
                  20026808    00000004     app_pem4.oem4 (.const:ti_sysbios_knl_Task_Module_State_inactiveQ__O)
                  2002680c    00000004     app_pem4.oem4 (.const:ti_sysbios_knl_Task_Module__diagsEnabled__C)
                  20026810    00000004     app_pem4.oem4 (.const:ti_sysbios_knl_Task_Module__diagsIncluded__C)
                  20026814    00000004     app_pem4.oem4 (.const:ti_sysbios_knl_Task_Module__diagsMask__C)
                  20026818    00000004     app_pem4.oem4 (.const:ti_sysbios_knl_Task_Module__loggerFxn2__C)
                  2002681c    00000004     app_pem4.oem4 (.const:ti_sysbios_knl_Task_Module__loggerFxn4__C)
                  20026820    00000004     app_pem4.oem4 (.const:ti_sysbios_knl_Task_Module__loggerObj__C)
                  20026824    00000004     app_pem4.oem4 (.const:ti_sysbios_knl_Task_Object__count__C)
                  20026828    00000004     app_pem4.oem4 (.const:ti_sysbios_knl_Task_allBlockedFunc__C)
                  2002682c    00000004     app_pem4.oem4 (.const:ti_sysbios_knl_Task_defaultStackHeap__C)
                  20026830    00000004     app_pem4.oem4 (.const:ti_sysbios_knl_Task_defaultStackSize__C)
                  20026834    00000004     app_pem4.oem4 (.const:ti_sysbios_knl_Task_numConstructedTasks__C)
                  20026838    00000004     app_pem4.oem4 (.const:xdc_runtime_Assert_E_assertFailed__C)
                  2002683c    00000004     app_pem4.oem4 (.const:xdc_runtime_Core_A_initializedParams__C)
                  20026840    00000004     app_pem4.oem4 (.const:xdc_runtime_Core_Module__diagsEnabled__C)
                  20026844    00000004     app_pem4.oem4 (.const:xdc_runtime_Core_Module__diagsIncluded__C)
                  20026848    00000004     app_pem4.oem4 (.const:xdc_runtime_Core_Module__diagsMask__C)
                  2002684c    00000004     app_pem4.oem4 (.const:xdc_runtime_Error_E_memory__C)
                  20026850    00000004     app_pem4.oem4 (.const:xdc_runtime_Error_Module__diagsEnabled__C)
                  20026854    00000004     app_pem4.oem4 (.const:xdc_runtime_Error_Module__diagsIncluded__C)
                  20026858    00000004     app_pem4.oem4 (.const:xdc_runtime_Error_Module__diagsMask__C)
                  2002685c    00000004     app_pem4.oem4 (.const:xdc_runtime_Error_Module__loggerFxn8__C)
                  20026860    00000004     app_pem4.oem4 (.const:xdc_runtime_Error_Module__loggerObj__C)
                  20026864    00000004     app_pem4.oem4 (.const:xdc_runtime_Error_policyFxn__C)
                  20026868    00000004     app_pem4.oem4 (.const:xdc_runtime_Error_raiseHook__C)
                  2002686c    00000004     app_pem4.oem4 (.const:xdc_runtime_IFilterLogger_Interface__BASE__C)
                  20026870    00000004     app_pem4.oem4 (.const:xdc_runtime_IGateProvider_Interface__BASE__C)
                  20026874    00000004     app_pem4.oem4 (.const:xdc_runtime_IHeap_Interface__BASE__C)
                  20026878    00000004     app_pem4.oem4 (.const:xdc_runtime_ILogger_Interface__BASE__C)
                  2002687c    00000004     app_pem4.oem4 (.const:xdc_runtime_IModule_Interface__BASE__C)
                  20026880    00000004     app_pem4.oem4 (.const:xdc_runtime_Log_L_error__C)
                  20026884    00000004     app_pem4.oem4 (.const:xdc_runtime_LoggerBuf_E_badLevel__C)
                  20026888    00000004     app_pem4.oem4 (.const:xdc_runtime_LoggerBuf_Module__gateObj__C)
                  2002688c    00000004     app_pem4.oem4 (.const:xdc_runtime_LoggerBuf_Object__count__C)
                  20026890    00000004     app_pem4.oem4 (.const:xdc_runtime_LoggerBuf_statusLogger__C)
                  20026894    00000004     app_pem4.oem4 (.const:xdc_runtime_Memory_defaultHeapInstance__C)
                  20026898    00000004     app_pem4.oem4 (.const:xdc_runtime_Startup_execImpl__C)
                  2002689c    00000004     app_pem4.oem4 (.const:xdc_runtime_Startup_maxPasses__C)
                  200268a0    00000004     app_pem4.oem4 (.const:xdc_runtime_Startup_sfxnRts__C)
                  200268a4    00000004     app_pem4.oem4 (.const:xdc_runtime_Startup_sfxnTab__C)
                  200268a8    00000004     app_pem4.oem4 (.const:xdc_runtime_SysMin_bufSize__C)
                  200268ac    00000004     app_pem4.oem4 (.const:xdc_runtime_SysMin_outputFunc__C)
                  200268b0    00000004     app_pem4.oem4 (.const:xdc_runtime_System_Module__gateObj__C)
                  200268b4    00000004     app_pem4.oem4 (.const:xdc_runtime_System_abortFxn__C)
                  200268b8    00000004     app_pem4.oem4 (.const:xdc_runtime_System_exitFxn__C)
                  200268bc    00000004     app_pem4.oem4 (.const:xdc_runtime_System_extendFxn__C)
                  200268c0    00000004     app_pem4.oem4 (.const:xdc_runtime_System_maxAtexitHandlers__C)
                  200268c4    00000004     app_pem4.oem4 (.const:xdc_runtime_Text_charTab__C)
                  200268c8    00000004     app_pem4.oem4 (.const:xdc_runtime_Text_nameEmpty__C)
                  200268cc    00000004     app_pem4.oem4 (.const:xdc_runtime_Text_nameStatic__C)
                  200268d0    00000004     app_pem4.oem4 (.const:xdc_runtime_Text_nameUnknown__C)
                  200268d4    00000004     app_pem4.oem4 (.const:xdc_runtime_Text_nodeTab__C)
                  200268d8    00000004     app_pem4.oem4 (.const:xdc_runtime_Text_visitRopeFxn__C)
                  200268dc    00000003     mqtt.a : sl_mqtt_client.obj (.const)
                  200268df    00000001     --HOLE-- [fill = 0]
                  200268e0    00000002     app_pem4.oem4 (.const:ti_sysbios_family_arm_m3_TimestampProvider_configTimer__C)
                  200268e2    00000002     app_pem4.oem4 (.const:ti_sysbios_gates_GateMutex_Module__id__C)
                  200268e4    00000002     app_pem4.oem4 (.const:ti_sysbios_hal_Hwi_Module__id__C)
                  200268e6    00000002     app_pem4.oem4 (.const:ti_sysbios_heaps_HeapMem_Module__id__C)
                  200268e8    00000002     app_pem4.oem4 (.const:ti_sysbios_knl_Clock_Module__id__C)
                  200268ea    00000002     app_pem4.oem4 (.const:ti_sysbios_knl_Clock_Module__loggerDefined__C)
                  200268ec    00000002     app_pem4.oem4 (.const:ti_sysbios_knl_Mailbox_Module__id__C)
                  200268ee    00000002     app_pem4.oem4 (.const:ti_sysbios_knl_Semaphore_Module__id__C)
                  200268f0    00000002     app_pem4.oem4 (.const:ti_sysbios_knl_Semaphore_Module__loggerDefined__C)
                  200268f2    00000002     app_pem4.oem4 (.const:ti_sysbios_knl_Swi_Module__id__C)
                  200268f4    00000002     app_pem4.oem4 (.const:ti_sysbios_knl_Swi_Module__loggerDefined__C)
                  200268f6    00000002     app_pem4.oem4 (.const:ti_sysbios_knl_Task_Module__id__C)
                  200268f8    00000002     app_pem4.oem4 (.const:ti_sysbios_knl_Task_Module__loggerDefined__C)
                  200268fa    00000002     app_pem4.oem4 (.const:ti_sysbios_knl_Task_initStackFlag__C)
                  200268fc    00000002     app_pem4.oem4 (.const:xdc_runtime_Core_Module__id__C)
                  200268fe    00000002     app_pem4.oem4 (.const:xdc_runtime_Error_Module__loggerDefined__C)
                  20026900    00000002     app_pem4.oem4 (.const:xdc_runtime_Error_maxDepth__C)
                  20026902    00000002     app_pem4.oem4 (.const:xdc_runtime_LoggerBuf_Module__id__C)
                  20026904    00000002     app_pem4.oem4 (.const:xdc_runtime_LoggerBuf_filterByLevel__C)
                  20026906    00000002     app_pem4.oem4 (.const:xdc_runtime_Memory_Module__id__C)
                  20026908    00000002     app_pem4.oem4 (.const:xdc_runtime_SysMin_flushAtExit__C)
                  2002690a    00000002     app_pem4.oem4 (.const:xdc_runtime_Text_charCnt__C)
                  2002690c    00000002     app_pem4.oem4 (.const:xdc_runtime_Text_isLoaded__C)
                  2002690e    00000002     app_pem4.oem4 (.const:xdc_runtime_Text_registryModsLastId__C)
                  20026910    00000002     app_pem4.oem4 (.const:xdc_runtime_Text_unnamedModsLastId__C)

.cinit     0    20026918    00000d10     
                  20026918    00000ce7     (.cinit..data.load) [load image, compression = rle]
                  200275ff    00000001     --HOLE-- [fill = 0]
                  20027600    0000000c     (__TI_handler_table)
                  2002760c    00000004     --HOLE-- [fill = 0]
                  20027610    00000008     (.cinit..bss.load) [load image, compression = zero_init]
                  20027618    00000010     (__TI_cinit_table)

.bss       0    2002bf00    0000f2de     UNINITIALIZED
                  2002bf00    0000a000     app_pem4.oem4 (.bss:ti_sysbios_heaps_HeapMem_Instance_State_0_buf__A)
                  20035f00    00000800     mqtt.a : sl_mqtt_client.obj (.bss:buf_vec)
                  20036700    00000800     npi.a : uart_def.obj (.bss:g_ucUartAckRxBuffer)
                  20036f00    00000800           : uart_def.obj (.bss:g_ucUartRxBuffer)
                  20037700    00000800     app_pem4.oem4 (.bss:taskStackSection)
                  20037f00    000005a0     ota.a : OtaHttp.obj (.bss:recv_buf)
                  200384a0    0000044c           : OtaClient.obj (.bss:g_OtaCheckUpdateResponse)
                  200388ec    00000400     app_pem4.oem4 (.bss:xdc_runtime_LoggerBuf_Instance_State_0_entryArr__A)
                  20038cec    00000400     app_pem4.oem4 (.bss:xdc_runtime_SysMin_Module_State_0_outbuf__A)
                  200390ec    000003fc     cli.a : cli.obj (.bss:his_tbl)
                  200394e8    000003d8     ota.a : OtaClient.obj (.bss:g_OtaFileMetadata)
                  200398c0    0000030c     app_pem4.oem4 (.bss:ti_sysbios_family_arm_m3_Hwi_dispatchTable)
                  20039bcc    000002d0     mqtt.a : mqtt_client.obj (.bss:clients)
                  20039e9c    00000258     http.obj (.bss:gw_charlist)
                  2003a0f4    00000240     otatask.obj (.bss:g_otaOptServerInfo)
                  2003a334    00000200     ota.a : OtaHttp.obj (.bss:send_buf)
                  2003a534    00000178     simplelink.a : driver.obj (.bss:g_StatMem)
                  2003a6ac    00000150     cli.a : cli.obj (.bss:cmd_tbl)
                  2003a7fc    0000012c     mqtt_app.a : CC2650_SensorTag.obj (.bss:sensor_message)
                  2003a928    0000012c     mqtt.a : sl_mqtt_client.obj (.bss:sl_cli_ctx)
                  2003aa54    00000120     rtsv7M4_T_le_eabi.lib : trgmsg.obj (.bss:__CIOBUF_)
                  2003ab74    00000078     http.obj (.bss:gw_scanlist)
                  2003abec    00000074     ota.a : CdnClient.obj (.bss:g_CdnClient)
                  2003ac60    00000064     cli.a : cli.obj (.bss:cmdl)
                  2003acc4    00000064     mqtt_app.a : mqtt_app_main.obj (.bss:gw_scanres_message)
                  2003ad28    0000005c     gateway.a : gateway_task.obj (.bss:gw_context)
                  2003ad84    00000050     simplelink.a : cc_pal.obj (.bss:g_ucDinDout)
                  2003add4    0000004c     ota.a : OtaApp.obj (.bss:g_OtaApp)
                  2003ae20    0000004c           : OtaApp.obj (.bss:g_OtaApp_statistics)
                  2003ae6c    00000048     http.obj (.bss:gw_connlist)
                  2003aeb4    00000048     mqtt.a : sl_mqtt_client.obj (.bss:mqp_vec)
                  2003aefc    00000034     mqtt_app.a : mqtt_app_main.obj (.bss:gw_link_message)
                  2003af30    00000034                : device_mqtt.obj (.bss:listcharstr)
                  2003af64    00000030     npi.a : gap_packets.obj (.bss:gGapPacket)
                  2003af94    00000030           : gatt.obj (.bss:gGattPacket)
                  2003afc4    00000028     gateway.a : database.obj (.bss:DeviceRec)
                  2003afec    00000028     schema.a : schema.obj (.bss:sch_nvmemload)
                  2003b014    00000024     ota.a : OtaClient.obj (.bss:g_OtaClient)
                  2003b038    00000024     wifi.obj (.bss:g_ucConnectionSSID)
                  2003b05c    0000001a     (.common:attWriteReq)
                  2003b076    00000002     (.common:attReadReq)
                  2003b078    00000018     (.common:blefiCfgRec)
                  2003b090    00000018     (.common:recv_hvec)
                  2003b0a8    00000015     (.common:attReadByTypeReq)
                  2003b0bd    00000001     (.common:RxIrqCnt)
                  2003b0be    00000001     (.common:cCountScanDevices)
                  2003b0bf    00000001     (.common:g_ucPacketEvent)
                  2003b0c0    00000014     (.common:g_FlcSflashCb)
                  2003b0d4    00000010     (.common:blefi_mac_string)
                  2003b0e4    00000010     (.common:gapCentralRoleIRK)
                  2003b0f4    00000010     (.common:gapCentralRoleSRK)
                  2003b104    00000010     (.common:str$2)
                  2003b114    00000008     (.common:bdAddr)
                  2003b11c    00000008     (.common:bdaddress)
                  2003b124    00000008     (.common:g_LogClient)
                  2003b12c    00000008     (.common:g_macAddressVal)
                  2003b134    00000008     (.common:g_ucConnectionBSSID)
                  2003b13c    00000008     (.common:gapCentralRoleBdAddr)
                  2003b144    00000008     (.common:parmbuf)
                  2003b14c    00000008     (.common:sBootInfo)
                  2003b154    00000008     (.common:wlan_mac)
                  2003b15c    00000004     (.common:DMAMsgQ)
                  2003b160    00000004     (.common:GC_ApiLockObj)
                  2003b164    00000004     (.common:RecvQue$1)
                  2003b168    00000004     (.common:ReportLockObj)
                  2003b16c    00000004     (.common:SimpleLinkSpawnTaskHndl)
                  2003b170    00000004     (.common:__Errorlog)
                  2003b174    00000004     (.common:blefiCfgData)
                  2003b178    00000004     (.common:gIntHdlr)
                  2003b17c    00000004     (.common:gNPI_SyncObj)
                  2003b180    00000004     (.common:g_GWGenSyncObj)
                  2003b184    00000004     (.common:g_Mqtt_queue)
                  2003b188    00000004     (.common:g_NetStatSyncObj)
                  2003b18c    00000004     (.common:g_OTAStatSyncObj)
                  2003b190    00000004     (.common:g_cDummy)
                  2003b194    00000004     (.common:g_rx_task_hndl)
                  2003b198    00000004     (.common:g_rx_tx_sync_obj)
                  2003b19c    00000004     (.common:g_wait_secs)
                  2003b1a0    00000004     (.common:gw_blefi_linke_topic)
                  2003b1a4    00000004     (.common:gw_blefi_linkt_topic)
                  2003b1a8    00000004     (.common:gw_blefi_scan_topic)
                  2003b1ac    00000004     (.common:mqttQStimeout)
                  2003b1b0    00000004     (.common:mqtt_lib_lockobj)
                  2003b1b4    00000004     (.common:pGC_StateCB)
                  2003b1b8    00000004     (.common:pNpiEvtCb)
                  2003b1bc    00000004     (.common:pcliSyncObj)
                  2003b1c0    00000004     (.common:pvOtaApp)
                  2003b1c4    00000004     (.common:sGC_AppMsgQueue)
                  2003b1c8    00000004     (.common:sGC_StackMsgQueue)
                  2003b1cc    00000004     (.common:sMsg)
                  2003b1d0    00000004     (.common:sblFileHandle)
                  2003b1d4    00000004     (.common:simpleLink_mailbox)
                  2003b1d8    00000004     (.common:tokenList)
                  2003b1dc    00000001     (.common:g_ucPacketLen)
                  2003b1dd    00000001     (.common:g_ucPacketType)

.data      0    2003b1e0    00000f40     UNINITIALIZED
                  2003b1e0    000005dc     http.obj (.data:g_gettoken_getchar)
                  2003b7bc    00000138     app_pem4.oem4 (.data)
                  2003b8f4    000000fc     mqtt_app.a : device_mqtt.obj (.data:device_hdl)
                  2003b9f0    000000c8     http.obj (.data:g_gettoken_scan)
                  2003bab8    00000096     http.obj (.data:g_posttoken)
                  2003bb4e    00000002     gateway.a : gateway_cmds.obj (.data)
                  2003bb50    00000080     app_pem4.oem4 (.data:ti_sysbios_knl_Swi_Module_State_0_readyQ__A)
                  2003bbd0    00000080     app_pem4.oem4 (.data:ti_sysbios_knl_Task_Module_State_0_readyQ__A)
                  2003bc50    00000078     http.obj (.data:g_gettoken_conn)
                  2003bcc8    00000070     mqtt_app.a : mqtt_app_main.obj (.data:gw_connect_config)
                  2003bd38    0000004c     mqtt.a : mqtt_client.obj (.data)
                  2003bd84    0000004c     app_pem4.oem4 (.data:ti_sysbios_knl_Task_Object__table__V)
                  2003bdd0    00000048     mqtt_app.a : device_mqtt.obj (.data:mqtt_device_cfg)
                  2003be18    00000044     app_pem4.oem4 (.data:ti_sysbios_knl_Task_Module__state__V)
                  2003be5c    0000003c     http.obj (.data:getsetParams)
                  2003be98    00000038     app_pem4.oem4 (.data:ti_sysbios_gates_GateMutex_Object__table__V)
                  2003bed0    00000034     app_pem4.oem4 (.data:ti_sysbios_family_arm_m3_Hwi_Module__state__V)
                  2003bf04    00000032     http.obj (.data:g_gettoken_other)
                  2003bf36    00000001     cli.a : cli_handler.obj (.data)
                  2003bf37    00000001     gateway.a : gateway_api.obj (.data)
                  2003bf38    00000030     app_pem4.oem4 (.data:ti_sysbios_family_arm_m3_Timer_Object__table__V)
                  2003bf68    00000030     app_pem4.oem4 (.data:ti_sysbios_knl_Swi_Object__table__V)
                  2003bf98    0000002c     mqtt_app.a : mqtt_app_main.obj (.data)
                  2003bfc4    0000002c     app_pem4.oem4 (.data:ti_sysbios_knl_Clock_Module__state__V)
                  2003bff0    00000028     mqtt.a : sl_mqtt_client.obj (.data:net)
                  2003c018    00000024     app_pem4.oem4 (.data:ti_sysbios_BIOS_Module__state__V)
                  2003c03c    00000024     app_pem4.oem4 (.data:xdc_runtime_LoggerBuf_Object__table__V)
                  2003c060    00000023     gateway.a : gapbondmgr.obj (.data)
                  2003c083    00000001               : gateway_task.obj (.data)
                  2003c084    00000014     mqtt_app.a : CC2650_SensorTag.obj (.data)
                  2003c098    0000000d     wifi.obj (.data)
                  2003c0a5    00000003     npi.a : ble_events.obj (.data)
                  2003c0a8    0000000c     generic_task.obj (.data)
                  2003c0b4    0000000c     http.obj (.data)
                  2003c0c0    0000000c     npi.a : npi_cc3200_if.obj (.data)
                  2003c0cc    00000009     simplelink.a : cc_pal.obj (.data)
                  2003c0d5    00000001     mqtt.a : sl_mqtt_client.obj (.data)
                  2003c0d6    00000001     npi.a : gap_packets.obj (.data)
                  2003c0d7    00000001     --HOLE--
                  2003c0d8    00000009     simplelink.a : driver.obj (.data)
                  2003c0e1    00000003     --HOLE--
                  2003c0e4    00000008     cli.a : cli.obj (.data)
                  2003c0ec    00000008     mqtt_app.a : device_mqtt.obj (.data)
                  2003c0f4    00000008     rtsv7M4_T_le_eabi.lib : _lock.obj (.data)
                  2003c0fc    00000008                           : exit.obj (.data)
                  2003c104    00000005     gateway.a : ble_central.obj (.data)
                  2003c109    00000003     --HOLE--
                  2003c10c    00000004     npi.a : uart_def.obj (.data)
                  2003c110    00000004     ota.a : OtaHttp.obj (.data)
                  2003c114    00000004     rtsv7M4_T_le_eabi.lib : errno.obj (.data)
                  2003c118    00000004                           : stkdepth_vars.obj (.data)
                  2003c11c    00000004                           : strtok.obj (.data)

.stack     0    2003cdfc    00002000     UNINITIALIZED
                  2003cdfc    00002000     --HOLE--


LINKER GENERATED COPY TABLES

__TI_cinit_table @ 20027618 records: 2, size/record: 8, table size: 16
	.data: load addr=20026918, load size=00000ce7 bytes, run addr=2003b1e0, run size=00000f40 bytes, compression=rle
	.bss: load addr=20027610, load size=00000008 bytes, run addr=2002bf00, run size=0000f2de bytes, compression=zero_init


LINKER GENERATED HANDLER TABLE

__TI_handler_table @ 20027600 records: 3, size/record: 4, table size: 12
	index: 0, handler: __TI_decompress_rle24
	index: 1, handler: __TI_decompress_none
	index: 2, handler: __TI_zero_init


GLOBAL SYMBOLS: SORTED ALPHABETICALLY BY Name 

address    name
--------   ----
2001ef53   BLEAPI_checkReceivedEvent
2001ef1b   BLEAPI_decodeIncomingPacket
2001ef73   BLEAPI_waitForSpecficEvent
2001b80d   BlefiDisplayBanner
2001b7b5   BlefiVersion
2001b83b   Blefi_HW_Init
2001144d   BlinkLed
200114f1   Button2Init
20011531   Button2IntClear
20011543   Button2IntDisable
200115a3   Button2IntEnable
200220f5   C$$EXIT
20021247   C$$IO$$
2001b7b9   CC26xx_Init
2000e76d   CC26xx_SBL_CheckIfUpdateFwNeeded
200116fb   CC26xx_SBL_Dnld_Init
2000c4f1   CLI_DataCb
2000c469   CLI_EventCb
2000dccb   CLI_Init
20023cd3   CPUcpsie
2001371b   CallGwDataCB
20013695   CallGwEventCB
200180cb   CdnClient_CloseServer
200180e9   CdnClient_ConnectByUrl
20018099   CdnClient_Init
20017f63   CdnClient_Run
20017f59   CdnClient_SetFileInfo
20018217   ClearTerm
2000d1e9   CliGetcharOs
2000d129   CliPuts
2000dc83   ClitaskFxn
2000f139   ConnectToNetwork
20012631   CopyDeviceName
200224d7   CopyPingResultsToReport
2000a95f   DB_Build
2000b381   DB_BuildCharDescsTable
2000ad2d   DB_BuildCharTable
2000aa61   DB_BuildPrimServTable
2000aef5   DB_CharDescsTableDeInit
2000aeb5   DB_CharDescsTableInit
2000a8d7   DB_DevRecDbInit
2000a707   DB_DevRecDeInit
2000a635   DB_DevRecInit
2000a865   DB_DevRecReady
2000ace1   DB_DiscAllCharinService
2000b19d   DB_FillCurrentGetCharName
2000afb5   DB_FindCharHandle
2000b1eb   DB_FindCharNameString
2000b4e9   DB_FlushSyncObjects
2000a7a3   DB_FreeCharDescsTable
2000a7eb   DB_FreeDbUuidInfo
2000a767   DB_FreePrimserv
2000abaf   DB_GATT_DiscAllChars
2000a777   DB_GATT_DiscAllPrimaryServices
2000b259   DB_GATT_FindCharDescriptions
2000ac2f   DB_GATT_FindCharDescs
2000a8e9   DB_GATT_ReadUsingCharUuid
2000b30b   DB_GetCharDescription
2000b49f   DB_GetDevCharList
2000b0b9   DB_GetSetChar
2000afff   DB_GetSetCharValue
2000b4cd   DB_IsConnIdValid
2000a609   DB_IsConnhandleValid
2000a955   DB_LinkDevRec
2000af3b   DB_ParseString
2000b429   DB_PrintCharDescsTable
2000ae9f   DB_PrintCharTable
2000ab1d   DB_PrintPrimServTable
2000a841   DB_SyncObjSignal
2000ae45   DB_UpdateCharName
2000b45d   DB_UpdateDeviceName
2000a753   DB_deleteDevRec
2000b48b   DB_getDevAddrPtr
2000b495   DB_getDevNamePtr
2003b15c   DMAMsgQ
2003afc4   DeviceRec
20022e01   DmaSpiSwIntHandler
2000cb97   DoAddOtaMeta
2000cbdd   DoAutoScan
2000cf37   DoAutoconnect
2000cb7b   DoCc26xxFwUpdate
2000cdaf   DoDefault
2000c5ed   DoDevList
2000c923   DoGet
2000c649   DoLinkEstablish
2000c695   DoLinkTerminate
2000c711   DoListChar
2000cc2d   DoMqttAddDev
2000cc47   DoMqttDelDev
2000cde1   DoPairList
2000cb8d   DoReset
2000c5c5   DoScan
2000cab5   DoSet
2000ce67   DoUnPair
2000cb77   DoWlanDisconnect
2000cb21   DoWlanconnect
2000e67b   Do_SBL_Dnld
2000cd2f   DomqttDevMode
2000ccaf   DomqttGwMode
20018221   Error
2001131b   FlashIsFilePresent
2001120f   FlashReadFile
20011131   FlashWriteFile
20010a53   GAPBondMgr_GetParam
20016dff   GAPBondMgr_GetParameter
20010b75   GAPBondMgr_LinkEst
20010c5d   GAPBondMgr_LinkTerm
20010ce5   GAPBondMgr_PasscodeRsp
20010aff   GAPBondMgr_ResolveAddr
20010939   GAPBondMgr_SetParam
20016d9b   GAPBondMgr_SetParameter
20010c79   GAPBondMgr_SlaveReqSecurity
20015b83   GAPBondMgr_getParameterPacketize
20015b2d   GAPBondMgr_setParameterPacketize
2001ab6d   GAPCentralRole_CancelDiscovery
2001ab11   GAPCentralRole_EstablishLink
2001aaaf   GAPCentralRole_GetParameter
2001aa53   GAPCentralRole_SetParameter
2001aa25   GAPCentralRole_StartDevice
2001ab57   GAPCentralRole_StartDiscovery
2001ab03   GAPCentralRole_TerminateLink
2001ab33   GAPCentralRole_UpdateLink
20016b93   GAP_Authenticate
20016c0b   GAP_Bond
20015977   GAP_BondPacketize
20016aab   GAP_ConfigDeviceAddr
20016b7d   GAP_DeviceDiscoveryCancel
20016b61   GAP_DeviceDiscoveryRequest
20016a59   GAP_DeviceInit
20016aed   GAP_EstablishLinkReq
20016d03   GAP_GetParamValue
20016c8f   GAP_PasskeyUpdate
20015a93   GAP_PasskeyUpdatePacketize
20016d2f   GAP_ResolvePrivateAddr
20015ad9   GAP_ResolvePrivateAddrPacketize
20016d65   GAP_SendSlaveSecurityRequest
20015b2b   GAP_SendSlaveSecurityRequestPacketize
20016ccb   GAP_SetParamValue
20016c53   GAP_Signable
20015a25   GAP_SignablePacketize
20016bcf   GAP_TerminateAuth
200159ff   GAP_TerminateAuthPacketize
20016b25   GAP_TerminateLinkReq
20016b09   GAP_UpdateLinkParamReq
20016e41   GAP_advertDataUpdateDone
2001583d   GAP_authenticatePacketize
20015697   GAP_configDeviceAddrPacketize
200156ff   GAP_deviceDiscoveryCancelPacketize
200156d9   GAP_deviceDiscoveryRequestPacketize
20016e31   GAP_deviceInitDone
2001560b   GAP_deviceInitPacketize
200157b7   GAP_endDiscoverablePacketize
200157cf   GAP_establishLinkRequestPacketize
20015abd   GAP_getParameterPacketize
20016e61   GAP_linkEstablished
20016e71   GAP_linkTerminated
20016e51   GAP_makeDiscoverableDone
20015717   GAP_makeDiscoverablePacketize
20015a95   GAP_setParameterPacketize
20015817   GAP_terminateLinkRequestPackeize
2001576b   GAP_updateAdvertisingDataPacketize
2001592d   GAP_updateLinkParamterRequestPacketize
20016a49   GATT_AppCompletedMsg
200165fb   GATT_DeregisterService
20016865   GATT_DiscAllCharDescs
200167b9   GATT_DiscAllChars
200166ef   GATT_DiscAllPrimaryServices
200167f7   GATT_DiscCharsByUUID
20016721   GATT_DiscPrimaryServiceByUUID
200166eb   GATT_ExchangeMTU
200165ef   GATT_ExecuteWriteReq
20016611   GATT_FindHandle
2001660d   GATT_FindHandleUUID
2001677b   GATT_FindIncludedServices
20016615   GATT_FindNextAttr
2001661d   GATT_Indication
20016a4d   GATT_Init
200165e5   GATT_InitClient
200165f3   GATT_InitServer
20016683   GATT_Notification
200165eb   GATT_PrepareWriteReq
20016a4f   GATT_ProcessEvent
20016a37   GATT_ReadCharDesc
200168a3   GATT_ReadCharValue
20016a3b   GATT_ReadLongCharDesc
2001694b   GATT_ReadLongCharValue
2001694f   GATT_ReadMultiCharValues
200168dd   GATT_ReadUsingCharUUID
200165e9   GATT_RegisterForInd
200165ff   GATT_RegisterForReq
200165f7   GATT_RegisterService
20016a33   GATT_ReliableWrites
20016609   GATT_ServiceChangedInd
20016619   GATT_ServiceNumAttrs
20016a47   GATT_SetHostToAppFlowCtrl
20016a4b   GATT_SetNextHandle
200169c5   GATT_SignedWriteNoRsp
20016601   GATT_VerifyReadPermissions
20016605   GATT_VerifyWritePermissions
20016a3f   GATT_WriteCharDesc
200169c9   GATT_WriteCharValue
20016a43   GATT_WriteLongCharDesc
20016a2f   GATT_WriteLongCharValue
20016953   GATT_WriteNoRsp
2003b160   GC_ApiLockObj
20014b97   GC_DeviceConnList
20014b69   GC_DeviceScanList
20014bbb   GC_DeviceScanListBdAddr
20014e97   GC_EraseAllBondings
20014e4b   GC_GATT_DiscAllChars
20014d39   GC_GATT_DiscAllPrimaryServices
20014d79   GC_GATT_DiscPrimaryServiceByUUID
20014e8d   GC_GetDevCharList
2000b0b9   GC_GetSet
20014e9b   GC_IsBLEReady
20014bc5   GC_LinkEstablish
20014cad   GC_LinkTerminate
200110b1   GC_PairDevList
20014adb   GC_Scan
20013791   GC_StackEventHandler_CB
200110e1   GC_UnPair
200228f5   GPIODirModeSet
20023ce7   GPIOIntClear
20023869   GPIOIntDisable
20023883   GPIOIntEnable
20023335   GPIOIntStatus
20020555   GPIOIntTypeSet
2001d375   GPIOLedButtonPinMuxConfig
20023a23   GPIOPinRead
20023423   GPIOPinWrite
2001d3f9   GPIOSBLPinMuxConfig
200145eb   GW_GenericTask_Init
20013595   GatewayCentral_RegisterGC_CB
2001a34d   GatewayCentral_handleinput
200129c9   GatewayCentral_processGattEvent
20012685   GatewayCentral_processRoleEvent
2001490f   Gateway_ButtonInit
200132db   Gateway_Init
2001825f   GetCmd
200148ef   GwButtonHandler
200145a5   GwGenericTask
2002115d   HCI_commandStatus
20021181   HCI_decodeHeader
20019429   HOSTclock
200193f1   HOSTclose
200193b3   HOSTgetenv
20019357   HOSTlseek
20019305   HOSTopen
200192b9   HOSTread
2001925b   HOSTrename
20019221   HOSTtime
200191e9   HOSTunlink
2001919d   HOSTwrite
2000946f   HTTP_DataCb
20009449   HTTP_EventCb
2001160f   HandleError
20009ff5   HttpGetToken
20009991   HttpGetTokenConn
20009bed   HttpGetTokenGetChar
20009d73   HttpGetTokenOther
2000971f   HttpGetTokenScan
2000a1b5   HttpPostToken
2000a5e1   Http_Init
20014a69   IfBondingEnabled
20007e41   InitDevModeServer
200181a1   InitTerm
2001f075   IntDisable
2001f11d   IntEnable
20024051   IntMasterEnable
20021685   IntPendClear
2000f43f   IsSimpleLinkReady
20014621   KickGenericTask
200147f9   LoadBleFiCfg
200189c7   LogClient_Close
200189df   LogClient_ConnectAndPrint
20018991   LogClient_ConnectServer
20018979   LogClient_Init
20018835   LogClient_Print
200240d3   LoggerBuf_instanceStartup
20009185   MQTT_Init
200181eb   Message
20008a49   MqttBleFiHandler
200091c9   MqttBlefiMAC
20008fc5   MqttClient
20007b5d   MqttDevClean
20008881   MqttDevConnectPublish
20006b4d   MqttDevDataCB
2000898b   MqttDevDisconnectPublish
20008659   MqttDevListPublish
20007707   MqttDeviceCtxAdd
20007615   MqttDeviceCtxClean
20007661   MqttDeviceCtxDel
20008b7b   MqttDeviceCtxInit
20007435   MqttDeviceGetHandler
2000735d   MqttDeviceGetPublish
2000759d   MqttDeviceHandler
20007299   MqttDeviceListCharPublish
20007ee9   MqttDevicePubsishQS
20007491   MqttDeviceSetHandler
20007559   MqttDeviceWhoamiPublish
2000851d   MqttGwBuildTopics
2000820b   MqttGwEventCB
20008c25   MqttInitGwContext
2003bfa8   MqttIpAcquired
20008339   MqttIpAcquiredPostMsg
2003bfa9   MqttLibInit
2003bfaa   MqttTopicBuilt
2000838d   MqttTriggerScan
2003bfb0   Mqtt_Client
20018b7d   NPI_CreateSyncObj
20018c3b   NPI_DisableGpioInt
20018c23   NPI_EnableGPIOInt
20018c6d   NPI_GpioPinRead
20018c5d   NPI_GpioPinWrite
200132cd   NPI_Init
20018e4d   NPI_IsReady
20018beb   NPI_RegisterGpioInterrupt
2001ef15   NPI_RegisterTask
20018b8d   NPI_Sleep
20018b91   NPI_SpiInit
20018c81   NPI_SpiReadPacket
20018cc3   NPI_SpiWritePacket
20018b85   NPI_SyncObjSignal
20018b89   NPI_SyncObjSignalFromISR
20018b81   NPI_SyncObjWait
20018b6d   NPI_TaskCreate
20018e3d   NPI_UartDisableInt
20018e45   NPI_UartEnableInt
20017cd5   NPI_UartEventCreateTask
20017b1b   NPI_UartEventTaskFxn
20018db5   NPI_UartInit
20018e09   NPI_UartReadPacket
20018e23   NPI_UartWritePacket
2000f377   NetworkInit
20023f91   NwpMaskInterrupt
2002276d   NwpPowerOff
20022e2d   NwpPowerOn
200203c9   NwpPowerOnPreamble
20023081   NwpRegisterInterruptHandler
20023f9d   NwpUnMaskInterrupt
200150ab   OTAServerInfoSet
200152b9   OTAUpdateTask
20015485   OTA_Init
20025fac   OpcodeTranslateTable
2001506d   OtaAddOtaMeta
20015387   OtaButtonHandler
20015409   OtaButtonInit
20017263   OtaClient_CloseServer
2001722d   OtaClient_ConnectServer
200171fb   OtaClient_GetNextUpdate
200171c9   OtaClient_Init
200170f3   OtaClient_ResourceMetadata
20016f2f   OtaClient_ResourceNameConvert
20016e81   OtaClient_UpdateCheck
2001527b   OtaCommit
200154d7   OtaDownload
2001518f   OtaUpdateLoop
2001ca21   PRCMCC3200MCUInit
20023c65   PRCMHIBRegRead
20023c7b   PRCMHIBRegWrite
20023a3d   PRCMHibernateEnter
2001ff8d   PRCMHibernateIntervalSet
20021d15   PRCMHibernateWakeupSourceEnable
20023009   PRCMPeripheralClkDisable
20022515   PRCMPeripheralClkEnable
2001f9f1   PRCMPeripheralClockGet
200216dd   PRCMPeripheralReset
2002292d   PRCMPeripheralStatusGet
200207d9   PRCMRTCGet
20024083   PRCMRTCInUseSet
2002188d   PRCMSlowClkCtrGet
20022e59   PRCMSysResetCauseGet
20011ab7   ParseJSONData
20020015   PinConfigSet
20022399   PinModeSet
2001d43d   PinMuxConfig
20022b33   PinTypeGPIO
2002389d   PinTypeUART
2001195d   ReadFileFromDevice
20009249   ReadMQTTMode
20015035   RebootMCU
2001365d   RegisterGwCB
20018427   Report
2003b168   ReportLockObj
2003b0bd   RxIrqCnt
20026154   RxMsgClassLUT
2001382d   SBL_IsDone
UNDEFED    SHT$$INIT_ARRAY$$Base
UNDEFED    SHT$$INIT_ARRAY$$Limit
20023031   SL_FD_ISSET
20023357   SL_FD_SET
20023e29   SL_FD_ZERO
20023a55   SPICSDisable
20023a6d   SPICSEnable
2001f50d   SPIConfigSetExpClk
20023443   SPIDataGet
20023685   SPIDataPut
20023a85   SPIDisable
200238b7   SPIDmaEnable
20023a9d   SPIEnable
200238d1   SPIFIFOEnable
20022961   SPIFIFOLevelSet
20021d5d   SPIIntClear
20021a1d   SPIIntEnable
20023379   SPIReset
2002339b   SPIWordCountSet
20011a75   Schema_DelProfile
200119d9   Schema_FindCharString
20011879   Schema_FindProfile
20011a6d   Schema_FindString
20011865   Schema_init
2001190d   Schema_loadfile
2000ed8d   SimpleLinkGeneralEventHandler
2000ed5b   SimpleLinkHttpServerCallback
2000ec87   SimpleLinkNetAppEventHandler
2000edc5   SimpleLinkSockEventHandler
2003b16c   SimpleLinkSpawnTaskHndl
2000ea93   SimpleLinkWlanEventHandler
2000f3bd   SimpleLink_Init
2001e3c9   SmartConfigConnect
2001e43f   SmartConfigStop
20026638   StartResponseLUT
2003bd84   TSK_idle
20018353   TrimSpace
2001138b   TurnOffLed
2001134f   TurnOnLed
20023c91   UARTCharGet
200236fd   UARTCharGetNonBlocking
200236a3   UARTCharPut
20023ab5   UARTCharsAvail
20020ab5   UARTConfigSetExpClk
20022b65   UARTDisable
2002313d   UARTEnable
20023acd   UARTFIFOLevelSet
20023d89   UARTIntClear
20023ae5   UARTIntDisable
20023afd   UARTIntEnable
2001d341   UARTPinMuxConfig
20017d07   UartWritePacket
200148e1   UpdateBlefiCfg
200137df   Util_convertBdAddr2Str
200240a3   UtilsDelay
20015f13   VDeleteSimpleLinkSpawnTask
2001014b   VMqttRecvTask
20015eb9   VStartSimpleLinkSpawnTask
2001ab75   WaitForEvent
2000f3f3   Wifi_GetMAC
2000f29b   WlanConnectAP
2000f293   WlanDisconnectAP
20023f75   _Dclass
20022139   _Dtest
2003c114   _Errno
20017efb   _OpenStorageFile
200176c9   _OtaCleanToIdle
20017ead   _ReadFileHeaders
200177b7   _ReadStatFile
20017ea1   _RecvFileChunk
2002618c   _SlAcceptCmdCtrl
200260d4   _SlActionLookupTable
2001ec41   _SlAsyncEventGenericHandler
20021da5   _SlDrvBasicCmd
2001e21d   _SlDrvClassifyRxMsg
200205d9   _SlDrvCmdOp
20020cf1   _SlDrvCmdSend
2001cdb1   _SlDrvDataReadOp
2001d769   _SlDrvDataWriteOp
20022b95   _SlDrvDeviceEventHandler
2001b939   _SlDrvDriverCBInit
20023ca7   _SlDrvMemZero
20013ead   _SlDrvMsgRead
2001ea0d   _SlDrvMsgReadCmdCtx
2001f64d   _SlDrvMsgReadSpawnCtx
2001add5   _SlDrvMsgWrite
2001db79   _SlDrvNetAppEventHandler
20023719   _SlDrvObjLockWaitForever
20023b15   _SlDrvObjUnLock
20021a69   _SlDrvProtectAsyncRespSetting
20023161   _SlDrvProtectionObjLockWaitForever
20023465   _SlDrvProtectionObjUnLock
2001ac05   _SlDrvReleasePoolObj
20023f59   _SlDrvResetCmdExt
200196e1   _SlDrvRxHdrRead
20021ab5   _SlDrvRxIrqHandler
20023b2d   _SlDrvSyncObjSignal
20023735   _SlDrvSyncObjWaitForever
2001b315   _SlDrvWaitForPoolObj
2001baad   _SlFindAndSetActiveObj
20026110   _SlFsCloseCmdCtrl
20026120   _SlFsDeleteCmdCtrl
2002611c   _SlFsGetInfoCmdCtrl
2002610c   _SlFsOpenCmdCtrl
20026114   _SlFsReadCmdCtrl
20026118   _SlFsWriteCmdCtrl
200262b0   _SlGetHostByNameCtrl
200262ac   _SlGetHostByServiceCtrl
200262a4   _SlGetServiceListeCtrl
20026198   _SlGetSockOptCmdCtrl
20026188   _SlListenCmdCtrl
200262bc   _SlNetAppGetCmdCtrl
200262b8   _SlNetAppSendTokenValueCmdCtrl
200262b4   _SlNetAppSetCmdCtrl
2002629c   _SlNetAppStartCtrl
200262a0   _SlNetAppStopCtrl
20026644   _SlNetCfgGetCmdCtrl
20026640   _SlNetCfgSetCmdCtrl
200265ed   _SlPayloadByProtocolLUT
20025fec   _SlPolicyGetCmdCtrl
20025fe8   _SlPolicySetCmdCtrl
20025ff4   _SlProfileDelCmdCtrl
20025ff0   _SlProfileGetCmdCtrl
20026190   _SlRecvCmdCtrl
20026180   _SlRecvfomCmdCtrl
200262a8   _SlRegisterServiceCtrl
2001e88d   _SlRemoveFromList
20025ffc   _SlRxFilterAddtCmdCtrl
20026004   _SlRxFilterGetCmdCtrl
20026000   _SlRxFilterSetCmdCtrl
2002619c   _SlSelectCmdCtrl
20026184   _SlSendCmdCtrl
20026194   _SlSetSockOptCmdCtrl
20026008   _SlSmartConfigStartCmdCtrl
2002617c   _SlSockCloseCmdCtrl
20026178   _SlSockSocketCmdCtrl
20026014   _SlWlanCfgGetCmdCtrl
20026010   _SlWlanCfgSetCmdCtrl
20025ff8   _SlWlanGetNetworkListCtrl
2002600c   _SlWlanSetModeCmdCtrl
20017769   _WriteStatFile
00000000   __ASM__
2003aa54   __CIOBUF_
00000071   __ISA__
00000084   __PLAT__
2003edfc   __STACK_END
00002000   __STACK_SIZE
000000ab   __TARG__
20027618   __TI_CINIT_Base
20027628   __TI_CINIT_Limit
20027600   __TI_Handler_Table_Base
2002760c   __TI_Handler_Table_Limit
00000001   __TI_args_main
2001f5ad   __TI_auto_init
2003c0fc   __TI_cleanup_ptr
20023f67   __TI_decompress_none
200240af   __TI_decompress_rle24
2003c100   __TI_dtors_ptr
2000c15f   __TI_printfi
2002124b   __TI_readmsg
20026918   __TI_static_base__
2002121d   __TI_writemsg
20023d9b   __TI_zero_init
000000d0   __TRDR__
200202bd   __aeabi_cdcmpeq
200202bd   __aeabi_cdcmple
20020343   __aeabi_cdrcmple
20021ded   __aeabi_d2iz
2001b167   __aeabi_dadd
2001c8e9   __aeabi_ddiv
2001dc77   __aeabi_dmul
2001b15d   __aeabi_dsub
20022dd3   __aeabi_i2d
20023b8d   __aeabi_lmul
200209c5   __aeabi_memclr
200209c5   __aeabi_memclr4
200209c5   __aeabi_memclr8
2001f6e9   __aeabi_memcpy
2001f6e9   __aeabi_memcpy4
2001f6e9   __aeabi_memcpy8
200209c7   __aeabi_memset
200209c7   __aeabi_memset4
200209c7   __aeabi_memset8
20022315   __aeabi_uidivmod
2001a831   __aeabi_uldivmod
ffffffff   __binit__
ffffffff   __c_args__
2003cdfc   __stack
200240a9   __xdc__init
2003b8f0   __xdc__init__addr
20023b75   _args_main
20022029   _c_int00
200258da   _ctypes_
2003c0f4   _lock
20023d0b   _nop
20017e45   _readSignature
20023d03   _register_lock
20023cfd   _register_unlock
20021b01   _sl_BuildAddress
2001f959   _sl_GetCreateFsMode
20023b45   _sl_GetStartResponseConvert
200210fd   _sl_HandleAsync_Accept
2002094d   _sl_HandleAsync_Connect
2001fde9   _sl_HandleAsync_DnsGetHostByName
2001e639   _sl_HandleAsync_DnsGetHostByService
20020855   _sl_HandleAsync_InitComplete
2001fe75   _sl_HandleAsync_PingResponse
200217e5   _sl_HandleAsync_Select
200218dd   _sl_HandleAsync_Stop
20020e35   _sl_NetAppSendTokenValue
20022bc5   _sl_Strlen
20022551   _sl_TruncatePayloadByProtocol
2003c0f8   _unlock
200220f9   abort
2000e66d   addressInFlash
20021cc9   atod
20021b4d   atoi
20021b99   atol
20021cdd   atolong
2003b0a8   attReadByTypeReq
2003b076   attReadReq
2003b05c   attWriteReq
2003c0b0   autoScanTimeout
2003b114   bdAddr
2003b11c   bdaddress
ffffffff   binit
2003b174   blefiCfgData
2003b078   blefiCfgRec
2003b0d4   blefi_mac_string
2003b0be   cCountScanDevices
2000e349   calcCrcLikeChip
20008015   cfgDevMqttMode
200092f5   cfgGwMqttMode
2003c0ac   cfgSize
2003c084   charNameMqtt
2000ff13   cl_ctx_remove
2000fe73   cl_ctx_reset
2000fea3   cl_ctx_timeout_insert
2000ff69   cl_ctx_timeout_update
2003c0e4   cli_cmd_count
2000e593   cmdDownload
2000e607   cmdSendData
2003a6ac   cmd_tbl
20016121   collectCC26XXSensorData
20012321   comm_close
20012189   comm_open
20014917   configureAutoScan
200220b1   copy_in
2003bd48   debug_printf
2003b8f4   device_hdl
200149a5   disableAutoconnect
20014995   doHandleCmdtimeout
2001449d   doPeriodicScan
200091cd   dummy_print
200149bb   enableAutoconnect
2001497d   enforceCC26XXFwChecsum
2000e1c5   eraseFlashRange
20022101   exit
200110a3   fillBondDefaultCfg
2001451f   fillDefaultCfgVal
200091d9   fillMqttDefaultCfg
200154ed   fillOtaMetaDefaultCfg
2000c627   fnPtrCLIPRINT
2000c6d5   fnPtrDevCharListCLIPRINT
20009695   fnPtrDevCharListHttpPRINT
200071d9   fnPtrDevCharListMqttPrint
200095c7   fnPtrHTTPconnlist
200094f7   fnPtrHTTPscanlist
20008b59   fnPtrMqttAddCon
2000868d   fnPtrMqttAdvBuild
20008759   fnPtrMqttConBuild
2000cdcb   fnPtrPairPRINT
20023b5d   free
2003c0a7   gAckEvent
2003c0a6   gCC2650Packet
2003c0e5   gCLIChar
2003c0e0   gFirstCmdMode
2003af64   gGapPacket
2003af94   gGattPacket
2003b178   gIntHdlr
2003b17c   gNPI_SyncObj
2003c0c0   gNpiReady
2003c0a5   gOutGoingPacket
2003c083   gSblDone
2003abec   g_CdnClient
2003c110   g_ConsecutiveNetAccessNetErrors
2003b0c0   g_FlcSflashCb
2003b180   g_GWGenSyncObj
2002614c   g_H2NCnysPattern
20026144   g_H2NSyncPattern
2003b124   g_LogClient
2003b184   g_Mqtt_queue
2003add4   g_OtaApp
2003ae20   g_OtaApp_statistics
200384a0   g_OtaCheckUpdateResponse
2003b014   g_OtaClient
200394e8   g_OtaFileMetadata
2003c0cc   g_SpiFd
2003a534   g_StatMem
2003b190   g_cDummy
2003c0b6   g_charIndex
2003c0b5   g_connIndex
2003bc50   g_gettoken_conn
2003b1e0   g_gettoken_getchar
2003bf04   g_gettoken_other
2003b9f0   g_gettoken_scan
2003c0a4   g_macAddressGet
2003c0a3   g_macAddressLen
2003b12c   g_macAddressVal
2003c0d5   g_multi_srvr_conn
2003c0d8   g_pCB
2003c0d0   g_pHostIntHdl
2003bab8   g_posttoken
2003b194   g_rx_task_hndl
2003b198   g_rx_tx_sync_obj
2003c0b4   g_scanIndex
2003c0a0   g_ucConnectedToConfAP
2003b134   g_ucConnectionBSSID
2003b038   g_ucConnectionSSID
2003c0d4   g_ucDMAEnabled
2003ad84   g_ucDinDout
2003b0bf   g_ucPacketEvent
2003b1dc   g_ucPacketLen
2003b1dd   g_ucPacketType
2003c0a2   g_ucPriority
2003c0a1   g_ucProvisioningDone
2003c0d6   g_ucStartUARTSend
20036700   g_ucUartAckRxBuffer
2003c0c9   g_ucUartByteCount
2003c0cb   g_ucUartPacketState
2003c0c8   g_ucUartReadLen
2003c0ca   g_ucUartReadState
20036f00   g_ucUartRxBuffer
2003c0c4   g_uiUartRxBufHead
2003c10c   g_uiUartRxBufTail
2003c09c   g_ulStatus
2003b19c   g_wait_secs
20010e99   gapBondMgrAddBond
20010f01   gapBondMgrEraseAllBondings
20010df7   gapBondMgrFindBondEntry
20010dbb   gapBondMgrFindEmpty
200148e1   gapBondMgrFlashBondRecUpdate
2003b13c   gapCentralRoleBdAddr
2003b0e4   gapCentralRoleIRK
2003c108   gapCentralRoleMaxScanRes
2003b0f4   gapCentralRoleSRK
2003c104   gapCentralRoleSignCounter
2000de67   generateCheckSum
2000df2f   getCmdResponse
20014499   getGenericTaskTicksPerSec
2000dff7   getResponseData
2001109d   getSizeofBondCfg
200091d5   getSizeofMqttCfg
200154e9   getSizeofOtaMeta
2000a62b   get_devState
2001352d   get_gwCallType
20013565   get_gwDevCnt
200134bf   get_gwState
2001357b   get_gw_devConnectionid
2001356d   get_gw_devState
2003b1a0   gw_blefi_linke_topic
2003b1a4   gw_blefi_linkt_topic
2003b1a8   gw_blefi_scan_topic
2003bcc8   gw_connect_config
2003ae6c   gw_connlist
2003ad28   gw_context
2000a801   gw_createDeviceRec
2003aefc   gw_link_message
2003ab74   gw_scanlist
2003acc4   gw_scanres_message
200135d1   gwcontext_Init
200135ff   gwcontext_IsScanIdValid
20013205   http_build_request
20013127   http_connect_server
200130bd   http_extract_domain_by_url
200130b9   http_recv_buf
200130b5   http_send_buf
20012feb   http_skip_headers
20007f41   is_anyDeviceMqttConnected
2003bf37   is_bleStackReady
2003c0a8   is_blefiCfgReady
2003c0a9   is_blefiCfgupdate
2003bf36   is_notiEnable
2003c098   is_slReady
2000e9e1   itoa
20013e8f   jsmn_init
20013b7d   jsmn_parse
20012f89   json_parse_dropbox_media_url
20012e41   json_parse_dropbox_metadata
20012e07   json_parse_rsrc_metadata_url
20012ce5   json_parse_update_check_resp
2003af30   listcharstr
200177b3   local_filter
20021629   ltoa
2001b863   main
2003c118   main_func_sp
20022da5   malloc
20015f2f   mem_Free
20015f23   mem_Malloc
20015f4f   mem_copy
20015f3b   mem_set
20023751   memccpy
200233bd   memcmp
2001f6e9   memcpy
20023185   memmove
200209cd   memset
2000fa71   mqp_ack_wlist_append
2000fb17   mqp_ack_wlist_purge
2000faa7   mqp_ack_wlist_remove
2000f7fd   mqp_buf_rd_remlen
2000f78d   mqp_buf_tail_wr_remlen
2000f71b   mqp_buf_wr_utf8
20006399   mqp_client_alloc
2000f675   mqp_free
2000f6c1   mqp_init
2000fb69   mqp_prep_fh
2000f999   mqp_proc_msg_id_ack_rx
2000f9cf   mqp_proc_pub_rx
2000f98d   mqp_proc_vh_msg_id_rx
2000f8bd   mqp_pub_append_data
2000f80d   mqp_pub_append_topic
2000fbdf   mqp_recv
2000f6b5   mqp_reset
20008da5   mqttCleanupCtx
2003c0ec   mqttDevMode
2003bfac   mqttGwMode
20007f81   mqttPublishData
2003b1ac   mqttQStimeout
2000628d   mqtt_client_await_msg
200063ed   mqtt_client_buffers_register
20005f81   mqtt_client_ctx_await_msg
20006675   mqtt_client_ctx_create
20006727   mqtt_client_ctx_delete
200064f9   mqtt_client_ctx_info_register
20005fd3   mqtt_client_ctx_run
20006471   mqtt_client_ctx_will_register
20004955   mqtt_client_is_connected
20006809   mqtt_client_lib_exit
20006789   mqtt_client_lib_init
20006579   mqtt_client_net_svc_register
2000494d   mqtt_client_new_msg_id
2000512b   mqtt_client_pub_dispatch
2000509d   mqtt_client_pub_msg_send
200062f5   mqtt_client_run
20004b0d   mqtt_client_send_progress
20004f4d   mqtt_connect_msg_send
2003bdd0   mqtt_device_cfg
2003c0ee   mqtt_device_connected
20005497   mqtt_disconn_send
2003b1b0   mqtt_lib_lockobj
2000545b   mqtt_pingreq_send
20005373   mqtt_sub_dispatch
2000535d   mqtt_sub_msg_send
2000539d   mqtt_unsub_dispatch
20005387   mqtt_unsub_msg_send
2001033d   mutex_lockup
2001034d   mutex_unlock
2003bff0   net
200160cb   osi_ContextRestore
200160c9   osi_ContextSave
20015f63   osi_EnterCritical
20015f75   osi_ExitCritical
20015c43   osi_InterruptDeRegister
20015beb   osi_InterruptRegister
20015d45   osi_LockObjCreate
20015ded   osi_LockObjDelete
20015dfb   osi_LockObjLock
20015e53   osi_LockObjUnlock
20015f81   osi_MsgQCreate
20015fb7   osi_MsgQDelete
2001602b   osi_MsgQRead
20015fc5   osi_MsgQWrite
2001608d   osi_Sleep
20015e63   osi_Spawn
20015d2d   osi_SyncObjClear
20015c5f   osi_SyncObjCreate
20015ca7   osi_SyncObjDelete
20015cb5   osi_SyncObjSignal
20015cc5   osi_SyncObjSignalFromISR
20015cd5   osi_SyncObjWait
20015d87   osi_TaskCreate
20015de1   osi_TaskDelete
200160ad   osi_TaskDisable
200160b5   osi_TaskEnable
200160c1   osi_start
200154c7   otaSignalWLANConnect
2003b1b4   pGC_StateCB
2003b1b8   pNpiEvtCb
2003c0dc   pPingCallBackFunc
2003b1bc   pcliSyncObj
2002348d   platform_get_time_in_secs
20023485   platform_timer_init
200160ed   pow
20012c75   printScanResponse
2000d399   print_usage
2001a2c3   process_GATTFindCharDescs
2001a2b3   process_GattDiscAllChars
2001a2a7   process_GattDiscAllPrimaryServices
2001a31f   process_GattReadUsingCharUuid
2001a251   process_LinkEstablish
2001a287   process_LinkTerminate
2001a2d3   process_ReadHandle
2001a211   process_Scan
2001a243   process_ScanStop
2001a2e1   process_WriteHandle
2003bf98   pub_gw_blefi_find_topic
2003bfa0   pub_gw_linkeres_topic
2003bfa4   pub_gw_linktres_topic
2003bf9c   pub_gw_scanres_topic
2001628f   publishCC26XXSensorData
2000fe03   qos2_pub_cq_check
2000fd81   qos2_pub_cq_logup
2000fd5f   qos2_pub_cq_reset
2000fdbf   qos2_pub_cq_unlog
20014961   readAutoScan
20008049   readDevMqttCfg
2000932d   readGwMqttCfg
2000e117   readStatus
20022499   realloc
20012591   recv_from
20012333   rtc_secs
2003b1c4   sGC_AppMsgQueue
2003b1c8   sGC_StackMsgQueue
2003b1cc   sMsg
2003b1d0   sblFileHandle
200116dd   sblUARTinit
2000de2b   sbl_close_bin
2000ddbf   sbl_get_bin_size
2000dda5   sbl_min
2000dde7   sbl_open_bin_for_read
2000de43   sbl_read_bin
20011ccf   sch_char_to_hex
20011dbd   sch_copy_char_uuid
20011ea5   sch_copy_charstring
20011cdf   sch_copy_serv_uuid
2003afec   sch_nvmemload
2000fb49   secure_conn_struct_init
2003bb4e   selfEntity
2000dfbd   sendAutoBaud
2000deab   sendCmd
2000e0c3   sendCmdResponse
20012511   send_dest
20016371   sensorTagEnableNoti
2003a7fc   sensor_message
2000a617   set_devState
200134e9   set_gwCallType
200134c5   set_gwState
2003b1d4   simpleLink_mailbox
2001c541   sl_Accept
20020125   sl_Bind
20022c25   sl_Close
2001d559   sl_Connect
200104d5   sl_ExtLib_MqttClientConnect
200101e5   sl_ExtLib_MqttClientCtxCreate
20010303   sl_ExtLib_MqttClientCtxDelete
20010635   sl_ExtLib_MqttClientDisconnect
20010425   sl_ExtLib_MqttClientExit
2001035d   sl_ExtLib_MqttClientInit
20010855   sl_ExtLib_MqttClientSend
20010479   sl_ExtLib_MqttClientSet
200106a1   sl_ExtLib_MqttClientSub
20010789   sl_ExtLib_MqttClientUnsub
200201ad   sl_FsClose
2002192d   sl_FsDel
200208d1   sl_FsGetInfo
20020a3d   sl_FsOpen
2001de71   sl_FsRead
2001e055   sl_FsWrite
20022357   sl_Htonl
2002258d   sl_Htons
200225c9   sl_Listen
2001d86d   sl_NetAppDnsGetHostByName
2001f1c5   sl_NetCfgGet
20020b2d   sl_Recv
2001d44d   sl_RecvFrom
20012cbd   sl_Recv_eagain
2001c2c9   sl_Select
2001d661   sl_Send
2001d119   sl_SendTo
20020e9d   sl_SetSockOpt
2002145d   sl_Socket
2001eac9   sl_Start
20019b71   sl_WlanConnect
20023fa9   sl_WlanDisconnect
2002127d   sl_WlanPolicySet
20019471   sl_WlanProfileAdd
2001fc41   sl_WlanSmartConfigStart
20023fb5   sl_WlanSmartConfigStop
20017a6b   sl_extLib_OtaGet
20017a03   sl_extLib_OtaInit
200177f9   sl_extLib_OtaRun
200176e7   sl_extLib_OtaSet
2001b769   sl_extlib_FlcAbortFile
2001b761   sl_extlib_FlcCloseFile
2001b729   sl_extlib_FlcCommit
2001b711   sl_extlib_FlcIsPendingCommit
2001b6cf   sl_extlib_FlcOpenFile
2001b6bd   sl_extlib_FlcReadFile
2001b68f   sl_extlib_FlcTest
2001b631   sl_extlib_FlcWriteFile
2001c039   spi_Open
2001e141   spi_Read
2001ff01   spi_Write
200211bd   sprintf
200238eb   strcat
20023ba5   strcmp
20023e39   strcpy
200233df   strcspn
20023d11   strlen
200230a7   strncmp
20022bf5   strncpy
20022f8d   strspn
20022995   strstr
200223d9   strtok
2001d231   strtoul
200124a3   tcp_accept
2001233b   tcp_listen
200122c1   tcp_recv
200123c7   tcp_select
2001229b   tcp_send
2003c018   ti_sysbios_BIOS_Module__state__V
200240d7   ti_sysbios_BIOS_RtsGateProxy_enter__E
200240db   ti_sysbios_BIOS_RtsGateProxy_leave__E
200240ef   ti_sysbios_BIOS_RtsGateProxy_query__E
20022c55   ti_sysbios_BIOS_atExitFunc__I
200231a9   ti_sysbios_BIOS_errorRaiseHook__I
20023cbd   ti_sysbios_BIOS_exitFunc__I
20011863   ti_sysbios_BIOS_nullFunc__I
200231cd   ti_sysbios_BIOS_registerRTSLock__I
200231f1   ti_sysbios_BIOS_removeRTSLock__I
2002376d   ti_sysbios_BIOS_rtsLock__I
20023bbd   ti_sysbios_BIOS_rtsUnlock__I
20023e49   ti_sysbios_BIOS_setThreadType__E
20023215   ti_sysbios_BIOS_startFunc__I
20023e59   ti_sysbios_BIOS_start__E
20026668   ti_sysbios_family_arm_m3_Hwi_E_NMI__C
2002666c   ti_sysbios_family_arm_m3_Hwi_E_alreadyDefined__C
20026670   ti_sysbios_family_arm_m3_Hwi_E_busFault__C
20026674   ti_sysbios_family_arm_m3_Hwi_E_debugMon__C
20026678   ti_sysbios_family_arm_m3_Hwi_E_hardFault__C
2002667c   ti_sysbios_family_arm_m3_Hwi_E_memFault__C
20026680   ti_sysbios_family_arm_m3_Hwi_E_noIsr__C
20026684   ti_sysbios_family_arm_m3_Hwi_E_reserved__C
20026688   ti_sysbios_family_arm_m3_Hwi_E_svCall__C
2002668c   ti_sysbios_family_arm_m3_Hwi_E_usageFault__C
20023905   ti_sysbios_family_arm_m3_Hwi_Handle__label__S
20022e85   ti_sysbios_family_arm_m3_Hwi_Instance_finalize__E
2001f785   ti_sysbios_family_arm_m3_Hwi_Instance_init__E
20026690   ti_sysbios_family_arm_m3_Hwi_LD_end__C
20026694   ti_sysbios_family_arm_m3_Hwi_LM_begin__C
2003b7dc   ti_sysbios_family_arm_m3_Hwi_Module_State_0_excActive__A
2003b7e0   ti_sysbios_family_arm_m3_Hwi_Module_State_0_excContext__A
2003b7e4   ti_sysbios_family_arm_m3_Hwi_Module_State_0_excStack__A
20026698   ti_sysbios_family_arm_m3_Hwi_Module__diagsEnabled__C
2002669c   ti_sysbios_family_arm_m3_Hwi_Module__diagsIncluded__C
200266a0   ti_sysbios_family_arm_m3_Hwi_Module__diagsMask__C
20025d4a   ti_sysbios_family_arm_m3_Hwi_Module__id__C
20026312   ti_sysbios_family_arm_m3_Hwi_Module__loggerDefined__C
200266a4   ti_sysbios_family_arm_m3_Hwi_Module__loggerFxn1__C
200266a8   ti_sysbios_family_arm_m3_Hwi_Module__loggerFxn8__C
200266ac   ti_sysbios_family_arm_m3_Hwi_Module__loggerObj__C
2003b7bc   ti_sysbios_family_arm_m3_Hwi_Module__root__V
20023bd5   ti_sysbios_family_arm_m3_Hwi_Module__startupDone__F
20023bd5   ti_sysbios_family_arm_m3_Hwi_Module__startupDone__S
2003bed0   ti_sysbios_family_arm_m3_Hwi_Module__state__V
2001e7c9   ti_sysbios_family_arm_m3_Hwi_Module_startup__E
200266b0   ti_sysbios_family_arm_m3_Hwi_NUM_INTERRUPTS__C
2002640c   ti_sysbios_family_arm_m3_Hwi_Object__DESC__C
200261e0   ti_sysbios_family_arm_m3_Hwi_Object__PARAMS__C
200266b4   ti_sysbios_family_arm_m3_Hwi_Object__count__C
200234a5   ti_sysbios_family_arm_m3_Hwi_Object__delete__S
20023d25   ti_sysbios_family_arm_m3_Hwi_Object__get__S
2003b7c4   ti_sysbios_family_arm_m3_Hwi_Object__table__V
20023fc1   ti_sysbios_family_arm_m3_Hwi_Params__init__S
200266b8   ti_sysbios_family_arm_m3_Hwi_ccr__C
20020f6d   ti_sysbios_family_arm_m3_Hwi_create
200240df   ti_sysbios_family_arm_m3_Hwi_delete
20023fcd   ti_sysbios_family_arm_m3_Hwi_disableFxn__E
2002217d   ti_sysbios_family_arm_m3_Hwi_disableInterrupt__E
2001c405   ti_sysbios_family_arm_m3_Hwi_dispatchC__I
200398c0   ti_sysbios_family_arm_m3_Hwi_dispatchTable
2001e49d   ti_sysbios_family_arm_m3_Hwi_dispatch__I
2002408b   ti_sysbios_family_arm_m3_Hwi_doSwiRestore__I
20023239   ti_sysbios_family_arm_m3_Hwi_doTaskRestore__I
200221c1   ti_sysbios_family_arm_m3_Hwi_enableInterrupt__E
2001bc1d   ti_sysbios_family_arm_m3_Hwi_excBusFault__I
2001efc5   ti_sysbios_family_arm_m3_Hwi_excDebugMon__I
200172a5   ti_sysbios_family_arm_m3_Hwi_excDumpRegs__I
200234c5   ti_sysbios_family_arm_m3_Hwi_excHandlerAsm__I
200266bc   ti_sysbios_family_arm_m3_Hwi_excHandlerFunc__C
2001a639   ti_sysbios_family_arm_m3_Hwi_excHandlerMax__I
200234e5   ti_sysbios_family_arm_m3_Hwi_excHandler__I
2001ecf9   ti_sysbios_family_arm_m3_Hwi_excHardFault__I
20026648   ti_sysbios_family_arm_m3_Hwi_excHookFuncs__A
200266c0   ti_sysbios_family_arm_m3_Hwi_excHookFuncs__C
2001c189   ti_sysbios_family_arm_m3_Hwi_excMemFault__I
200229c9   ti_sysbios_family_arm_m3_Hwi_excNmi__I
200227a5   ti_sysbios_family_arm_m3_Hwi_excNoIsr__I
20021e35   ti_sysbios_family_arm_m3_Hwi_excReserved__I
20022605   ti_sysbios_family_arm_m3_Hwi_excSvCall__I
2001bee5   ti_sysbios_family_arm_m3_Hwi_excUsageFault__I
20023e69   ti_sysbios_family_arm_m3_Hwi_getHandle__E
200227dd   ti_sysbios_family_arm_m3_Hwi_getStackInfo__E
2002044d   ti_sysbios_family_arm_m3_Hwi_initNVIC__E
20021e7d   ti_sysbios_family_arm_m3_Hwi_initStacks__E
200266c4   ti_sysbios_family_arm_m3_Hwi_nullIsrFunc__C
e000e000   ti_sysbios_family_arm_m3_Hwi_nvic
2002391f   ti_sysbios_family_arm_m3_Hwi_pendSV__I
20020ba1   ti_sysbios_family_arm_m3_Hwi_postInit__I
200266c8   ti_sysbios_family_arm_m3_Hwi_priGroup__C
20004000   ti_sysbios_family_arm_m3_Hwi_resetVectors
200240b5   ti_sysbios_family_arm_m3_Hwi_restoreFxn__E
20023937   ti_sysbios_family_arm_m3_Hwi_return
20023789   ti_sysbios_family_arm_m3_Hwi_setPriority__E
20024093   ti_sysbios_family_arm_m3_Hwi_startup__E
20023d39   ti_sysbios_family_arm_m3_Hwi_switchFromBootStack__E
200240e3   ti_sysbios_family_arm_m3_TaskSupport_Module__startupDone__S
20021be5   ti_sysbios_family_arm_m3_TaskSupport_buildTaskStack
20023fd9   ti_sysbios_family_arm_m3_TaskSupport_checkStack__E
20023fe5   ti_sysbios_family_arm_m3_TaskSupport_getStackAlignment__E
20023e79   ti_sysbios_family_arm_m3_TaskSupport_glue
200266cc   ti_sysbios_family_arm_m3_TaskSupport_stackAlignment__C
20022815   ti_sysbios_family_arm_m3_TaskSupport_start__E
20023e89   ti_sysbios_family_arm_m3_TaskSupport_swap__E
200266d0   ti_sysbios_family_arm_m3_Timer_E_cannotSupport__C
20026562   ti_sysbios_family_arm_m3_Timer_Module__id__C
2003b7e8   ti_sysbios_family_arm_m3_Timer_Module__root__V
20023bed   ti_sysbios_family_arm_m3_Timer_Module__startupDone__F
20023bed   ti_sysbios_family_arm_m3_Timer_Module__startupDone__S
2003b7f0   ti_sysbios_family_arm_m3_Timer_Module__state__V
20022419   ti_sysbios_family_arm_m3_Timer_Module_startup__E
2003bf38   ti_sysbios_family_arm_m3_Timer_Object__table__V
200240e7   ti_sysbios_family_arm_m3_Timer_getMaxTicks__E
20021ec5   ti_sysbios_family_arm_m3_Timer_initDevice__I
200229fd   ti_sysbios_family_arm_m3_Timer_periodicStub__I
200214b9   ti_sysbios_family_arm_m3_Timer_setPeriod__E
20021839   ti_sysbios_family_arm_m3_Timer_start__E
200266d4   ti_sysbios_family_arm_m3_Timer_startupNeeded__C
2002325d   ti_sysbios_family_arm_m3_Timer_startup__E
2003b7fc   ti_sysbios_family_arm_m3_TimestampProvider_Module__state__V
20023505   ti_sysbios_family_arm_m3_TimestampProvider_Module_startup__E
200268e0   ti_sysbios_family_arm_m3_TimestampProvider_configTimer__C
200212dd   ti_sysbios_family_arm_m3_TimestampProvider_get64__E
200236df   ti_sysbios_family_xxx_Hwi_switchAndRunFunc
20023939   ti_sysbios_gates_GateHwi_Handle__label__S
200184f7   ti_sysbios_gates_GateHwi_Instance_init__E
20026314   ti_sysbios_gates_GateHwi_Module__FXNS__C
2003b800   ti_sysbios_gates_GateHwi_Module__root__V
2002642c   ti_sysbios_gates_GateHwi_Object__DESC__C
2002657c   ti_sysbios_gates_GateHwi_Object__PARAMS__C
20022c85   ti_sysbios_gates_GateHwi_Object__create__S
20023525   ti_sysbios_gates_GateHwi_Object__delete__S
2003b808   ti_sysbios_gates_GateHwi_Object__table__V
20023ff1   ti_sysbios_gates_GateHwi_enter__E
200240bb   ti_sysbios_gates_GateHwi_leave__E
200240eb   ti_sysbios_gates_GateHwi_query__E
200266d8   ti_sysbios_gates_GateMutex_A_badContext__C
20023953   ti_sysbios_gates_GateMutex_Handle__label__S
200266dc   ti_sysbios_gates_GateMutex_Instance_State_sem__O
20023e99   ti_sysbios_gates_GateMutex_Instance_finalize__E
200237a5   ti_sysbios_gates_GateMutex_Instance_init__E
20026338   ti_sysbios_gates_GateMutex_Module__FXNS__C
200266e0   ti_sysbios_gates_GateMutex_Module__diagsEnabled__C
200266e4   ti_sysbios_gates_GateMutex_Module__diagsIncluded__C
200266e8   ti_sysbios_gates_GateMutex_Module__diagsMask__C
200268e2   ti_sysbios_gates_GateMutex_Module__id__C
2003b80c   ti_sysbios_gates_GateMutex_Module__root__V
2002644c   ti_sysbios_gates_GateMutex_Object__DESC__C
20026594   ti_sysbios_gates_GateMutex_Object__PARAMS__C
20022cb5   ti_sysbios_gates_GateMutex_Object__create__S
20023281   ti_sysbios_gates_GateMutex_Object__delete__S
2003be98   ti_sysbios_gates_GateMutex_Object__table__V
2001edad   ti_sysbios_gates_GateMutex_enter__E
20023c05   ti_sysbios_gates_GateMutex_leave__E
200240ef   ti_sysbios_gates_GateMutex_query__E
200266ec   ti_sysbios_hal_Hwi_E_stackOverflow__C
200240f3   ti_sysbios_hal_Hwi_HwiProxy_Module__startupDone__S
2002217d   ti_sysbios_hal_Hwi_HwiProxy_disableInterrupt__E
20023fcd   ti_sysbios_hal_Hwi_HwiProxy_disable__E
200221c1   ti_sysbios_hal_Hwi_HwiProxy_enableInterrupt__E
200227dd   ti_sysbios_hal_Hwi_HwiProxy_getStackInfo__E
200240b5   ti_sysbios_hal_Hwi_HwiProxy_restore__E
20024093   ti_sysbios_hal_Hwi_HwiProxy_startup__E
20023d39   ti_sysbios_hal_Hwi_HwiProxy_switchFromBootStack__E
200268e4   ti_sysbios_hal_Hwi_Module__id__C
2003b814   ti_sysbios_hal_Hwi_Module__root__V
20023dad   ti_sysbios_hal_Hwi_Module_startup__E
20022a31   ti_sysbios_hal_Hwi_checkStack
2002217d   ti_sysbios_hal_Hwi_disableInterrupt__E
20023fcd   ti_sysbios_hal_Hwi_disable__E
200221c1   ti_sysbios_hal_Hwi_enableInterrupt__E
200227dd   ti_sysbios_hal_Hwi_getStackInfo__E
20022eb1   ti_sysbios_hal_Hwi_initStack
200240b5   ti_sysbios_hal_Hwi_restore__E
20024093   ti_sysbios_hal_Hwi_startup__E
2003b81c   ti_sysbios_hal_Timer_Module__root__V
20023dbf   ti_sysbios_hal_Timer_Module_startup__E
200240f7   ti_sysbios_hal_Timer_TimerProxy_Module__startupDone__S
2002325d   ti_sysbios_hal_Timer_TimerProxy_startup__E
2002325d   ti_sysbios_hal_Timer_startup__E
200266f0   ti_sysbios_heaps_HeapMem_A_align__C
200266f4   ti_sysbios_heaps_HeapMem_A_heapSize__C
200266f8   ti_sysbios_heaps_HeapMem_A_invalidFree__C
200266fc   ti_sysbios_heaps_HeapMem_A_zeroBlock__C
20026700   ti_sysbios_heaps_HeapMem_E_memory__C
2002396d   ti_sysbios_heaps_HeapMem_Handle__label__S
2002bf00   ti_sysbios_heaps_HeapMem_Instance_State_0_buf__A
2001c679   ti_sysbios_heaps_HeapMem_Instance_init__E
200240fb   ti_sysbios_heaps_HeapMem_Module_GateProxy_enter__E
200240ff   ti_sysbios_heaps_HeapMem_Module_GateProxy_leave__E
200240ef   ti_sysbios_heaps_HeapMem_Module_GateProxy_query__E
200262c4   ti_sysbios_heaps_HeapMem_Module__FXNS__C
20026704   ti_sysbios_heaps_HeapMem_Module__diagsEnabled__C
20026708   ti_sysbios_heaps_HeapMem_Module__diagsIncluded__C
2002670c   ti_sysbios_heaps_HeapMem_Module__diagsMask__C
20026710   ti_sysbios_heaps_HeapMem_Module__gateObj__C
200268e6   ti_sysbios_heaps_HeapMem_Module__id__C
2003b824   ti_sysbios_heaps_HeapMem_Module__root__V
2002646c   ti_sysbios_heaps_HeapMem_Object__DESC__C
2002635c   ti_sysbios_heaps_HeapMem_Object__PARAMS__C
20026714   ti_sysbios_heaps_HeapMem_Object__count__C
20022ce5   ti_sysbios_heaps_HeapMem_Object__create__S
20023545   ti_sysbios_heaps_HeapMem_Object__delete__S
20023d4d   ti_sysbios_heaps_HeapMem_Object__get__S
2003b82c   ti_sysbios_heaps_HeapMem_Object__table__V
20019db5   ti_sysbios_heaps_HeapMem_alloc__E
20019929   ti_sysbios_heaps_HeapMem_free__E
20021f0d   ti_sysbios_heaps_HeapMem_getStats__E
20022641   ti_sysbios_heaps_HeapMem_init__I
200240c1   ti_sysbios_heaps_HeapMem_isBlocking__E
20026718   ti_sysbios_heaps_HeapMem_reqAlign__C
2002671c   ti_sysbios_knl_Clock_LM_begin__C
20026720   ti_sysbios_knl_Clock_LM_tick__C
20026724   ti_sysbios_knl_Clock_LW_delayed__C
20026728   ti_sysbios_knl_Clock_Module_State_clockQ__O
2002672c   ti_sysbios_knl_Clock_Module__diagsEnabled__C
20026730   ti_sysbios_knl_Clock_Module__diagsIncluded__C
20026734   ti_sysbios_knl_Clock_Module__diagsMask__C
200268e8   ti_sysbios_knl_Clock_Module__id__C
200268ea   ti_sysbios_knl_Clock_Module__loggerDefined__C
20026738   ti_sysbios_knl_Clock_Module__loggerFxn1__C
2002673c   ti_sysbios_knl_Clock_Module__loggerFxn2__C
20026740   ti_sysbios_knl_Clock_Module__loggerObj__C
2003b844   ti_sysbios_knl_Clock_Module__root__V
2003bfc4   ti_sysbios_knl_Clock_Module__state__V
200232a5   ti_sysbios_knl_Clock_Module_startup__E
20024103   ti_sysbios_knl_Clock_TimerProxy_Module__startupDone__S
20024107   ti_sysbios_knl_Clock_TimerProxy_getMaxTicks__E
2002325d   ti_sysbios_knl_Clock_TimerProxy_startup__E
20022edd   ti_sysbios_knl_Clock_doTick__I
2002133d   ti_sysbios_knl_Clock_logTick__E
20026744   ti_sysbios_knl_Clock_tickPeriod__C
2001cc85   ti_sysbios_knl_Clock_workFunc__E
2003b84c   ti_sysbios_knl_Event_Module__root__V
20026748   ti_sysbios_knl_Idle_funcList__A
20026650   ti_sysbios_knl_Idle_funcList__C
2002409b   ti_sysbios_knl_Idle_loop__E
20023565   ti_sysbios_knl_Idle_run__E
2002674c   ti_sysbios_knl_Mailbox_A_invalidBufSize__C
20026750   ti_sysbios_knl_Mailbox_Instance_State_dataQue__O
20026754   ti_sysbios_knl_Mailbox_Instance_State_dataSem__O
20026758   ti_sysbios_knl_Mailbox_Instance_State_freeQue__O
2002675c   ti_sysbios_knl_Mailbox_Instance_State_freeSem__O
20020c11   ti_sysbios_knl_Mailbox_Instance_finalize__E
2001bd85   ti_sysbios_knl_Mailbox_Instance_init__E
20026760   ti_sysbios_knl_Mailbox_Module__diagsEnabled__C
20026764   ti_sysbios_knl_Mailbox_Module__diagsIncluded__C
20026768   ti_sysbios_knl_Mailbox_Module__diagsMask__C
200268ec   ti_sysbios_knl_Mailbox_Module__id__C
2003b854   ti_sysbios_knl_Mailbox_Module__root__V
20020235   ti_sysbios_knl_Mailbox_Module_startup__E
2002648c   ti_sysbios_knl_Mailbox_Object__DESC__C
200261ac   ti_sysbios_knl_Mailbox_Object__PARAMS__C
2002676c   ti_sysbios_knl_Mailbox_Object__count__C
20023585   ti_sysbios_knl_Mailbox_Object__delete__S
20023ea9   ti_sysbios_knl_Mailbox_Object__get__S
20020fd1   ti_sysbios_knl_Mailbox_create
2002410b   ti_sysbios_knl_Mailbox_delete
20026770   ti_sysbios_knl_Mailbox_maxTypeAlign__C
200204d1   ti_sysbios_knl_Mailbox_pend__E
20022459   ti_sysbios_knl_Mailbox_postInit__I
2001fa85   ti_sysbios_knl_Mailbox_post__E
200240c7   ti_sysbios_knl_Queue_Instance_init__E
2003b85c   ti_sysbios_knl_Queue_Module__root__V
200264ac   ti_sysbios_knl_Queue_Object__DESC__C
200265ac   ti_sysbios_knl_Queue_Object__PARAMS__C
200237c1   ti_sysbios_knl_Queue_Object__destruct__S
20023ffd   ti_sysbios_knl_Queue_Object__get__S
20022f09   ti_sysbios_knl_Queue_construct
2002410f   ti_sysbios_knl_Queue_destruct
20023f83   ti_sysbios_knl_Queue_empty__E
20026774   ti_sysbios_knl_Semaphore_A_badContext__C
20026778   ti_sysbios_knl_Semaphore_A_noEvents__C
2002677c   ti_sysbios_knl_Semaphore_A_overflow__C
20026780   ti_sysbios_knl_Semaphore_A_pendTaskDisabled__C
20026784   ti_sysbios_knl_Semaphore_Instance_State_pendQ__O
20023eb9   ti_sysbios_knl_Semaphore_Instance_finalize__E
2001f821   ti_sysbios_knl_Semaphore_Instance_init__E
20026788   ti_sysbios_knl_Semaphore_LM_pend__C
2002678c   ti_sysbios_knl_Semaphore_LM_post__C
20026790   ti_sysbios_knl_Semaphore_Module__diagsEnabled__C
20026794   ti_sysbios_knl_Semaphore_Module__diagsIncluded__C
20026798   ti_sysbios_knl_Semaphore_Module__diagsMask__C
200268ee   ti_sysbios_knl_Semaphore_Module__id__C
200268f0   ti_sysbios_knl_Semaphore_Module__loggerDefined__C
2002679c   ti_sysbios_knl_Semaphore_Module__loggerFxn2__C
200267a0   ti_sysbios_knl_Semaphore_Module__loggerFxn4__C
200267a4   ti_sysbios_knl_Semaphore_Module__loggerObj__C
2003b864   ti_sysbios_knl_Semaphore_Module__root__V
200264cc   ti_sysbios_knl_Semaphore_Object__DESC__C
20026380   ti_sysbios_knl_Semaphore_Object__PARAMS__C
200232c9   ti_sysbios_knl_Semaphore_Object__delete__S
200235a5   ti_sysbios_knl_Semaphore_Object__destruct__S
20024009   ti_sysbios_knl_Semaphore_Params__init__S
20022d15   ti_sysbios_knl_Semaphore_construct
20022a65   ti_sysbios_knl_Semaphore_create
20024113   ti_sysbios_knl_Semaphore_delete
20024117   ti_sysbios_knl_Semaphore_destruct
20022b01   ti_sysbios_knl_Semaphore_pendTimeout__I
20018e99   ti_sysbios_knl_Semaphore_pend__E
2001c7b1   ti_sysbios_knl_Semaphore_post__E
20023987   ti_sysbios_knl_Swi_Handle__label__S
200267a8   ti_sysbios_knl_Swi_LD_end__C
200267ac   ti_sysbios_knl_Swi_LM_begin__C
200267b0   ti_sysbios_knl_Swi_LM_post__C
2003bb50   ti_sysbios_knl_Swi_Module_State_0_readyQ__A
200267b4   ti_sysbios_knl_Swi_Module__diagsEnabled__C
200267b8   ti_sysbios_knl_Swi_Module__diagsIncluded__C
200267bc   ti_sysbios_knl_Swi_Module__diagsMask__C
200268f2   ti_sysbios_knl_Swi_Module__id__C
200268f4   ti_sysbios_knl_Swi_Module__loggerDefined__C
200267c0   ti_sysbios_knl_Swi_Module__loggerFxn1__C
200267c4   ti_sysbios_knl_Swi_Module__loggerFxn4__C
200267c8   ti_sysbios_knl_Swi_Module__loggerObj__C
2003b86c   ti_sysbios_knl_Swi_Module__root__V
2003b874   ti_sysbios_knl_Swi_Module__state__V
200232ed   ti_sysbios_knl_Swi_Module_startup__E
200267cc   ti_sysbios_knl_Swi_Object__count__C
20023d61   ti_sysbios_knl_Swi_Object__get__S
2003bf68   ti_sysbios_knl_Swi_Object__table__V
20023ec9   ti_sysbios_knl_Swi_disable__E
2001f26d   ti_sysbios_knl_Swi_post__E
20021735   ti_sysbios_knl_Swi_restoreHwi__E
20021c31   ti_sysbios_knl_Swi_runLoop__I
2001ced9   ti_sysbios_knl_Swi_run__I
2002178d   ti_sysbios_knl_Swi_schedule__I
2002267d   ti_sysbios_knl_Swi_startup__E
200267d0   ti_sysbios_knl_Task_A_badPriority__C
200267d4   ti_sysbios_knl_Task_A_badTaskState__C
200267d8   ti_sysbios_knl_Task_A_badThreadType__C
200267dc   ti_sysbios_knl_Task_A_badTimeout__C
200267e0   ti_sysbios_knl_Task_A_noPendElem__C
200267e4   ti_sysbios_knl_Task_A_sleepTaskDisabled__C
200267e8   ti_sysbios_knl_Task_E_spOutOfBounds__C
200267ec   ti_sysbios_knl_Task_E_stackOverflow__C
200239a1   ti_sysbios_knl_Task_Handle__label__S
20037700   ti_sysbios_knl_Task_Instance_State_0_stack__A
20019fe9   ti_sysbios_knl_Task_Instance_finalize__E
2001afa1   ti_sysbios_knl_Task_Instance_init__E
200267f0   ti_sysbios_knl_Task_LD_block__C
200267f4   ti_sysbios_knl_Task_LD_exit__C
200267f8   ti_sysbios_knl_Task_LD_ready__C
200267fc   ti_sysbios_knl_Task_LM_sleep__C
20026800   ti_sysbios_knl_Task_LM_switch__C
20026804   ti_sysbios_knl_Task_LM_yield__C
2003b898   ti_sysbios_knl_Task_Module_State_0_idleTask__A
2003bbd0   ti_sysbios_knl_Task_Module_State_0_readyQ__A
20026808   ti_sysbios_knl_Task_Module_State_inactiveQ__O
2002680c   ti_sysbios_knl_Task_Module__diagsEnabled__C
20026810   ti_sysbios_knl_Task_Module__diagsIncluded__C
20026814   ti_sysbios_knl_Task_Module__diagsMask__C
200268f6   ti_sysbios_knl_Task_Module__id__C
200268f8   ti_sysbios_knl_Task_Module__loggerDefined__C
20026818   ti_sysbios_knl_Task_Module__loggerFxn2__C
2002681c   ti_sysbios_knl_Task_Module__loggerFxn4__C
20026820   ti_sysbios_knl_Task_Module__loggerObj__C
2003b890   ti_sysbios_knl_Task_Module__root__V
2003be18   ti_sysbios_knl_Task_Module__state__V
2001b4a5   ti_sysbios_knl_Task_Module_startup__E
200264ec   ti_sysbios_knl_Task_Object__DESC__C
20026024   ti_sysbios_knl_Task_Object__PARAMS__C
20026824   ti_sysbios_knl_Task_Object__count__C
200235c5   ti_sysbios_knl_Task_Object__delete__S
20023ed9   ti_sysbios_knl_Task_Object__get__S
2003bd84   ti_sysbios_knl_Task_Object__table__V
20024015   ti_sysbios_knl_Task_Params__init__S
2002411b   ti_sysbios_knl_Task_SupportProxy_Module__startupDone__S
20023fd9   ti_sysbios_knl_Task_SupportProxy_checkStack__E
20023fe5   ti_sysbios_knl_Task_SupportProxy_getStackAlignment__E
20022815   ti_sysbios_knl_Task_SupportProxy_start__E
20023e89   ti_sysbios_knl_Task_SupportProxy_swap__E
20026828   ti_sysbios_knl_Task_allBlockedFunc__C
20022205   ti_sysbios_knl_Task_allBlockedFunction__I
2001f315   ti_sysbios_knl_Task_blockI__E
2001ee61   ti_sysbios_knl_Task_checkStacks__E
20021515   ti_sysbios_knl_Task_create
2002682c   ti_sysbios_knl_Task_defaultStackHeap__C
20026830   ti_sysbios_knl_Task_defaultStackSize__C
2002411f   ti_sysbios_knl_Task_delete
20023ee9   ti_sysbios_knl_Task_disable__E
200235e5   ti_sysbios_knl_Task_enter__I
2001e94d   ti_sysbios_knl_Task_exit__E
200268fa   ti_sysbios_knl_Task_initStackFlag__C
20026834   ti_sysbios_knl_Task_numConstructedTasks__C
2001f3bd   ti_sysbios_knl_Task_postInit__I
2002284d   ti_sysbios_knl_Task_processVitalTaskFlag__I
20022f35   ti_sysbios_knl_Task_restore__E
2001e701   ti_sysbios_knl_Task_schedule__I
200239bb   ti_sysbios_knl_Task_sleepTimeout__I
2001a431   ti_sysbios_knl_Task_sleep__E
2001eb85   ti_sysbios_knl_Task_startCore__E
20024123   ti_sysbios_knl_Task_startup__E
20023e91   ti_sysbios_knl_Task_swapReturn
2001fb19   ti_sysbios_knl_Task_unblockI__E
2001f465   ti_sysbios_knl_Task_yield__E
2003b1d8   tokenList
2003c0b8   tokenmatch_conn_index
2003c0b9   tokenmatch_getchar_index
2003c0b7   tokenmatch_scan_index
2000cbcd   triggerOta
20021c7d   uDMAChannelAssign
20021035   uDMAChannelAttributeDisable
20021099   uDMAChannelAttributeEnable
200226b9   uDMAChannelControlSet
200237dd   uDMAChannelEnable
2001df65   uDMAChannelTransferSet
2000d1cb   uarta0IntFuncHandler
2000e19b   ulToCharArray
2002009d   vsnprintf
2003b154   wlan_mac
2001483b   writeBleCfg
2000e439   writeFlashRange
20026838   xdc_runtime_Assert_E_assertFailed__C
20021f55   xdc_runtime_Assert_raise__I
2002683c   xdc_runtime_Core_A_initializedParams__C
20026840   xdc_runtime_Core_Module__diagsEnabled__C
20026844   xdc_runtime_Core_Module__diagsIncluded__C
20026848   xdc_runtime_Core_Module__diagsMask__C
200268fc   xdc_runtime_Core_Module__id__C
20022a99   xdc_runtime_Core_assignLabel__I
20021f9d   xdc_runtime_Core_assignParams__I
2001e56d   xdc_runtime_Core_constructObject__I
2001d971   xdc_runtime_Core_createObject__I
20020f05   xdc_runtime_Core_deleteObject__I
2002684c   xdc_runtime_Error_E_memory__C
20026850   xdc_runtime_Error_Module__diagsEnabled__C
20026854   xdc_runtime_Error_Module__diagsIncluded__C
20026858   xdc_runtime_Error_Module__diagsMask__C
200268fe   xdc_runtime_Error_Module__loggerDefined__C
2002685c   xdc_runtime_Error_Module__loggerFxn8__C
20026860   xdc_runtime_Error_Module__loggerObj__C
2003b89c   xdc_runtime_Error_Module__state__V
20023c1d   xdc_runtime_Error_check__E
20024127   xdc_runtime_Error_getSite__E
20024021   xdc_runtime_Error_init__E
20026900   xdc_runtime_Error_maxDepth__C
2001cff9   xdc_runtime_Error_policyDefault__E
20026864   xdc_runtime_Error_policyFxn__C
200263eb   xdc_runtime_Error_policy__C
20020d5d   xdc_runtime_Error_print__E
20026868   xdc_runtime_Error_raiseHook__C
200237f9   xdc_runtime_Error_raiseX__E
20022249   xdc_runtime_Error_setX__E
2002402d   xdc_runtime_Gate_enterSystem__E
20023ef9   xdc_runtime_Gate_leaveSystem__E
2002686c   xdc_runtime_IFilterLogger_Interface__BASE__C
20026870   xdc_runtime_IGateProvider_Interface__BASE__C
20026874   xdc_runtime_IHeap_Interface__BASE__C
20026878   xdc_runtime_ILogger_Interface__BASE__C
2002687c   xdc_runtime_IModule_Interface__BASE__C
20026880   xdc_runtime_Log_L_error__C
20026884   xdc_runtime_LoggerBuf_E_badLevel__C
200239d5   xdc_runtime_LoggerBuf_Handle__label__S
200388ec   xdc_runtime_LoggerBuf_Instance_State_0_entryArr__A
20023dd1   xdc_runtime_LoggerBuf_Instance_finalize__E
20022731   xdc_runtime_LoggerBuf_Instance_init__E
2002412b   xdc_runtime_LoggerBuf_Module_GateProxy_enter__E
2002412f   xdc_runtime_LoggerBuf_Module_GateProxy_leave__E
200240eb   xdc_runtime_LoggerBuf_Module_GateProxy_query__E
20026060   xdc_runtime_LoggerBuf_Module__FXNS__C
20026888   xdc_runtime_LoggerBuf_Module__gateObj__C
20026902   xdc_runtime_LoggerBuf_Module__id__C
2003b8a0   xdc_runtime_LoggerBuf_Module__root__V
2003b8a8   xdc_runtime_LoggerBuf_Module__state__V
20023059   xdc_runtime_LoggerBuf_Module_startup__E
2002650c   xdc_runtime_LoggerBuf_Object__DESC__C
200263a4   xdc_runtime_LoggerBuf_Object__PARAMS__C
2002688c   xdc_runtime_LoggerBuf_Object__count__C
20021571   xdc_runtime_LoggerBuf_Object__create__S
20023605   xdc_runtime_LoggerBuf_Object__delete__S
20023d75   xdc_runtime_LoggerBuf_Object__get__S
2003c03c   xdc_runtime_LoggerBuf_Object__table__V
200212dd   xdc_runtime_LoggerBuf_TimestampProxy_get64__E
2002406f   xdc_runtime_LoggerBuf_disable__E
20024079   xdc_runtime_LoggerBuf_enable__E
20026904   xdc_runtime_LoggerBuf_filterByLevel__C
2002228d   xdc_runtime_LoggerBuf_filterOutEvent__I
20020dc9   xdc_runtime_LoggerBuf_getFilterLevel__E
20023625   xdc_runtime_LoggerBuf_reset__E
20020759   xdc_runtime_LoggerBuf_setFilterLevel__E
20026890   xdc_runtime_LoggerBuf_statusLogger__C
20023f09   xdc_runtime_LoggerBuf_write0__E
20023de3   xdc_runtime_LoggerBuf_write1__E
20023df5   xdc_runtime_LoggerBuf_write2__E
2001e2f5   xdc_runtime_LoggerBuf_write4__E
2001cb55   xdc_runtime_LoggerBuf_write8__E
200240eb   xdc_runtime_Main_Module_GateProxy_query__E
20024133   xdc_runtime_Memory_HeapProxy_alloc__E
20024137   xdc_runtime_Memory_HeapProxy_free__E
20026906   xdc_runtime_Memory_Module__id__C
2003b8b0   xdc_runtime_Memory_Module__state__V
20020c81   xdc_runtime_Memory_alloc__E
20024039   xdc_runtime_Memory_calloc__E
20026894   xdc_runtime_Memory_defaultHeapInstance__C
20023f19   xdc_runtime_Memory_free__E
20024045   xdc_runtime_Memory_getMaxDefaultTypeAlign__E
20023815   xdc_runtime_Memory_valloc__E
2003b8b4   xdc_runtime_Registry_Module__state__V
20023645   xdc_runtime_Registry_findById__E
2003b8bc   xdc_runtime_Startup_Module__state__V
00000001   xdc_runtime_Startup__EXECFXN__C
00000001   xdc_runtime_Startup__RESETFXN__C
20026898   xdc_runtime_Startup_execImpl__C
2002197d   xdc_runtime_Startup_exec__E
20023e07   xdc_runtime_Startup_exec__I
20026618   xdc_runtime_Startup_firstFxns__A
20026658   xdc_runtime_Startup_firstFxns__C
20026660   xdc_runtime_Startup_lastFxns__C
2002689c   xdc_runtime_Startup_maxPasses__C
2001b313   xdc_runtime_Startup_reset__I
200265c4   xdc_runtime_Startup_sfxnRts__A
200268a0   xdc_runtime_Startup_sfxnRts__C
20026210   xdc_runtime_Startup_sfxnTab__A
200268a4   xdc_runtime_Startup_sfxnTab__C
2001dd75   xdc_runtime_Startup_startMods__I
20038cec   xdc_runtime_SysMin_Module_State_0_outbuf__A
2003b8c4   xdc_runtime_SysMin_Module__state__V
20023665   xdc_runtime_SysMin_Module_startup__E
20022d45   xdc_runtime_SysMin_abort__E
200268a8   xdc_runtime_SysMin_bufSize__C
20023831   xdc_runtime_SysMin_exit__E
20026908   xdc_runtime_SysMin_flushAtExit__C
200222d1   xdc_runtime_SysMin_flush__E
200268ac   xdc_runtime_SysMin_outputFunc__C
20023401   xdc_runtime_SysMin_output__I
20022885   xdc_runtime_SysMin_putch__E
20023f29   xdc_runtime_SysMin_ready__E
2002413b   xdc_runtime_System_Module_GateProxy_enter__E
2002413f   xdc_runtime_System_Module_GateProxy_leave__E
200240eb   xdc_runtime_System_Module_GateProxy_query__E
2003b8d0   xdc_runtime_System_Module_State_0_atexitHandlers__A
200268b0   xdc_runtime_System_Module__gateObj__C
2003b8e0   xdc_runtime_System_Module__state__V
200240cd   xdc_runtime_System_Module_startup__E
20022d45   xdc_runtime_System_SupportProxy_abort__E
20023831   xdc_runtime_System_SupportProxy_exit__E
200222d1   xdc_runtime_System_SupportProxy_flush__E
20022885   xdc_runtime_System_SupportProxy_putch__E
20023f29   xdc_runtime_System_SupportProxy_ready__E
200268b4   xdc_runtime_System_abortFxn__C
200220f9   xdc_runtime_System_abortStd__E
2002384d   xdc_runtime_System_abort__E
200239ef   xdc_runtime_System_aprintf__E
20024143   xdc_runtime_System_aprintf_va__F
200228bd   xdc_runtime_System_atexit__E
200230cd   xdc_runtime_System_avprintf__E
200184f9   xdc_runtime_System_doPrint__I
200268b8   xdc_runtime_System_exitFxn__C
20022101   xdc_runtime_System_exitStd__E
20023c35   xdc_runtime_System_exit__E
200268bc   xdc_runtime_System_extendFxn__C
200222d1   xdc_runtime_System_flush__E
2002139d   xdc_runtime_System_formatNum__I
200268c0   xdc_runtime_System_maxAtexitHandlers__C
2001da75   xdc_runtime_System_printfExtend__I
20023a09   xdc_runtime_System_printf__E
20024147   xdc_runtime_System_printf_va__F
20022d75   xdc_runtime_System_processAtExit__E
20022fb7   xdc_runtime_System_putchar__I
20023311   xdc_runtime_System_vprintf__E
20023f39   xdc_runtime_System_vsnprintf__E
2003b8e8   xdc_runtime_Text_Module__state__V
2002690a   xdc_runtime_Text_charCnt__C
2002414c   xdc_runtime_Text_charTab__A
200268c4   xdc_runtime_Text_charTab__C
20022f61   xdc_runtime_Text_cordText__E
2002690c   xdc_runtime_Text_isLoaded__C
200268c8   xdc_runtime_Text_nameEmpty__C
200268cc   xdc_runtime_Text_nameStatic__C
200268d0   xdc_runtime_Text_nameUnknown__C
20025c92   xdc_runtime_Text_nodeTab__A
200268d4   xdc_runtime_Text_nodeTab__C
20022acd   xdc_runtime_Text_printVisFxn__I
200215cd   xdc_runtime_Text_putLab__E
2001fbad   xdc_runtime_Text_putMod__E
2001f8bd   xdc_runtime_Text_putSite__E
2002690e   xdc_runtime_Text_registryModsLastId__C
20023c4d   xdc_runtime_Text_ropeText__E
20026910   xdc_runtime_Text_unnamedModsLastId__C
200219cd   xdc_runtime_Text_visitRope2__I
200268d8   xdc_runtime_Text_visitRopeFxn__C
20023f49   xdc_runtime_Text_visitRope__I
200226f5   xdc_runtime_Text_xprintf__I
200212dd   xdc_runtime_Timestamp_SupportProxy_get64__E
200212dd   xdc_runtime_Timestamp_get64__E


GLOBAL SYMBOLS: SORTED BY Symbol Address 

address    name
--------   ----
00000000   __ASM__
00000001   __TI_args_main
00000001   xdc_runtime_Startup__EXECFXN__C
00000001   xdc_runtime_Startup__RESETFXN__C
00000071   __ISA__
00000084   __PLAT__
000000ab   __TARG__
000000d0   __TRDR__
00002000   __STACK_SIZE
20004000   ti_sysbios_family_arm_m3_Hwi_resetVectors
2000494d   mqtt_client_new_msg_id
20004955   mqtt_client_is_connected
20004b0d   mqtt_client_send_progress
20004f4d   mqtt_connect_msg_send
2000509d   mqtt_client_pub_msg_send
2000512b   mqtt_client_pub_dispatch
2000535d   mqtt_sub_msg_send
20005373   mqtt_sub_dispatch
20005387   mqtt_unsub_msg_send
2000539d   mqtt_unsub_dispatch
2000545b   mqtt_pingreq_send
20005497   mqtt_disconn_send
20005f81   mqtt_client_ctx_await_msg
20005fd3   mqtt_client_ctx_run
2000628d   mqtt_client_await_msg
200062f5   mqtt_client_run
20006399   mqp_client_alloc
200063ed   mqtt_client_buffers_register
20006471   mqtt_client_ctx_will_register
200064f9   mqtt_client_ctx_info_register
20006579   mqtt_client_net_svc_register
20006675   mqtt_client_ctx_create
20006727   mqtt_client_ctx_delete
20006789   mqtt_client_lib_init
20006809   mqtt_client_lib_exit
20006b4d   MqttDevDataCB
200071d9   fnPtrDevCharListMqttPrint
20007299   MqttDeviceListCharPublish
2000735d   MqttDeviceGetPublish
20007435   MqttDeviceGetHandler
20007491   MqttDeviceSetHandler
20007559   MqttDeviceWhoamiPublish
2000759d   MqttDeviceHandler
20007615   MqttDeviceCtxClean
20007661   MqttDeviceCtxDel
20007707   MqttDeviceCtxAdd
20007b5d   MqttDevClean
20007e41   InitDevModeServer
20007ee9   MqttDevicePubsishQS
20007f41   is_anyDeviceMqttConnected
20007f81   mqttPublishData
20008015   cfgDevMqttMode
20008049   readDevMqttCfg
2000820b   MqttGwEventCB
20008339   MqttIpAcquiredPostMsg
2000838d   MqttTriggerScan
2000851d   MqttGwBuildTopics
20008659   MqttDevListPublish
2000868d   fnPtrMqttAdvBuild
20008759   fnPtrMqttConBuild
20008881   MqttDevConnectPublish
2000898b   MqttDevDisconnectPublish
20008a49   MqttBleFiHandler
20008b59   fnPtrMqttAddCon
20008b7b   MqttDeviceCtxInit
20008c25   MqttInitGwContext
20008da5   mqttCleanupCtx
20008fc5   MqttClient
20009185   MQTT_Init
200091c9   MqttBlefiMAC
200091cd   dummy_print
200091d5   getSizeofMqttCfg
200091d9   fillMqttDefaultCfg
20009249   ReadMQTTMode
200092f5   cfgGwMqttMode
2000932d   readGwMqttCfg
20009449   HTTP_EventCb
2000946f   HTTP_DataCb
200094f7   fnPtrHTTPscanlist
200095c7   fnPtrHTTPconnlist
20009695   fnPtrDevCharListHttpPRINT
2000971f   HttpGetTokenScan
20009991   HttpGetTokenConn
20009bed   HttpGetTokenGetChar
20009d73   HttpGetTokenOther
20009ff5   HttpGetToken
2000a1b5   HttpPostToken
2000a5e1   Http_Init
2000a609   DB_IsConnhandleValid
2000a617   set_devState
2000a62b   get_devState
2000a635   DB_DevRecInit
2000a707   DB_DevRecDeInit
2000a753   DB_deleteDevRec
2000a767   DB_FreePrimserv
2000a777   DB_GATT_DiscAllPrimaryServices
2000a7a3   DB_FreeCharDescsTable
2000a7eb   DB_FreeDbUuidInfo
2000a801   gw_createDeviceRec
2000a841   DB_SyncObjSignal
2000a865   DB_DevRecReady
2000a8d7   DB_DevRecDbInit
2000a8e9   DB_GATT_ReadUsingCharUuid
2000a955   DB_LinkDevRec
2000a95f   DB_Build
2000aa61   DB_BuildPrimServTable
2000ab1d   DB_PrintPrimServTable
2000abaf   DB_GATT_DiscAllChars
2000ac2f   DB_GATT_FindCharDescs
2000ace1   DB_DiscAllCharinService
2000ad2d   DB_BuildCharTable
2000ae45   DB_UpdateCharName
2000ae9f   DB_PrintCharTable
2000aeb5   DB_CharDescsTableInit
2000aef5   DB_CharDescsTableDeInit
2000af3b   DB_ParseString
2000afb5   DB_FindCharHandle
2000afff   DB_GetSetCharValue
2000b0b9   DB_GetSetChar
2000b0b9   GC_GetSet
2000b19d   DB_FillCurrentGetCharName
2000b1eb   DB_FindCharNameString
2000b259   DB_GATT_FindCharDescriptions
2000b30b   DB_GetCharDescription
2000b381   DB_BuildCharDescsTable
2000b429   DB_PrintCharDescsTable
2000b45d   DB_UpdateDeviceName
2000b48b   DB_getDevAddrPtr
2000b495   DB_getDevNamePtr
2000b49f   DB_GetDevCharList
2000b4cd   DB_IsConnIdValid
2000b4e9   DB_FlushSyncObjects
2000c15f   __TI_printfi
2000c469   CLI_EventCb
2000c4f1   CLI_DataCb
2000c5c5   DoScan
2000c5ed   DoDevList
2000c627   fnPtrCLIPRINT
2000c649   DoLinkEstablish
2000c695   DoLinkTerminate
2000c6d5   fnPtrDevCharListCLIPRINT
2000c711   DoListChar
2000c923   DoGet
2000cab5   DoSet
2000cb21   DoWlanconnect
2000cb77   DoWlanDisconnect
2000cb7b   DoCc26xxFwUpdate
2000cb8d   DoReset
2000cb97   DoAddOtaMeta
2000cbcd   triggerOta
2000cbdd   DoAutoScan
2000cc2d   DoMqttAddDev
2000cc47   DoMqttDelDev
2000ccaf   DomqttGwMode
2000cd2f   DomqttDevMode
2000cdaf   DoDefault
2000cdcb   fnPtrPairPRINT
2000cde1   DoPairList
2000ce67   DoUnPair
2000cf37   DoAutoconnect
2000d129   CliPuts
2000d1cb   uarta0IntFuncHandler
2000d1e9   CliGetcharOs
2000d399   print_usage
2000dc83   ClitaskFxn
2000dccb   CLI_Init
2000dda5   sbl_min
2000ddbf   sbl_get_bin_size
2000dde7   sbl_open_bin_for_read
2000de2b   sbl_close_bin
2000de43   sbl_read_bin
2000de67   generateCheckSum
2000deab   sendCmd
2000df2f   getCmdResponse
2000dfbd   sendAutoBaud
2000dff7   getResponseData
2000e0c3   sendCmdResponse
2000e117   readStatus
2000e19b   ulToCharArray
2000e1c5   eraseFlashRange
2000e349   calcCrcLikeChip
2000e439   writeFlashRange
2000e593   cmdDownload
2000e607   cmdSendData
2000e66d   addressInFlash
2000e67b   Do_SBL_Dnld
2000e76d   CC26xx_SBL_CheckIfUpdateFwNeeded
2000e9e1   itoa
2000ea93   SimpleLinkWlanEventHandler
2000ec87   SimpleLinkNetAppEventHandler
2000ed5b   SimpleLinkHttpServerCallback
2000ed8d   SimpleLinkGeneralEventHandler
2000edc5   SimpleLinkSockEventHandler
2000f139   ConnectToNetwork
2000f293   WlanDisconnectAP
2000f29b   WlanConnectAP
2000f377   NetworkInit
2000f3bd   SimpleLink_Init
2000f3f3   Wifi_GetMAC
2000f43f   IsSimpleLinkReady
2000f675   mqp_free
2000f6b5   mqp_reset
2000f6c1   mqp_init
2000f71b   mqp_buf_wr_utf8
2000f78d   mqp_buf_tail_wr_remlen
2000f7fd   mqp_buf_rd_remlen
2000f80d   mqp_pub_append_topic
2000f8bd   mqp_pub_append_data
2000f98d   mqp_proc_vh_msg_id_rx
2000f999   mqp_proc_msg_id_ack_rx
2000f9cf   mqp_proc_pub_rx
2000fa71   mqp_ack_wlist_append
2000faa7   mqp_ack_wlist_remove
2000fb17   mqp_ack_wlist_purge
2000fb49   secure_conn_struct_init
2000fb69   mqp_prep_fh
2000fbdf   mqp_recv
2000fd5f   qos2_pub_cq_reset
2000fd81   qos2_pub_cq_logup
2000fdbf   qos2_pub_cq_unlog
2000fe03   qos2_pub_cq_check
2000fe73   cl_ctx_reset
2000fea3   cl_ctx_timeout_insert
2000ff13   cl_ctx_remove
2000ff69   cl_ctx_timeout_update
2001014b   VMqttRecvTask
200101e5   sl_ExtLib_MqttClientCtxCreate
20010303   sl_ExtLib_MqttClientCtxDelete
2001033d   mutex_lockup
2001034d   mutex_unlock
2001035d   sl_ExtLib_MqttClientInit
20010425   sl_ExtLib_MqttClientExit
20010479   sl_ExtLib_MqttClientSet
200104d5   sl_ExtLib_MqttClientConnect
20010635   sl_ExtLib_MqttClientDisconnect
200106a1   sl_ExtLib_MqttClientSub
20010789   sl_ExtLib_MqttClientUnsub
20010855   sl_ExtLib_MqttClientSend
20010939   GAPBondMgr_SetParam
20010a53   GAPBondMgr_GetParam
20010aff   GAPBondMgr_ResolveAddr
20010b75   GAPBondMgr_LinkEst
20010c5d   GAPBondMgr_LinkTerm
20010c79   GAPBondMgr_SlaveReqSecurity
20010ce5   GAPBondMgr_PasscodeRsp
20010dbb   gapBondMgrFindEmpty
20010df7   gapBondMgrFindBondEntry
20010e99   gapBondMgrAddBond
20010f01   gapBondMgrEraseAllBondings
2001109d   getSizeofBondCfg
200110a3   fillBondDefaultCfg
200110b1   GC_PairDevList
200110e1   GC_UnPair
20011131   FlashWriteFile
2001120f   FlashReadFile
2001131b   FlashIsFilePresent
2001134f   TurnOnLed
2001138b   TurnOffLed
2001144d   BlinkLed
200114f1   Button2Init
20011531   Button2IntClear
20011543   Button2IntDisable
200115a3   Button2IntEnable
2001160f   HandleError
200116dd   sblUARTinit
200116fb   CC26xx_SBL_Dnld_Init
20011863   ti_sysbios_BIOS_nullFunc__I
20011865   Schema_init
20011879   Schema_FindProfile
2001190d   Schema_loadfile
2001195d   ReadFileFromDevice
200119d9   Schema_FindCharString
20011a6d   Schema_FindString
20011a75   Schema_DelProfile
20011ab7   ParseJSONData
20011ccf   sch_char_to_hex
20011cdf   sch_copy_serv_uuid
20011dbd   sch_copy_char_uuid
20011ea5   sch_copy_charstring
20012189   comm_open
2001229b   tcp_send
200122c1   tcp_recv
20012321   comm_close
20012333   rtc_secs
2001233b   tcp_listen
200123c7   tcp_select
200124a3   tcp_accept
20012511   send_dest
20012591   recv_from
20012631   CopyDeviceName
20012685   GatewayCentral_processRoleEvent
200129c9   GatewayCentral_processGattEvent
20012c75   printScanResponse
20012cbd   sl_Recv_eagain
20012ce5   json_parse_update_check_resp
20012e07   json_parse_rsrc_metadata_url
20012e41   json_parse_dropbox_metadata
20012f89   json_parse_dropbox_media_url
20012feb   http_skip_headers
200130b5   http_send_buf
200130b9   http_recv_buf
200130bd   http_extract_domain_by_url
20013127   http_connect_server
20013205   http_build_request
200132cd   NPI_Init
200132db   Gateway_Init
200134bf   get_gwState
200134c5   set_gwState
200134e9   set_gwCallType
2001352d   get_gwCallType
20013565   get_gwDevCnt
2001356d   get_gw_devState
2001357b   get_gw_devConnectionid
20013595   GatewayCentral_RegisterGC_CB
200135d1   gwcontext_Init
200135ff   gwcontext_IsScanIdValid
2001365d   RegisterGwCB
20013695   CallGwEventCB
2001371b   CallGwDataCB
20013791   GC_StackEventHandler_CB
200137df   Util_convertBdAddr2Str
2001382d   SBL_IsDone
20013b7d   jsmn_parse
20013e8f   jsmn_init
20013ead   _SlDrvMsgRead
20014499   getGenericTaskTicksPerSec
2001449d   doPeriodicScan
2001451f   fillDefaultCfgVal
200145a5   GwGenericTask
200145eb   GW_GenericTask_Init
20014621   KickGenericTask
200147f9   LoadBleFiCfg
2001483b   writeBleCfg
200148e1   UpdateBlefiCfg
200148e1   gapBondMgrFlashBondRecUpdate
200148ef   GwButtonHandler
2001490f   Gateway_ButtonInit
20014917   configureAutoScan
20014961   readAutoScan
2001497d   enforceCC26XXFwChecsum
20014995   doHandleCmdtimeout
200149a5   disableAutoconnect
200149bb   enableAutoconnect
20014a69   IfBondingEnabled
20014adb   GC_Scan
20014b69   GC_DeviceScanList
20014b97   GC_DeviceConnList
20014bbb   GC_DeviceScanListBdAddr
20014bc5   GC_LinkEstablish
20014cad   GC_LinkTerminate
20014d39   GC_GATT_DiscAllPrimaryServices
20014d79   GC_GATT_DiscPrimaryServiceByUUID
20014e4b   GC_GATT_DiscAllChars
20014e8d   GC_GetDevCharList
20014e97   GC_EraseAllBondings
20014e9b   GC_IsBLEReady
20015035   RebootMCU
2001506d   OtaAddOtaMeta
200150ab   OTAServerInfoSet
2001518f   OtaUpdateLoop
2001527b   OtaCommit
200152b9   OTAUpdateTask
20015387   OtaButtonHandler
20015409   OtaButtonInit
20015485   OTA_Init
200154c7   otaSignalWLANConnect
200154d7   OtaDownload
200154e9   getSizeofOtaMeta
200154ed   fillOtaMetaDefaultCfg
2001560b   GAP_deviceInitPacketize
20015697   GAP_configDeviceAddrPacketize
200156d9   GAP_deviceDiscoveryRequestPacketize
200156ff   GAP_deviceDiscoveryCancelPacketize
20015717   GAP_makeDiscoverablePacketize
2001576b   GAP_updateAdvertisingDataPacketize
200157b7   GAP_endDiscoverablePacketize
200157cf   GAP_establishLinkRequestPacketize
20015817   GAP_terminateLinkRequestPackeize
2001583d   GAP_authenticatePacketize
2001592d   GAP_updateLinkParamterRequestPacketize
20015977   GAP_BondPacketize
200159ff   GAP_TerminateAuthPacketize
20015a25   GAP_SignablePacketize
20015a93   GAP_PasskeyUpdatePacketize
20015a95   GAP_setParameterPacketize
20015abd   GAP_getParameterPacketize
20015ad9   GAP_ResolvePrivateAddrPacketize
20015b2b   GAP_SendSlaveSecurityRequestPacketize
20015b2d   GAPBondMgr_setParameterPacketize
20015b83   GAPBondMgr_getParameterPacketize
20015beb   osi_InterruptRegister
20015c43   osi_InterruptDeRegister
20015c5f   osi_SyncObjCreate
20015ca7   osi_SyncObjDelete
20015cb5   osi_SyncObjSignal
20015cc5   osi_SyncObjSignalFromISR
20015cd5   osi_SyncObjWait
20015d2d   osi_SyncObjClear
20015d45   osi_LockObjCreate
20015d87   osi_TaskCreate
20015de1   osi_TaskDelete
20015ded   osi_LockObjDelete
20015dfb   osi_LockObjLock
20015e53   osi_LockObjUnlock
20015e63   osi_Spawn
20015eb9   VStartSimpleLinkSpawnTask
20015f13   VDeleteSimpleLinkSpawnTask
20015f23   mem_Malloc
20015f2f   mem_Free
20015f3b   mem_set
20015f4f   mem_copy
20015f63   osi_EnterCritical
20015f75   osi_ExitCritical
20015f81   osi_MsgQCreate
20015fb7   osi_MsgQDelete
20015fc5   osi_MsgQWrite
2001602b   osi_MsgQRead
2001608d   osi_Sleep
200160ad   osi_TaskDisable
200160b5   osi_TaskEnable
200160c1   osi_start
200160c9   osi_ContextSave
200160cb   osi_ContextRestore
200160ed   pow
20016121   collectCC26XXSensorData
2001628f   publishCC26XXSensorData
20016371   sensorTagEnableNoti
200165e5   GATT_InitClient
200165e9   GATT_RegisterForInd
200165eb   GATT_PrepareWriteReq
200165ef   GATT_ExecuteWriteReq
200165f3   GATT_InitServer
200165f7   GATT_RegisterService
200165fb   GATT_DeregisterService
200165ff   GATT_RegisterForReq
20016601   GATT_VerifyReadPermissions
20016605   GATT_VerifyWritePermissions
20016609   GATT_ServiceChangedInd
2001660d   GATT_FindHandleUUID
20016611   GATT_FindHandle
20016615   GATT_FindNextAttr
20016619   GATT_ServiceNumAttrs
2001661d   GATT_Indication
20016683   GATT_Notification
200166eb   GATT_ExchangeMTU
200166ef   GATT_DiscAllPrimaryServices
20016721   GATT_DiscPrimaryServiceByUUID
2001677b   GATT_FindIncludedServices
200167b9   GATT_DiscAllChars
200167f7   GATT_DiscCharsByUUID
20016865   GATT_DiscAllCharDescs
200168a3   GATT_ReadCharValue
200168dd   GATT_ReadUsingCharUUID
2001694b   GATT_ReadLongCharValue
2001694f   GATT_ReadMultiCharValues
20016953   GATT_WriteNoRsp
200169c5   GATT_SignedWriteNoRsp
200169c9   GATT_WriteCharValue
20016a2f   GATT_WriteLongCharValue
20016a33   GATT_ReliableWrites
20016a37   GATT_ReadCharDesc
20016a3b   GATT_ReadLongCharDesc
20016a3f   GATT_WriteCharDesc
20016a43   GATT_WriteLongCharDesc
20016a47   GATT_SetHostToAppFlowCtrl
20016a49   GATT_AppCompletedMsg
20016a4b   GATT_SetNextHandle
20016a4d   GATT_Init
20016a4f   GATT_ProcessEvent
20016a59   GAP_DeviceInit
20016aab   GAP_ConfigDeviceAddr
20016aed   GAP_EstablishLinkReq
20016b09   GAP_UpdateLinkParamReq
20016b25   GAP_TerminateLinkReq
20016b61   GAP_DeviceDiscoveryRequest
20016b7d   GAP_DeviceDiscoveryCancel
20016b93   GAP_Authenticate
20016bcf   GAP_TerminateAuth
20016c0b   GAP_Bond
20016c53   GAP_Signable
20016c8f   GAP_PasskeyUpdate
20016ccb   GAP_SetParamValue
20016d03   GAP_GetParamValue
20016d2f   GAP_ResolvePrivateAddr
20016d65   GAP_SendSlaveSecurityRequest
20016d9b   GAPBondMgr_SetParameter
20016dff   GAPBondMgr_GetParameter
20016e31   GAP_deviceInitDone
20016e41   GAP_advertDataUpdateDone
20016e51   GAP_makeDiscoverableDone
20016e61   GAP_linkEstablished
20016e71   GAP_linkTerminated
20016e81   OtaClient_UpdateCheck
20016f2f   OtaClient_ResourceNameConvert
200170f3   OtaClient_ResourceMetadata
200171c9   OtaClient_Init
200171fb   OtaClient_GetNextUpdate
2001722d   OtaClient_ConnectServer
20017263   OtaClient_CloseServer
200172a5   ti_sysbios_family_arm_m3_Hwi_excDumpRegs__I
200176c9   _OtaCleanToIdle
200176e7   sl_extLib_OtaSet
20017769   _WriteStatFile
200177b3   local_filter
200177b7   _ReadStatFile
200177f9   sl_extLib_OtaRun
20017a03   sl_extLib_OtaInit
20017a6b   sl_extLib_OtaGet
20017b1b   NPI_UartEventTaskFxn
20017cd5   NPI_UartEventCreateTask
20017d07   UartWritePacket
20017e45   _readSignature
20017ea1   _RecvFileChunk
20017ead   _ReadFileHeaders
20017efb   _OpenStorageFile
20017f59   CdnClient_SetFileInfo
20017f63   CdnClient_Run
20018099   CdnClient_Init
200180cb   CdnClient_CloseServer
200180e9   CdnClient_ConnectByUrl
200181a1   InitTerm
200181eb   Message
20018217   ClearTerm
20018221   Error
2001825f   GetCmd
20018353   TrimSpace
20018427   Report
200184f7   ti_sysbios_gates_GateHwi_Instance_init__E
200184f9   xdc_runtime_System_doPrint__I
20018835   LogClient_Print
20018979   LogClient_Init
20018991   LogClient_ConnectServer
200189c7   LogClient_Close
200189df   LogClient_ConnectAndPrint
20018b6d   NPI_TaskCreate
20018b7d   NPI_CreateSyncObj
20018b81   NPI_SyncObjWait
20018b85   NPI_SyncObjSignal
20018b89   NPI_SyncObjSignalFromISR
20018b8d   NPI_Sleep
20018b91   NPI_SpiInit
20018beb   NPI_RegisterGpioInterrupt
20018c23   NPI_EnableGPIOInt
20018c3b   NPI_DisableGpioInt
20018c5d   NPI_GpioPinWrite
20018c6d   NPI_GpioPinRead
20018c81   NPI_SpiReadPacket
20018cc3   NPI_SpiWritePacket
20018db5   NPI_UartInit
20018e09   NPI_UartReadPacket
20018e23   NPI_UartWritePacket
20018e3d   NPI_UartDisableInt
20018e45   NPI_UartEnableInt
20018e4d   NPI_IsReady
20018e99   ti_sysbios_knl_Semaphore_pend__E
2001919d   HOSTwrite
200191e9   HOSTunlink
20019221   HOSTtime
2001925b   HOSTrename
200192b9   HOSTread
20019305   HOSTopen
20019357   HOSTlseek
200193b3   HOSTgetenv
200193f1   HOSTclose
20019429   HOSTclock
20019471   sl_WlanProfileAdd
200196e1   _SlDrvRxHdrRead
20019929   ti_sysbios_heaps_HeapMem_free__E
20019b71   sl_WlanConnect
20019db5   ti_sysbios_heaps_HeapMem_alloc__E
20019fe9   ti_sysbios_knl_Task_Instance_finalize__E
2001a211   process_Scan
2001a243   process_ScanStop
2001a251   process_LinkEstablish
2001a287   process_LinkTerminate
2001a2a7   process_GattDiscAllPrimaryServices
2001a2b3   process_GattDiscAllChars
2001a2c3   process_GATTFindCharDescs
2001a2d3   process_ReadHandle
2001a2e1   process_WriteHandle
2001a31f   process_GattReadUsingCharUuid
2001a34d   GatewayCentral_handleinput
2001a431   ti_sysbios_knl_Task_sleep__E
2001a639   ti_sysbios_family_arm_m3_Hwi_excHandlerMax__I
2001a831   __aeabi_uldivmod
2001aa25   GAPCentralRole_StartDevice
2001aa53   GAPCentralRole_SetParameter
2001aaaf   GAPCentralRole_GetParameter
2001ab03   GAPCentralRole_TerminateLink
2001ab11   GAPCentralRole_EstablishLink
2001ab33   GAPCentralRole_UpdateLink
2001ab57   GAPCentralRole_StartDiscovery
2001ab6d   GAPCentralRole_CancelDiscovery
2001ab75   WaitForEvent
2001ac05   _SlDrvReleasePoolObj
2001add5   _SlDrvMsgWrite
2001afa1   ti_sysbios_knl_Task_Instance_init__E
2001b15d   __aeabi_dsub
2001b167   __aeabi_dadd
2001b313   xdc_runtime_Startup_reset__I
2001b315   _SlDrvWaitForPoolObj
2001b4a5   ti_sysbios_knl_Task_Module_startup__E
2001b631   sl_extlib_FlcWriteFile
2001b68f   sl_extlib_FlcTest
2001b6bd   sl_extlib_FlcReadFile
2001b6cf   sl_extlib_FlcOpenFile
2001b711   sl_extlib_FlcIsPendingCommit
2001b729   sl_extlib_FlcCommit
2001b761   sl_extlib_FlcCloseFile
2001b769   sl_extlib_FlcAbortFile
2001b7b5   BlefiVersion
2001b7b9   CC26xx_Init
2001b80d   BlefiDisplayBanner
2001b83b   Blefi_HW_Init
2001b863   main
2001b939   _SlDrvDriverCBInit
2001baad   _SlFindAndSetActiveObj
2001bc1d   ti_sysbios_family_arm_m3_Hwi_excBusFault__I
2001bd85   ti_sysbios_knl_Mailbox_Instance_init__E
2001bee5   ti_sysbios_family_arm_m3_Hwi_excUsageFault__I
2001c039   spi_Open
2001c189   ti_sysbios_family_arm_m3_Hwi_excMemFault__I
2001c2c9   sl_Select
2001c405   ti_sysbios_family_arm_m3_Hwi_dispatchC__I
2001c541   sl_Accept
2001c679   ti_sysbios_heaps_HeapMem_Instance_init__E
2001c7b1   ti_sysbios_knl_Semaphore_post__E
2001c8e9   __aeabi_ddiv
2001ca21   PRCMCC3200MCUInit
2001cb55   xdc_runtime_LoggerBuf_write8__E
2001cc85   ti_sysbios_knl_Clock_workFunc__E
2001cdb1   _SlDrvDataReadOp
2001ced9   ti_sysbios_knl_Swi_run__I
2001cff9   xdc_runtime_Error_policyDefault__E
2001d119   sl_SendTo
2001d231   strtoul
2001d341   UARTPinMuxConfig
2001d375   GPIOLedButtonPinMuxConfig
2001d3f9   GPIOSBLPinMuxConfig
2001d43d   PinMuxConfig
2001d44d   sl_RecvFrom
2001d559   sl_Connect
2001d661   sl_Send
2001d769   _SlDrvDataWriteOp
2001d86d   sl_NetAppDnsGetHostByName
2001d971   xdc_runtime_Core_createObject__I
2001da75   xdc_runtime_System_printfExtend__I
2001db79   _SlDrvNetAppEventHandler
2001dc77   __aeabi_dmul
2001dd75   xdc_runtime_Startup_startMods__I
2001de71   sl_FsRead
2001df65   uDMAChannelTransferSet
2001e055   sl_FsWrite
2001e141   spi_Read
2001e21d   _SlDrvClassifyRxMsg
2001e2f5   xdc_runtime_LoggerBuf_write4__E
2001e3c9   SmartConfigConnect
2001e43f   SmartConfigStop
2001e49d   ti_sysbios_family_arm_m3_Hwi_dispatch__I
2001e56d   xdc_runtime_Core_constructObject__I
2001e639   _sl_HandleAsync_DnsGetHostByService
2001e701   ti_sysbios_knl_Task_schedule__I
2001e7c9   ti_sysbios_family_arm_m3_Hwi_Module_startup__E
2001e88d   _SlRemoveFromList
2001e94d   ti_sysbios_knl_Task_exit__E
2001ea0d   _SlDrvMsgReadCmdCtx
2001eac9   sl_Start
2001eb85   ti_sysbios_knl_Task_startCore__E
2001ec41   _SlAsyncEventGenericHandler
2001ecf9   ti_sysbios_family_arm_m3_Hwi_excHardFault__I
2001edad   ti_sysbios_gates_GateMutex_enter__E
2001ee61   ti_sysbios_knl_Task_checkStacks__E
2001ef15   NPI_RegisterTask
2001ef1b   BLEAPI_decodeIncomingPacket
2001ef53   BLEAPI_checkReceivedEvent
2001ef73   BLEAPI_waitForSpecficEvent
2001efc5   ti_sysbios_family_arm_m3_Hwi_excDebugMon__I
2001f075   IntDisable
2001f11d   IntEnable
2001f1c5   sl_NetCfgGet
2001f26d   ti_sysbios_knl_Swi_post__E
2001f315   ti_sysbios_knl_Task_blockI__E
2001f3bd   ti_sysbios_knl_Task_postInit__I
2001f465   ti_sysbios_knl_Task_yield__E
2001f50d   SPIConfigSetExpClk
2001f5ad   __TI_auto_init
2001f64d   _SlDrvMsgReadSpawnCtx
2001f6e9   __aeabi_memcpy
2001f6e9   __aeabi_memcpy4
2001f6e9   __aeabi_memcpy8
2001f6e9   memcpy
2001f785   ti_sysbios_family_arm_m3_Hwi_Instance_init__E
2001f821   ti_sysbios_knl_Semaphore_Instance_init__E
2001f8bd   xdc_runtime_Text_putSite__E
2001f959   _sl_GetCreateFsMode
2001f9f1   PRCMPeripheralClockGet
2001fa85   ti_sysbios_knl_Mailbox_post__E
2001fb19   ti_sysbios_knl_Task_unblockI__E
2001fbad   xdc_runtime_Text_putMod__E
2001fc41   sl_WlanSmartConfigStart
2001fde9   _sl_HandleAsync_DnsGetHostByName
2001fe75   _sl_HandleAsync_PingResponse
2001ff01   spi_Write
2001ff8d   PRCMHibernateIntervalSet
20020015   PinConfigSet
2002009d   vsnprintf
20020125   sl_Bind
200201ad   sl_FsClose
20020235   ti_sysbios_knl_Mailbox_Module_startup__E
200202bd   __aeabi_cdcmpeq
200202bd   __aeabi_cdcmple
20020343   __aeabi_cdrcmple
200203c9   NwpPowerOnPreamble
2002044d   ti_sysbios_family_arm_m3_Hwi_initNVIC__E
200204d1   ti_sysbios_knl_Mailbox_pend__E
20020555   GPIOIntTypeSet
200205d9   _SlDrvCmdOp
20020759   xdc_runtime_LoggerBuf_setFilterLevel__E
200207d9   PRCMRTCGet
20020855   _sl_HandleAsync_InitComplete
200208d1   sl_FsGetInfo
2002094d   _sl_HandleAsync_Connect
200209c5   __aeabi_memclr
200209c5   __aeabi_memclr4
200209c5   __aeabi_memclr8
200209c7   __aeabi_memset
200209c7   __aeabi_memset4
200209c7   __aeabi_memset8
200209cd   memset
20020a3d   sl_FsOpen
20020ab5   UARTConfigSetExpClk
20020b2d   sl_Recv
20020ba1   ti_sysbios_family_arm_m3_Hwi_postInit__I
20020c11   ti_sysbios_knl_Mailbox_Instance_finalize__E
20020c81   xdc_runtime_Memory_alloc__E
20020cf1   _SlDrvCmdSend
20020d5d   xdc_runtime_Error_print__E
20020dc9   xdc_runtime_LoggerBuf_getFilterLevel__E
20020e35   _sl_NetAppSendTokenValue
20020e9d   sl_SetSockOpt
20020f05   xdc_runtime_Core_deleteObject__I
20020f6d   ti_sysbios_family_arm_m3_Hwi_create
20020fd1   ti_sysbios_knl_Mailbox_create
20021035   uDMAChannelAttributeDisable
20021099   uDMAChannelAttributeEnable
200210fd   _sl_HandleAsync_Accept
2002115d   HCI_commandStatus
20021181   HCI_decodeHeader
200211bd   sprintf
2002121d   __TI_writemsg
20021247   C$$IO$$
2002124b   __TI_readmsg
2002127d   sl_WlanPolicySet
200212dd   ti_sysbios_family_arm_m3_TimestampProvider_get64__E
200212dd   xdc_runtime_LoggerBuf_TimestampProxy_get64__E
200212dd   xdc_runtime_Timestamp_SupportProxy_get64__E
200212dd   xdc_runtime_Timestamp_get64__E
2002133d   ti_sysbios_knl_Clock_logTick__E
2002139d   xdc_runtime_System_formatNum__I
2002145d   sl_Socket
200214b9   ti_sysbios_family_arm_m3_Timer_setPeriod__E
20021515   ti_sysbios_knl_Task_create
20021571   xdc_runtime_LoggerBuf_Object__create__S
200215cd   xdc_runtime_Text_putLab__E
20021629   ltoa
20021685   IntPendClear
200216dd   PRCMPeripheralReset
20021735   ti_sysbios_knl_Swi_restoreHwi__E
2002178d   ti_sysbios_knl_Swi_schedule__I
200217e5   _sl_HandleAsync_Select
20021839   ti_sysbios_family_arm_m3_Timer_start__E
2002188d   PRCMSlowClkCtrGet
200218dd   _sl_HandleAsync_Stop
2002192d   sl_FsDel
2002197d   xdc_runtime_Startup_exec__E
200219cd   xdc_runtime_Text_visitRope2__I
20021a1d   SPIIntEnable
20021a69   _SlDrvProtectAsyncRespSetting
20021ab5   _SlDrvRxIrqHandler
20021b01   _sl_BuildAddress
20021b4d   atoi
20021b99   atol
20021be5   ti_sysbios_family_arm_m3_TaskSupport_buildTaskStack
20021c31   ti_sysbios_knl_Swi_runLoop__I
20021c7d   uDMAChannelAssign
20021cc9   atod
20021cdd   atolong
20021d15   PRCMHibernateWakeupSourceEnable
20021d5d   SPIIntClear
20021da5   _SlDrvBasicCmd
20021ded   __aeabi_d2iz
20021e35   ti_sysbios_family_arm_m3_Hwi_excReserved__I
20021e7d   ti_sysbios_family_arm_m3_Hwi_initStacks__E
20021ec5   ti_sysbios_family_arm_m3_Timer_initDevice__I
20021f0d   ti_sysbios_heaps_HeapMem_getStats__E
20021f55   xdc_runtime_Assert_raise__I
20021f9d   xdc_runtime_Core_assignParams__I
20022029   _c_int00
200220b1   copy_in
200220f5   C$$EXIT
200220f9   abort
200220f9   xdc_runtime_System_abortStd__E
20022101   exit
20022101   xdc_runtime_System_exitStd__E
20022139   _Dtest
2002217d   ti_sysbios_family_arm_m3_Hwi_disableInterrupt__E
2002217d   ti_sysbios_hal_Hwi_HwiProxy_disableInterrupt__E
2002217d   ti_sysbios_hal_Hwi_disableInterrupt__E
200221c1   ti_sysbios_family_arm_m3_Hwi_enableInterrupt__E
200221c1   ti_sysbios_hal_Hwi_HwiProxy_enableInterrupt__E
200221c1   ti_sysbios_hal_Hwi_enableInterrupt__E
20022205   ti_sysbios_knl_Task_allBlockedFunction__I
20022249   xdc_runtime_Error_setX__E
2002228d   xdc_runtime_LoggerBuf_filterOutEvent__I
200222d1   xdc_runtime_SysMin_flush__E
200222d1   xdc_runtime_System_SupportProxy_flush__E
200222d1   xdc_runtime_System_flush__E
20022315   __aeabi_uidivmod
20022357   sl_Htonl
20022399   PinModeSet
200223d9   strtok
20022419   ti_sysbios_family_arm_m3_Timer_Module_startup__E
20022459   ti_sysbios_knl_Mailbox_postInit__I
20022499   realloc
200224d7   CopyPingResultsToReport
20022515   PRCMPeripheralClkEnable
20022551   _sl_TruncatePayloadByProtocol
2002258d   sl_Htons
200225c9   sl_Listen
20022605   ti_sysbios_family_arm_m3_Hwi_excSvCall__I
20022641   ti_sysbios_heaps_HeapMem_init__I
2002267d   ti_sysbios_knl_Swi_startup__E
200226b9   uDMAChannelControlSet
200226f5   xdc_runtime_Text_xprintf__I
20022731   xdc_runtime_LoggerBuf_Instance_init__E
2002276d   NwpPowerOff
200227a5   ti_sysbios_family_arm_m3_Hwi_excNoIsr__I
200227dd   ti_sysbios_family_arm_m3_Hwi_getStackInfo__E
200227dd   ti_sysbios_hal_Hwi_HwiProxy_getStackInfo__E
200227dd   ti_sysbios_hal_Hwi_getStackInfo__E
20022815   ti_sysbios_family_arm_m3_TaskSupport_start__E
20022815   ti_sysbios_knl_Task_SupportProxy_start__E
2002284d   ti_sysbios_knl_Task_processVitalTaskFlag__I
20022885   xdc_runtime_SysMin_putch__E
20022885   xdc_runtime_System_SupportProxy_putch__E
200228bd   xdc_runtime_System_atexit__E
200228f5   GPIODirModeSet
2002292d   PRCMPeripheralStatusGet
20022961   SPIFIFOLevelSet
20022995   strstr
200229c9   ti_sysbios_family_arm_m3_Hwi_excNmi__I
200229fd   ti_sysbios_family_arm_m3_Timer_periodicStub__I
20022a31   ti_sysbios_hal_Hwi_checkStack
20022a65   ti_sysbios_knl_Semaphore_create
20022a99   xdc_runtime_Core_assignLabel__I
20022acd   xdc_runtime_Text_printVisFxn__I
20022b01   ti_sysbios_knl_Semaphore_pendTimeout__I
20022b33   PinTypeGPIO
20022b65   UARTDisable
20022b95   _SlDrvDeviceEventHandler
20022bc5   _sl_Strlen
20022bf5   strncpy
20022c25   sl_Close
20022c55   ti_sysbios_BIOS_atExitFunc__I
20022c85   ti_sysbios_gates_GateHwi_Object__create__S
20022cb5   ti_sysbios_gates_GateMutex_Object__create__S
20022ce5   ti_sysbios_heaps_HeapMem_Object__create__S
20022d15   ti_sysbios_knl_Semaphore_construct
20022d45   xdc_runtime_SysMin_abort__E
20022d45   xdc_runtime_System_SupportProxy_abort__E
20022d75   xdc_runtime_System_processAtExit__E
20022da5   malloc
20022dd3   __aeabi_i2d
20022e01   DmaSpiSwIntHandler
20022e2d   NwpPowerOn
20022e59   PRCMSysResetCauseGet
20022e85   ti_sysbios_family_arm_m3_Hwi_Instance_finalize__E
20022eb1   ti_sysbios_hal_Hwi_initStack
20022edd   ti_sysbios_knl_Clock_doTick__I
20022f09   ti_sysbios_knl_Queue_construct
20022f35   ti_sysbios_knl_Task_restore__E
20022f61   xdc_runtime_Text_cordText__E
20022f8d   strspn
20022fb7   xdc_runtime_System_putchar__I
20023009   PRCMPeripheralClkDisable
20023031   SL_FD_ISSET
20023059   xdc_runtime_LoggerBuf_Module_startup__E
20023081   NwpRegisterInterruptHandler
200230a7   strncmp
200230cd   xdc_runtime_System_avprintf__E
2002313d   UARTEnable
20023161   _SlDrvProtectionObjLockWaitForever
20023185   memmove
200231a9   ti_sysbios_BIOS_errorRaiseHook__I
200231cd   ti_sysbios_BIOS_registerRTSLock__I
200231f1   ti_sysbios_BIOS_removeRTSLock__I
20023215   ti_sysbios_BIOS_startFunc__I
20023239   ti_sysbios_family_arm_m3_Hwi_doTaskRestore__I
2002325d   ti_sysbios_family_arm_m3_Timer_startup__E
2002325d   ti_sysbios_hal_Timer_TimerProxy_startup__E
2002325d   ti_sysbios_hal_Timer_startup__E
2002325d   ti_sysbios_knl_Clock_TimerProxy_startup__E
20023281   ti_sysbios_gates_GateMutex_Object__delete__S
200232a5   ti_sysbios_knl_Clock_Module_startup__E
200232c9   ti_sysbios_knl_Semaphore_Object__delete__S
200232ed   ti_sysbios_knl_Swi_Module_startup__E
20023311   xdc_runtime_System_vprintf__E
20023335   GPIOIntStatus
20023357   SL_FD_SET
20023379   SPIReset
2002339b   SPIWordCountSet
200233bd   memcmp
200233df   strcspn
20023401   xdc_runtime_SysMin_output__I
20023423   GPIOPinWrite
20023443   SPIDataGet
20023465   _SlDrvProtectionObjUnLock
20023485   platform_timer_init
2002348d   platform_get_time_in_secs
200234a5   ti_sysbios_family_arm_m3_Hwi_Object__delete__S
200234c5   ti_sysbios_family_arm_m3_Hwi_excHandlerAsm__I
200234e5   ti_sysbios_family_arm_m3_Hwi_excHandler__I
20023505   ti_sysbios_family_arm_m3_TimestampProvider_Module_startup__E
20023525   ti_sysbios_gates_GateHwi_Object__delete__S
20023545   ti_sysbios_heaps_HeapMem_Object__delete__S
20023565   ti_sysbios_knl_Idle_run__E
20023585   ti_sysbios_knl_Mailbox_Object__delete__S
200235a5   ti_sysbios_knl_Semaphore_Object__destruct__S
200235c5   ti_sysbios_knl_Task_Object__delete__S
200235e5   ti_sysbios_knl_Task_enter__I
20023605   xdc_runtime_LoggerBuf_Object__delete__S
20023625   xdc_runtime_LoggerBuf_reset__E
20023645   xdc_runtime_Registry_findById__E
20023665   xdc_runtime_SysMin_Module_startup__E
20023685   SPIDataPut
200236a3   UARTCharPut
200236df   ti_sysbios_family_xxx_Hwi_switchAndRunFunc
200236fd   UARTCharGetNonBlocking
20023719   _SlDrvObjLockWaitForever
20023735   _SlDrvSyncObjWaitForever
20023751   memccpy
2002376d   ti_sysbios_BIOS_rtsLock__I
20023789   ti_sysbios_family_arm_m3_Hwi_setPriority__E
200237a5   ti_sysbios_gates_GateMutex_Instance_init__E
200237c1   ti_sysbios_knl_Queue_Object__destruct__S
200237dd   uDMAChannelEnable
200237f9   xdc_runtime_Error_raiseX__E
20023815   xdc_runtime_Memory_valloc__E
20023831   xdc_runtime_SysMin_exit__E
20023831   xdc_runtime_System_SupportProxy_exit__E
2002384d   xdc_runtime_System_abort__E
20023869   GPIOIntDisable
20023883   GPIOIntEnable
2002389d   PinTypeUART
200238b7   SPIDmaEnable
200238d1   SPIFIFOEnable
200238eb   strcat
20023905   ti_sysbios_family_arm_m3_Hwi_Handle__label__S
2002391f   ti_sysbios_family_arm_m3_Hwi_pendSV__I
20023937   ti_sysbios_family_arm_m3_Hwi_return
20023939   ti_sysbios_gates_GateHwi_Handle__label__S
20023953   ti_sysbios_gates_GateMutex_Handle__label__S
2002396d   ti_sysbios_heaps_HeapMem_Handle__label__S
20023987   ti_sysbios_knl_Swi_Handle__label__S
200239a1   ti_sysbios_knl_Task_Handle__label__S
200239bb   ti_sysbios_knl_Task_sleepTimeout__I
200239d5   xdc_runtime_LoggerBuf_Handle__label__S
200239ef   xdc_runtime_System_aprintf__E
20023a09   xdc_runtime_System_printf__E
20023a23   GPIOPinRead
20023a3d   PRCMHibernateEnter
20023a55   SPICSDisable
20023a6d   SPICSEnable
20023a85   SPIDisable
20023a9d   SPIEnable
20023ab5   UARTCharsAvail
20023acd   UARTFIFOLevelSet
20023ae5   UARTIntDisable
20023afd   UARTIntEnable
20023b15   _SlDrvObjUnLock
20023b2d   _SlDrvSyncObjSignal
20023b45   _sl_GetStartResponseConvert
20023b5d   free
20023b75   _args_main
20023b8d   __aeabi_lmul
20023ba5   strcmp
20023bbd   ti_sysbios_BIOS_rtsUnlock__I
20023bd5   ti_sysbios_family_arm_m3_Hwi_Module__startupDone__F
20023bd5   ti_sysbios_family_arm_m3_Hwi_Module__startupDone__S
20023bed   ti_sysbios_family_arm_m3_Timer_Module__startupDone__F
20023bed   ti_sysbios_family_arm_m3_Timer_Module__startupDone__S
20023c05   ti_sysbios_gates_GateMutex_leave__E
20023c1d   xdc_runtime_Error_check__E
20023c35   xdc_runtime_System_exit__E
20023c4d   xdc_runtime_Text_ropeText__E
20023c65   PRCMHIBRegRead
20023c7b   PRCMHIBRegWrite
20023c91   UARTCharGet
20023ca7   _SlDrvMemZero
20023cbd   ti_sysbios_BIOS_exitFunc__I
20023cd3   CPUcpsie
20023ce7   GPIOIntClear
20023cfd   _register_unlock
20023d03   _register_lock
20023d0b   _nop
20023d11   strlen
20023d25   ti_sysbios_family_arm_m3_Hwi_Object__get__S
20023d39   ti_sysbios_family_arm_m3_Hwi_switchFromBootStack__E
20023d39   ti_sysbios_hal_Hwi_HwiProxy_switchFromBootStack__E
20023d4d   ti_sysbios_heaps_HeapMem_Object__get__S
20023d61   ti_sysbios_knl_Swi_Object__get__S
20023d75   xdc_runtime_LoggerBuf_Object__get__S
20023d89   UARTIntClear
20023d9b   __TI_zero_init
20023dad   ti_sysbios_hal_Hwi_Module_startup__E
20023dbf   ti_sysbios_hal_Timer_Module_startup__E
20023dd1   xdc_runtime_LoggerBuf_Instance_finalize__E
20023de3   xdc_runtime_LoggerBuf_write1__E
20023df5   xdc_runtime_LoggerBuf_write2__E
20023e07   xdc_runtime_Startup_exec__I
20023e29   SL_FD_ZERO
20023e39   strcpy
20023e49   ti_sysbios_BIOS_setThreadType__E
20023e59   ti_sysbios_BIOS_start__E
20023e69   ti_sysbios_family_arm_m3_Hwi_getHandle__E
20023e79   ti_sysbios_family_arm_m3_TaskSupport_glue
20023e89   ti_sysbios_family_arm_m3_TaskSupport_swap__E
20023e89   ti_sysbios_knl_Task_SupportProxy_swap__E
20023e91   ti_sysbios_knl_Task_swapReturn
20023e99   ti_sysbios_gates_GateMutex_Instance_finalize__E
20023ea9   ti_sysbios_knl_Mailbox_Object__get__S
20023eb9   ti_sysbios_knl_Semaphore_Instance_finalize__E
20023ec9   ti_sysbios_knl_Swi_disable__E
20023ed9   ti_sysbios_knl_Task_Object__get__S
20023ee9   ti_sysbios_knl_Task_disable__E
20023ef9   xdc_runtime_Gate_leaveSystem__E
20023f09   xdc_runtime_LoggerBuf_write0__E
20023f19   xdc_runtime_Memory_free__E
20023f29   xdc_runtime_SysMin_ready__E
20023f29   xdc_runtime_System_SupportProxy_ready__E
20023f39   xdc_runtime_System_vsnprintf__E
20023f49   xdc_runtime_Text_visitRope__I
20023f59   _SlDrvResetCmdExt
20023f67   __TI_decompress_none
20023f75   _Dclass
20023f83   ti_sysbios_knl_Queue_empty__E
20023f91   NwpMaskInterrupt
20023f9d   NwpUnMaskInterrupt
20023fa9   sl_WlanDisconnect
20023fb5   sl_WlanSmartConfigStop
20023fc1   ti_sysbios_family_arm_m3_Hwi_Params__init__S
20023fcd   ti_sysbios_family_arm_m3_Hwi_disableFxn__E
20023fcd   ti_sysbios_hal_Hwi_HwiProxy_disable__E
20023fcd   ti_sysbios_hal_Hwi_disable__E
20023fd9   ti_sysbios_family_arm_m3_TaskSupport_checkStack__E
20023fd9   ti_sysbios_knl_Task_SupportProxy_checkStack__E
20023fe5   ti_sysbios_family_arm_m3_TaskSupport_getStackAlignment__E
20023fe5   ti_sysbios_knl_Task_SupportProxy_getStackAlignment__E
20023ff1   ti_sysbios_gates_GateHwi_enter__E
20023ffd   ti_sysbios_knl_Queue_Object__get__S
20024009   ti_sysbios_knl_Semaphore_Params__init__S
20024015   ti_sysbios_knl_Task_Params__init__S
20024021   xdc_runtime_Error_init__E
2002402d   xdc_runtime_Gate_enterSystem__E
20024039   xdc_runtime_Memory_calloc__E
20024045   xdc_runtime_Memory_getMaxDefaultTypeAlign__E
20024051   IntMasterEnable
2002406f   xdc_runtime_LoggerBuf_disable__E
20024079   xdc_runtime_LoggerBuf_enable__E
20024083   PRCMRTCInUseSet
2002408b   ti_sysbios_family_arm_m3_Hwi_doSwiRestore__I
20024093   ti_sysbios_family_arm_m3_Hwi_startup__E
20024093   ti_sysbios_hal_Hwi_HwiProxy_startup__E
20024093   ti_sysbios_hal_Hwi_startup__E
2002409b   ti_sysbios_knl_Idle_loop__E
200240a3   UtilsDelay
200240a9   __xdc__init
200240af   __TI_decompress_rle24
200240b5   ti_sysbios_family_arm_m3_Hwi_restoreFxn__E
200240b5   ti_sysbios_hal_Hwi_HwiProxy_restore__E
200240b5   ti_sysbios_hal_Hwi_restore__E
200240bb   ti_sysbios_gates_GateHwi_leave__E
200240c1   ti_sysbios_heaps_HeapMem_isBlocking__E
200240c7   ti_sysbios_knl_Queue_Instance_init__E
200240cd   xdc_runtime_System_Module_startup__E
200240d3   LoggerBuf_instanceStartup
200240d7   ti_sysbios_BIOS_RtsGateProxy_enter__E
200240db   ti_sysbios_BIOS_RtsGateProxy_leave__E
200240df   ti_sysbios_family_arm_m3_Hwi_delete
200240e3   ti_sysbios_family_arm_m3_TaskSupport_Module__startupDone__S
200240e7   ti_sysbios_family_arm_m3_Timer_getMaxTicks__E
200240eb   ti_sysbios_gates_GateHwi_query__E
200240eb   xdc_runtime_LoggerBuf_Module_GateProxy_query__E
200240eb   xdc_runtime_Main_Module_GateProxy_query__E
200240eb   xdc_runtime_System_Module_GateProxy_query__E
200240ef   ti_sysbios_BIOS_RtsGateProxy_query__E
200240ef   ti_sysbios_gates_GateMutex_query__E
200240ef   ti_sysbios_heaps_HeapMem_Module_GateProxy_query__E
200240f3   ti_sysbios_hal_Hwi_HwiProxy_Module__startupDone__S
200240f7   ti_sysbios_hal_Timer_TimerProxy_Module__startupDone__S
200240fb   ti_sysbios_heaps_HeapMem_Module_GateProxy_enter__E
200240ff   ti_sysbios_heaps_HeapMem_Module_GateProxy_leave__E
20024103   ti_sysbios_knl_Clock_TimerProxy_Module__startupDone__S
20024107   ti_sysbios_knl_Clock_TimerProxy_getMaxTicks__E
2002410b   ti_sysbios_knl_Mailbox_delete
2002410f   ti_sysbios_knl_Queue_destruct
20024113   ti_sysbios_knl_Semaphore_delete
20024117   ti_sysbios_knl_Semaphore_destruct
2002411b   ti_sysbios_knl_Task_SupportProxy_Module__startupDone__S
2002411f   ti_sysbios_knl_Task_delete
20024123   ti_sysbios_knl_Task_startup__E
20024127   xdc_runtime_Error_getSite__E
2002412b   xdc_runtime_LoggerBuf_Module_GateProxy_enter__E
2002412f   xdc_runtime_LoggerBuf_Module_GateProxy_leave__E
20024133   xdc_runtime_Memory_HeapProxy_alloc__E
20024137   xdc_runtime_Memory_HeapProxy_free__E
2002413b   xdc_runtime_System_Module_GateProxy_enter__E
2002413f   xdc_runtime_System_Module_GateProxy_leave__E
20024143   xdc_runtime_System_aprintf_va__F
20024147   xdc_runtime_System_printf_va__F
2002414c   xdc_runtime_Text_charTab__A
200258da   _ctypes_
20025c92   xdc_runtime_Text_nodeTab__A
20025d4a   ti_sysbios_family_arm_m3_Hwi_Module__id__C
20025fac   OpcodeTranslateTable
20025fe8   _SlPolicySetCmdCtrl
20025fec   _SlPolicyGetCmdCtrl
20025ff0   _SlProfileGetCmdCtrl
20025ff4   _SlProfileDelCmdCtrl
20025ff8   _SlWlanGetNetworkListCtrl
20025ffc   _SlRxFilterAddtCmdCtrl
20026000   _SlRxFilterSetCmdCtrl
20026004   _SlRxFilterGetCmdCtrl
20026008   _SlSmartConfigStartCmdCtrl
2002600c   _SlWlanSetModeCmdCtrl
20026010   _SlWlanCfgSetCmdCtrl
20026014   _SlWlanCfgGetCmdCtrl
20026024   ti_sysbios_knl_Task_Object__PARAMS__C
20026060   xdc_runtime_LoggerBuf_Module__FXNS__C
200260d4   _SlActionLookupTable
2002610c   _SlFsOpenCmdCtrl
20026110   _SlFsCloseCmdCtrl
20026114   _SlFsReadCmdCtrl
20026118   _SlFsWriteCmdCtrl
2002611c   _SlFsGetInfoCmdCtrl
20026120   _SlFsDeleteCmdCtrl
20026144   g_H2NSyncPattern
2002614c   g_H2NCnysPattern
20026154   RxMsgClassLUT
20026178   _SlSockSocketCmdCtrl
2002617c   _SlSockCloseCmdCtrl
20026180   _SlRecvfomCmdCtrl
20026184   _SlSendCmdCtrl
20026188   _SlListenCmdCtrl
2002618c   _SlAcceptCmdCtrl
20026190   _SlRecvCmdCtrl
20026194   _SlSetSockOptCmdCtrl
20026198   _SlGetSockOptCmdCtrl
2002619c   _SlSelectCmdCtrl
200261ac   ti_sysbios_knl_Mailbox_Object__PARAMS__C
200261e0   ti_sysbios_family_arm_m3_Hwi_Object__PARAMS__C
20026210   xdc_runtime_Startup_sfxnTab__A
2002629c   _SlNetAppStartCtrl
200262a0   _SlNetAppStopCtrl
200262a4   _SlGetServiceListeCtrl
200262a8   _SlRegisterServiceCtrl
200262ac   _SlGetHostByServiceCtrl
200262b0   _SlGetHostByNameCtrl
200262b4   _SlNetAppSetCmdCtrl
200262b8   _SlNetAppSendTokenValueCmdCtrl
200262bc   _SlNetAppGetCmdCtrl
200262c4   ti_sysbios_heaps_HeapMem_Module__FXNS__C
20026312   ti_sysbios_family_arm_m3_Hwi_Module__loggerDefined__C
20026314   ti_sysbios_gates_GateHwi_Module__FXNS__C
20026338   ti_sysbios_gates_GateMutex_Module__FXNS__C
2002635c   ti_sysbios_heaps_HeapMem_Object__PARAMS__C
20026380   ti_sysbios_knl_Semaphore_Object__PARAMS__C
200263a4   xdc_runtime_LoggerBuf_Object__PARAMS__C
200263eb   xdc_runtime_Error_policy__C
2002640c   ti_sysbios_family_arm_m3_Hwi_Object__DESC__C
2002642c   ti_sysbios_gates_GateHwi_Object__DESC__C
2002644c   ti_sysbios_gates_GateMutex_Object__DESC__C
2002646c   ti_sysbios_heaps_HeapMem_Object__DESC__C
2002648c   ti_sysbios_knl_Mailbox_Object__DESC__C
200264ac   ti_sysbios_knl_Queue_Object__DESC__C
200264cc   ti_sysbios_knl_Semaphore_Object__DESC__C
200264ec   ti_sysbios_knl_Task_Object__DESC__C
2002650c   xdc_runtime_LoggerBuf_Object__DESC__C
20026562   ti_sysbios_family_arm_m3_Timer_Module__id__C
2002657c   ti_sysbios_gates_GateHwi_Object__PARAMS__C
20026594   ti_sysbios_gates_GateMutex_Object__PARAMS__C
200265ac   ti_sysbios_knl_Queue_Object__PARAMS__C
200265c4   xdc_runtime_Startup_sfxnRts__A
200265ed   _SlPayloadByProtocolLUT
20026618   xdc_runtime_Startup_firstFxns__A
20026638   StartResponseLUT
20026640   _SlNetCfgSetCmdCtrl
20026644   _SlNetCfgGetCmdCtrl
20026648   ti_sysbios_family_arm_m3_Hwi_excHookFuncs__A
20026650   ti_sysbios_knl_Idle_funcList__C
20026658   xdc_runtime_Startup_firstFxns__C
20026660   xdc_runtime_Startup_lastFxns__C
20026668   ti_sysbios_family_arm_m3_Hwi_E_NMI__C
2002666c   ti_sysbios_family_arm_m3_Hwi_E_alreadyDefined__C
20026670   ti_sysbios_family_arm_m3_Hwi_E_busFault__C
20026674   ti_sysbios_family_arm_m3_Hwi_E_debugMon__C
20026678   ti_sysbios_family_arm_m3_Hwi_E_hardFault__C
2002667c   ti_sysbios_family_arm_m3_Hwi_E_memFault__C
20026680   ti_sysbios_family_arm_m3_Hwi_E_noIsr__C
20026684   ti_sysbios_family_arm_m3_Hwi_E_reserved__C
20026688   ti_sysbios_family_arm_m3_Hwi_E_svCall__C
2002668c   ti_sysbios_family_arm_m3_Hwi_E_usageFault__C
20026690   ti_sysbios_family_arm_m3_Hwi_LD_end__C
20026694   ti_sysbios_family_arm_m3_Hwi_LM_begin__C
20026698   ti_sysbios_family_arm_m3_Hwi_Module__diagsEnabled__C
2002669c   ti_sysbios_family_arm_m3_Hwi_Module__diagsIncluded__C
200266a0   ti_sysbios_family_arm_m3_Hwi_Module__diagsMask__C
200266a4   ti_sysbios_family_arm_m3_Hwi_Module__loggerFxn1__C
200266a8   ti_sysbios_family_arm_m3_Hwi_Module__loggerFxn8__C
200266ac   ti_sysbios_family_arm_m3_Hwi_Module__loggerObj__C
200266b0   ti_sysbios_family_arm_m3_Hwi_NUM_INTERRUPTS__C
200266b4   ti_sysbios_family_arm_m3_Hwi_Object__count__C
200266b8   ti_sysbios_family_arm_m3_Hwi_ccr__C
200266bc   ti_sysbios_family_arm_m3_Hwi_excHandlerFunc__C
200266c0   ti_sysbios_family_arm_m3_Hwi_excHookFuncs__C
200266c4   ti_sysbios_family_arm_m3_Hwi_nullIsrFunc__C
200266c8   ti_sysbios_family_arm_m3_Hwi_priGroup__C
200266cc   ti_sysbios_family_arm_m3_TaskSupport_stackAlignment__C
200266d0   ti_sysbios_family_arm_m3_Timer_E_cannotSupport__C
200266d4   ti_sysbios_family_arm_m3_Timer_startupNeeded__C
200266d8   ti_sysbios_gates_GateMutex_A_badContext__C
200266dc   ti_sysbios_gates_GateMutex_Instance_State_sem__O
200266e0   ti_sysbios_gates_GateMutex_Module__diagsEnabled__C
200266e4   ti_sysbios_gates_GateMutex_Module__diagsIncluded__C
200266e8   ti_sysbios_gates_GateMutex_Module__diagsMask__C
200266ec   ti_sysbios_hal_Hwi_E_stackOverflow__C
200266f0   ti_sysbios_heaps_HeapMem_A_align__C
200266f4   ti_sysbios_heaps_HeapMem_A_heapSize__C
200266f8   ti_sysbios_heaps_HeapMem_A_invalidFree__C
200266fc   ti_sysbios_heaps_HeapMem_A_zeroBlock__C
20026700   ti_sysbios_heaps_HeapMem_E_memory__C
20026704   ti_sysbios_heaps_HeapMem_Module__diagsEnabled__C
20026708   ti_sysbios_heaps_HeapMem_Module__diagsIncluded__C
2002670c   ti_sysbios_heaps_HeapMem_Module__diagsMask__C
20026710   ti_sysbios_heaps_HeapMem_Module__gateObj__C
20026714   ti_sysbios_heaps_HeapMem_Object__count__C
20026718   ti_sysbios_heaps_HeapMem_reqAlign__C
2002671c   ti_sysbios_knl_Clock_LM_begin__C
20026720   ti_sysbios_knl_Clock_LM_tick__C
20026724   ti_sysbios_knl_Clock_LW_delayed__C
20026728   ti_sysbios_knl_Clock_Module_State_clockQ__O
2002672c   ti_sysbios_knl_Clock_Module__diagsEnabled__C
20026730   ti_sysbios_knl_Clock_Module__diagsIncluded__C
20026734   ti_sysbios_knl_Clock_Module__diagsMask__C
20026738   ti_sysbios_knl_Clock_Module__loggerFxn1__C
2002673c   ti_sysbios_knl_Clock_Module__loggerFxn2__C
20026740   ti_sysbios_knl_Clock_Module__loggerObj__C
20026744   ti_sysbios_knl_Clock_tickPeriod__C
20026748   ti_sysbios_knl_Idle_funcList__A
2002674c   ti_sysbios_knl_Mailbox_A_invalidBufSize__C
20026750   ti_sysbios_knl_Mailbox_Instance_State_dataQue__O
20026754   ti_sysbios_knl_Mailbox_Instance_State_dataSem__O
20026758   ti_sysbios_knl_Mailbox_Instance_State_freeQue__O
2002675c   ti_sysbios_knl_Mailbox_Instance_State_freeSem__O
20026760   ti_sysbios_knl_Mailbox_Module__diagsEnabled__C
20026764   ti_sysbios_knl_Mailbox_Module__diagsIncluded__C
20026768   ti_sysbios_knl_Mailbox_Module__diagsMask__C
2002676c   ti_sysbios_knl_Mailbox_Object__count__C
20026770   ti_sysbios_knl_Mailbox_maxTypeAlign__C
20026774   ti_sysbios_knl_Semaphore_A_badContext__C
20026778   ti_sysbios_knl_Semaphore_A_noEvents__C
2002677c   ti_sysbios_knl_Semaphore_A_overflow__C
20026780   ti_sysbios_knl_Semaphore_A_pendTaskDisabled__C
20026784   ti_sysbios_knl_Semaphore_Instance_State_pendQ__O
20026788   ti_sysbios_knl_Semaphore_LM_pend__C
2002678c   ti_sysbios_knl_Semaphore_LM_post__C
20026790   ti_sysbios_knl_Semaphore_Module__diagsEnabled__C
20026794   ti_sysbios_knl_Semaphore_Module__diagsIncluded__C
20026798   ti_sysbios_knl_Semaphore_Module__diagsMask__C
2002679c   ti_sysbios_knl_Semaphore_Module__loggerFxn2__C
200267a0   ti_sysbios_knl_Semaphore_Module__loggerFxn4__C
200267a4   ti_sysbios_knl_Semaphore_Module__loggerObj__C
200267a8   ti_sysbios_knl_Swi_LD_end__C
200267ac   ti_sysbios_knl_Swi_LM_begin__C
200267b0   ti_sysbios_knl_Swi_LM_post__C
200267b4   ti_sysbios_knl_Swi_Module__diagsEnabled__C
200267b8   ti_sysbios_knl_Swi_Module__diagsIncluded__C
200267bc   ti_sysbios_knl_Swi_Module__diagsMask__C
200267c0   ti_sysbios_knl_Swi_Module__loggerFxn1__C
200267c4   ti_sysbios_knl_Swi_Module__loggerFxn4__C
200267c8   ti_sysbios_knl_Swi_Module__loggerObj__C
200267cc   ti_sysbios_knl_Swi_Object__count__C
200267d0   ti_sysbios_knl_Task_A_badPriority__C
200267d4   ti_sysbios_knl_Task_A_badTaskState__C
200267d8   ti_sysbios_knl_Task_A_badThreadType__C
200267dc   ti_sysbios_knl_Task_A_badTimeout__C
200267e0   ti_sysbios_knl_Task_A_noPendElem__C
200267e4   ti_sysbios_knl_Task_A_sleepTaskDisabled__C
200267e8   ti_sysbios_knl_Task_E_spOutOfBounds__C
200267ec   ti_sysbios_knl_Task_E_stackOverflow__C
200267f0   ti_sysbios_knl_Task_LD_block__C
200267f4   ti_sysbios_knl_Task_LD_exit__C
200267f8   ti_sysbios_knl_Task_LD_ready__C
200267fc   ti_sysbios_knl_Task_LM_sleep__C
20026800   ti_sysbios_knl_Task_LM_switch__C
20026804   ti_sysbios_knl_Task_LM_yield__C
20026808   ti_sysbios_knl_Task_Module_State_inactiveQ__O
2002680c   ti_sysbios_knl_Task_Module__diagsEnabled__C
20026810   ti_sysbios_knl_Task_Module__diagsIncluded__C
20026814   ti_sysbios_knl_Task_Module__diagsMask__C
20026818   ti_sysbios_knl_Task_Module__loggerFxn2__C
2002681c   ti_sysbios_knl_Task_Module__loggerFxn4__C
20026820   ti_sysbios_knl_Task_Module__loggerObj__C
20026824   ti_sysbios_knl_Task_Object__count__C
20026828   ti_sysbios_knl_Task_allBlockedFunc__C
2002682c   ti_sysbios_knl_Task_defaultStackHeap__C
20026830   ti_sysbios_knl_Task_defaultStackSize__C
20026834   ti_sysbios_knl_Task_numConstructedTasks__C
20026838   xdc_runtime_Assert_E_assertFailed__C
2002683c   xdc_runtime_Core_A_initializedParams__C
20026840   xdc_runtime_Core_Module__diagsEnabled__C
20026844   xdc_runtime_Core_Module__diagsIncluded__C
20026848   xdc_runtime_Core_Module__diagsMask__C
2002684c   xdc_runtime_Error_E_memory__C
20026850   xdc_runtime_Error_Module__diagsEnabled__C
20026854   xdc_runtime_Error_Module__diagsIncluded__C
20026858   xdc_runtime_Error_Module__diagsMask__C
2002685c   xdc_runtime_Error_Module__loggerFxn8__C
20026860   xdc_runtime_Error_Module__loggerObj__C
20026864   xdc_runtime_Error_policyFxn__C
20026868   xdc_runtime_Error_raiseHook__C
2002686c   xdc_runtime_IFilterLogger_Interface__BASE__C
20026870   xdc_runtime_IGateProvider_Interface__BASE__C
20026874   xdc_runtime_IHeap_Interface__BASE__C
20026878   xdc_runtime_ILogger_Interface__BASE__C
2002687c   xdc_runtime_IModule_Interface__BASE__C
20026880   xdc_runtime_Log_L_error__C
20026884   xdc_runtime_LoggerBuf_E_badLevel__C
20026888   xdc_runtime_LoggerBuf_Module__gateObj__C
2002688c   xdc_runtime_LoggerBuf_Object__count__C
20026890   xdc_runtime_LoggerBuf_statusLogger__C
20026894   xdc_runtime_Memory_defaultHeapInstance__C
20026898   xdc_runtime_Startup_execImpl__C
2002689c   xdc_runtime_Startup_maxPasses__C
200268a0   xdc_runtime_Startup_sfxnRts__C
200268a4   xdc_runtime_Startup_sfxnTab__C
200268a8   xdc_runtime_SysMin_bufSize__C
200268ac   xdc_runtime_SysMin_outputFunc__C
200268b0   xdc_runtime_System_Module__gateObj__C
200268b4   xdc_runtime_System_abortFxn__C
200268b8   xdc_runtime_System_exitFxn__C
200268bc   xdc_runtime_System_extendFxn__C
200268c0   xdc_runtime_System_maxAtexitHandlers__C
200268c4   xdc_runtime_Text_charTab__C
200268c8   xdc_runtime_Text_nameEmpty__C
200268cc   xdc_runtime_Text_nameStatic__C
200268d0   xdc_runtime_Text_nameUnknown__C
200268d4   xdc_runtime_Text_nodeTab__C
200268d8   xdc_runtime_Text_visitRopeFxn__C
200268e0   ti_sysbios_family_arm_m3_TimestampProvider_configTimer__C
200268e2   ti_sysbios_gates_GateMutex_Module__id__C
200268e4   ti_sysbios_hal_Hwi_Module__id__C
200268e6   ti_sysbios_heaps_HeapMem_Module__id__C
200268e8   ti_sysbios_knl_Clock_Module__id__C
200268ea   ti_sysbios_knl_Clock_Module__loggerDefined__C
200268ec   ti_sysbios_knl_Mailbox_Module__id__C
200268ee   ti_sysbios_knl_Semaphore_Module__id__C
200268f0   ti_sysbios_knl_Semaphore_Module__loggerDefined__C
200268f2   ti_sysbios_knl_Swi_Module__id__C
200268f4   ti_sysbios_knl_Swi_Module__loggerDefined__C
200268f6   ti_sysbios_knl_Task_Module__id__C
200268f8   ti_sysbios_knl_Task_Module__loggerDefined__C
200268fa   ti_sysbios_knl_Task_initStackFlag__C
200268fc   xdc_runtime_Core_Module__id__C
200268fe   xdc_runtime_Error_Module__loggerDefined__C
20026900   xdc_runtime_Error_maxDepth__C
20026902   xdc_runtime_LoggerBuf_Module__id__C
20026904   xdc_runtime_LoggerBuf_filterByLevel__C
20026906   xdc_runtime_Memory_Module__id__C
20026908   xdc_runtime_SysMin_flushAtExit__C
2002690a   xdc_runtime_Text_charCnt__C
2002690c   xdc_runtime_Text_isLoaded__C
2002690e   xdc_runtime_Text_registryModsLastId__C
20026910   xdc_runtime_Text_unnamedModsLastId__C
20026918   __TI_static_base__
20027600   __TI_Handler_Table_Base
2002760c   __TI_Handler_Table_Limit
20027618   __TI_CINIT_Base
20027628   __TI_CINIT_Limit
2002bf00   ti_sysbios_heaps_HeapMem_Instance_State_0_buf__A
20036700   g_ucUartAckRxBuffer
20036f00   g_ucUartRxBuffer
20037700   ti_sysbios_knl_Task_Instance_State_0_stack__A
200384a0   g_OtaCheckUpdateResponse
200388ec   xdc_runtime_LoggerBuf_Instance_State_0_entryArr__A
20038cec   xdc_runtime_SysMin_Module_State_0_outbuf__A
200394e8   g_OtaFileMetadata
200398c0   ti_sysbios_family_arm_m3_Hwi_dispatchTable
2003a534   g_StatMem
2003a6ac   cmd_tbl
2003a7fc   sensor_message
2003aa54   __CIOBUF_
2003ab74   gw_scanlist
2003abec   g_CdnClient
2003acc4   gw_scanres_message
2003ad28   gw_context
2003ad84   g_ucDinDout
2003add4   g_OtaApp
2003ae20   g_OtaApp_statistics
2003ae6c   gw_connlist
2003aefc   gw_link_message
2003af30   listcharstr
2003af64   gGapPacket
2003af94   gGattPacket
2003afc4   DeviceRec
2003afec   sch_nvmemload
2003b014   g_OtaClient
2003b038   g_ucConnectionSSID
2003b05c   attWriteReq
2003b076   attReadReq
2003b078   blefiCfgRec
2003b0a8   attReadByTypeReq
2003b0bd   RxIrqCnt
2003b0be   cCountScanDevices
2003b0bf   g_ucPacketEvent
2003b0c0   g_FlcSflashCb
2003b0d4   blefi_mac_string
2003b0e4   gapCentralRoleIRK
2003b0f4   gapCentralRoleSRK
2003b114   bdAddr
2003b11c   bdaddress
2003b124   g_LogClient
2003b12c   g_macAddressVal
2003b134   g_ucConnectionBSSID
2003b13c   gapCentralRoleBdAddr
2003b154   wlan_mac
2003b15c   DMAMsgQ
2003b160   GC_ApiLockObj
2003b168   ReportLockObj
2003b16c   SimpleLinkSpawnTaskHndl
2003b174   blefiCfgData
2003b178   gIntHdlr
2003b17c   gNPI_SyncObj
2003b180   g_GWGenSyncObj
2003b184   g_Mqtt_queue
2003b190   g_cDummy
2003b194   g_rx_task_hndl
2003b198   g_rx_tx_sync_obj
2003b19c   g_wait_secs
2003b1a0   gw_blefi_linke_topic
2003b1a4   gw_blefi_linkt_topic
2003b1a8   gw_blefi_scan_topic
2003b1ac   mqttQStimeout
2003b1b0   mqtt_lib_lockobj
2003b1b4   pGC_StateCB
2003b1b8   pNpiEvtCb
2003b1bc   pcliSyncObj
2003b1c4   sGC_AppMsgQueue
2003b1c8   sGC_StackMsgQueue
2003b1cc   sMsg
2003b1d0   sblFileHandle
2003b1d4   simpleLink_mailbox
2003b1d8   tokenList
2003b1dc   g_ucPacketLen
2003b1dd   g_ucPacketType
2003b1e0   g_gettoken_getchar
2003b7bc   ti_sysbios_family_arm_m3_Hwi_Module__root__V
2003b7c4   ti_sysbios_family_arm_m3_Hwi_Object__table__V
2003b7dc   ti_sysbios_family_arm_m3_Hwi_Module_State_0_excActive__A
2003b7e0   ti_sysbios_family_arm_m3_Hwi_Module_State_0_excContext__A
2003b7e4   ti_sysbios_family_arm_m3_Hwi_Module_State_0_excStack__A
2003b7e8   ti_sysbios_family_arm_m3_Timer_Module__root__V
2003b7f0   ti_sysbios_family_arm_m3_Timer_Module__state__V
2003b7fc   ti_sysbios_family_arm_m3_TimestampProvider_Module__state__V
2003b800   ti_sysbios_gates_GateHwi_Module__root__V
2003b808   ti_sysbios_gates_GateHwi_Object__table__V
2003b80c   ti_sysbios_gates_GateMutex_Module__root__V
2003b814   ti_sysbios_hal_Hwi_Module__root__V
2003b81c   ti_sysbios_hal_Timer_Module__root__V
2003b824   ti_sysbios_heaps_HeapMem_Module__root__V
2003b82c   ti_sysbios_heaps_HeapMem_Object__table__V
2003b844   ti_sysbios_knl_Clock_Module__root__V
2003b84c   ti_sysbios_knl_Event_Module__root__V
2003b854   ti_sysbios_knl_Mailbox_Module__root__V
2003b85c   ti_sysbios_knl_Queue_Module__root__V
2003b864   ti_sysbios_knl_Semaphore_Module__root__V
2003b86c   ti_sysbios_knl_Swi_Module__root__V
2003b874   ti_sysbios_knl_Swi_Module__state__V
2003b890   ti_sysbios_knl_Task_Module__root__V
2003b898   ti_sysbios_knl_Task_Module_State_0_idleTask__A
2003b89c   xdc_runtime_Error_Module__state__V
2003b8a0   xdc_runtime_LoggerBuf_Module__root__V
2003b8a8   xdc_runtime_LoggerBuf_Module__state__V
2003b8b0   xdc_runtime_Memory_Module__state__V
2003b8b4   xdc_runtime_Registry_Module__state__V
2003b8bc   xdc_runtime_Startup_Module__state__V
2003b8c4   xdc_runtime_SysMin_Module__state__V
2003b8d0   xdc_runtime_System_Module_State_0_atexitHandlers__A
2003b8e0   xdc_runtime_System_Module__state__V
2003b8e8   xdc_runtime_Text_Module__state__V
2003b8f0   __xdc__init__addr
2003b8f4   device_hdl
2003b9f0   g_gettoken_scan
2003bab8   g_posttoken
2003bb4e   selfEntity
2003bb50   ti_sysbios_knl_Swi_Module_State_0_readyQ__A
2003bbd0   ti_sysbios_knl_Task_Module_State_0_readyQ__A
2003bc50   g_gettoken_conn
2003bcc8   gw_connect_config
2003bd48   debug_printf
2003bd84   TSK_idle
2003bd84   ti_sysbios_knl_Task_Object__table__V
2003bdd0   mqtt_device_cfg
2003be18   ti_sysbios_knl_Task_Module__state__V
2003be98   ti_sysbios_gates_GateMutex_Object__table__V
2003bed0   ti_sysbios_family_arm_m3_Hwi_Module__state__V
2003bf04   g_gettoken_other
2003bf36   is_notiEnable
2003bf37   is_bleStackReady
2003bf38   ti_sysbios_family_arm_m3_Timer_Object__table__V
2003bf68   ti_sysbios_knl_Swi_Object__table__V
2003bf98   pub_gw_blefi_find_topic
2003bf9c   pub_gw_scanres_topic
2003bfa0   pub_gw_linkeres_topic
2003bfa4   pub_gw_linktres_topic
2003bfa8   MqttIpAcquired
2003bfa9   MqttLibInit
2003bfaa   MqttTopicBuilt
2003bfac   mqttGwMode
2003bfb0   Mqtt_Client
2003bfc4   ti_sysbios_knl_Clock_Module__state__V
2003bff0   net
2003c018   ti_sysbios_BIOS_Module__state__V
2003c03c   xdc_runtime_LoggerBuf_Object__table__V
2003c083   gSblDone
2003c084   charNameMqtt
2003c098   is_slReady
2003c09c   g_ulStatus
2003c0a0   g_ucConnectedToConfAP
2003c0a1   g_ucProvisioningDone
2003c0a2   g_ucPriority
2003c0a3   g_macAddressLen
2003c0a4   g_macAddressGet
2003c0a5   gOutGoingPacket
2003c0a6   gCC2650Packet
2003c0a7   gAckEvent
2003c0a8   is_blefiCfgReady
2003c0a9   is_blefiCfgupdate
2003c0ac   cfgSize
2003c0b0   autoScanTimeout
2003c0b4   g_scanIndex
2003c0b5   g_connIndex
2003c0b6   g_charIndex
2003c0b7   tokenmatch_scan_index
2003c0b8   tokenmatch_conn_index
2003c0b9   tokenmatch_getchar_index
2003c0c0   gNpiReady
2003c0c4   g_uiUartRxBufHead
2003c0c8   g_ucUartReadLen
2003c0c9   g_ucUartByteCount
2003c0ca   g_ucUartReadState
2003c0cb   g_ucUartPacketState
2003c0cc   g_SpiFd
2003c0d0   g_pHostIntHdl
2003c0d4   g_ucDMAEnabled
2003c0d5   g_multi_srvr_conn
2003c0d6   g_ucStartUARTSend
2003c0d8   g_pCB
2003c0dc   pPingCallBackFunc
2003c0e0   gFirstCmdMode
2003c0e4   cli_cmd_count
2003c0e5   gCLIChar
2003c0ec   mqttDevMode
2003c0ee   mqtt_device_connected
2003c0f4   _lock
2003c0f8   _unlock
2003c0fc   __TI_cleanup_ptr
2003c100   __TI_dtors_ptr
2003c104   gapCentralRoleSignCounter
2003c108   gapCentralRoleMaxScanRes
2003c10c   g_uiUartRxBufTail
2003c110   g_ConsecutiveNetAccessNetErrors
2003c114   _Errno
2003c118   main_func_sp
2003cdfc   __stack
2003edfc   __STACK_END
e000e000   ti_sysbios_family_arm_m3_Hwi_nvic
ffffffff   __binit__
ffffffff   __c_args__
ffffffff   binit
UNDEFED    SHT$$INIT_ARRAY$$Base
UNDEFED    SHT$$INIT_ARRAY$$Limit

[1592 symbols]
